:020000040100F9
:1000000038480020E5000001ED000001EF0000018C
:1000100000000000000000000000000000000000E0
:10002000000000000000000000000000F1000001DE
:100030000000000000000000F3000001F5000001D6
:10004000F7000001F7000001F7000001F7000001D0
:10005000F7000001F7000001F7000001F7000001C0
:10006000F7000001F7000001F7000001F7000001B0
:10007000F7000001F7000001F7000001F7000001A0
:10008000F7000001F7000001F7000001F700000190
:10009000F7000001F7000001F7000001F700000180
:1000A000F7000001F7000001F7000001F700000170
:1000B000F7000001F7000001F7000001F700000160
:1000C0000348854600F056F80048004751050001F6
:1000D0003848002040BA7047C0BA70470138FDD197
:1000E000704700000448804704480047FEE7FEE7E9
:1000F000FEE7FEE7FEE7FEE795030001C100000111
:1001000030B50B46014600202022012409E00D46AF
:10011000D5409D4205D31D469540491B2546954037
:1001200040191546521E002DF1DC30BD03460B432D
:100130009B0703D009E008C9121F08C0042AFAD29D
:1001400003E00B780370401C491C521EF9D2704723
:10015000D2B201E00270401C491EFBD2704700225F
:10016000F6E710B513460A4604461946FFF7F0FFB6
:10017000204610BD064C0125064E05E0E36807CC7D
:100180002B430C3C98471034B442F7D3FFF79CFF45
:10019000C0070001D0070001F7B5D4B004460E46F1
:1001A00000205390052052900025002700BFEFF358
:1001B00010800090FF21453101A8FFF7D0FF00F02B
:1001C000F1F905462448854218D1012000038442F4
:1001D00002D1002053902AE001204003844202D142
:1001E0004011539023E003200003844203D10120F7
:1001F000400253901BE0529857B0F0BD174885421B
:1002000013D101200003844201D153900FE001205B
:100210004003844201D1539009E00320000384424B
:1002200001D1539003E05298E6E75298E4E705AF16
:100230000137FF2241320A4901A8FFF777FF012069
:1002400000F04FF93146569A5398B84752900098AB
:1002500000F047F95298CFE7C440130085601300BF
:10026000E8050001F1B58AB0002009907D20C000AA
:1002700008900125AD020027002007907F200690FE
:1002800040240026002005900390200102900020C9
:1002900001903E490A98884206D83D4800686102AC
:1002A00088433B49086006E0394800680121C903DA
:1002B0000843374908607D21C9000A98FFF720FFED
:1002C0007D21C9000090FFF71BFF450100BF3048AA
:1002D00000687F21090288430190200201990843A8
:1002E0002B4908600520FFF7F9FE10E00120FFF719
:1002F000F5FE2748406B02210840002800D007E0A7
:100300000598411C05910899884200D900E0EDE765
:1003100000BF1F48C06B86B2AE4201D9771B00E018
:10032000AF1B0298874203D2E0B20390B8B20290AA
:10033000AE4201D3069400E007940699079840184E
:10034000C005000E04900498A04200D103E0049C74
:1003500009988742BBD800BF0D4800687F21090279
:1003600088430190039800020199084308490860F6
:100370000846406840084000486000BF04484068A4
:10038000042108400028F9D10BB0F0BD0090D00343
:100390000010024010B53E48C0690121090708431A
:1003A0003B49C861812000063A4908633A484861E0
:1003B0003A4808623A48006803218903884338496B
:1003C00008603421374800F073F836480069401C53
:1003D000002803D033480069002817D12C48406812
:1003E0000121090408432A4948600846406807215A
:1003F00009028843264948600846406809150843B1
:10040000234948602848FFF72DFF3FE021488069D5
:100410004409640123480078C006C00E04431D4807
:1004200084611B4800680121C9038843184908609A
:10043000084600687F21090288430446194800697C
:10044000000220431249086008464068012109045F
:1004500008430F494860084640680721090288435D
:100460000B49486008464068091508430849486038
:100470000846006A0D490840054908620846006AB6
:100480000849C968090208430149086210BD000013
:1004900000100240007000400F0800001800020029
:1004A00000100140004000200090D003FF00F8FF42
:1004B00070B504460D462A46214601200003FFF789
:1004C0006BFE70BD02E008C8121F08C1002AFAD1F5
:1004D00070477047002001E001C1121F002AFBD1C4
:1004E000704780F31088704730B502460B460021F4
:1004F000C94312E01078521C414000240BE0480828
:10050000CD07ED0F002D01D0074D00E0002568401C
:100510000146601CC4B2082CF1DB18465B1E0028A3
:10052000E8D1C84330BD00002083B8ED0446012067
:10053000C007204305490863206880F3088800BF8E
:1005400062B66068804700BFFEE7000000700040B0
:10055000114C124D1249206888421AD12821204698
:10056000FFF7C2FFA16A884213D16168022902D154
:100570002146183101E0214608310846074A016842
:10058000914205D3412292040168914200D205684C
:1005900000BF2846FFF7CAFF0040000100800001AD
:1005A00011C011CA70B5D2B00024002500BFEFF30E
:1005B00010800646FF21453101A8FFF7D0FD01ACB0
:1005C00001349822074901A8FFF7B0FD0120FFF789
:1005D00088FFA04705463046FFF783FF284652B004
:1005E00070BD00002807000140BA7047C0BA7047CC
:1005F0000138FDD170470000F7B50325AD06286A24
:1006000082B016460C46400840002862286A022143
:1006100008432862286A8007FCD4662068600127A6
:100620002F61A86AC005FCD5992068602F61A86A6F
:10063000C005FCD5FF209130FFF7DAFFFF2301331F
:10064000AB626846EF60352169602F61A96AC90510
:10065000FCD5AB62A969EF60C9B205226A602F615F
:10066000AA6AD205FCD5AB62AA690902D2B21143CB
:100670000180C80702D0032005B0F0BDAB626869F5
:10068000FF210831884368616869C91E08436861B1
:1006900002980002483068600820A860EE602F6170
:1006A000A86AC005FCD5FF200130A8620023F61C13
:1006B000B0080ED0B2081148006899006054060ACC
:1006C00009194E70060C000E8E705B1CC8709A42A1
:1006D000F1D8FF200130A8626869FF210831884302
:1006E0006861686938436861286A80088000286208
:1006F000286A38432862002005B0F0BD8000000C55
:10070000032080064169FF2208329143416142691A
:1007100001210A434261026A920892000262026A5F
:100720000A43026270470000002003218906096A1B
:10073000490849000322920611621146096A022201
:10074000114303229206116200BF03218906096A40
:10075000022211400229F8D0D101032292069162AF
:100760000321D1609F2151600121116100BF03214C
:100770008906896AFF22013211409142F7D1032292
:1007800092069162114688694969FF2208329143B5
:100790000322920651611146496901221143032245
:1007A000920651611146096A890889001162114651
:1007B000096A012211430322920611627047000068
:1007C000D00700010040002038080000D4040001D8
:1040000011C011CA010000000080000170D800003A
:10401000948E597115000100004002019CD90000E6
:0C40200074EDAEDA150001006719A92448
:106000007ADA12CA01000000F4010000000000006A
:106010000000000000000000000000000000000080
:106020000000000000000000000000000000000070
:04603000773E0CFCAF
:10800000D8B90020698100017181000139B10001F6
:108010000000000000000000000000000000000060
:10802000000000000000000000000000FDB400019E
:1080300000000000000000002781000101B50001E0
:108040007B8100017B8100017B8100017B8100013C
:108050007B8100017B8100017B8100017B8100012C
:108060007B8100017B8100017B8100017B8100011C
:108070007B8100017B8100017B8100017B8100010C
:108080007B8100017B8100017B8100017B810001FC
:108090007B8100017B8100017B8100017B810001EC
:1080A0007B8100017B8100017B8100017B810001DC
:1080B00009B700017B8100017B8100017B81000108
:1080C0000348854601F076F80048004711FC00019E
:1080D000D8B9002040BA7047C0BA70470138FDD106
:1080E0007047000040BA7047C0BA7047704670478A
:1080F000084B19680868203080F30988022080F353
:108100001488BFF36F8F3FBCAE4608BC04BC62B698
:1081100018470000B4470020EFF3108072B6704794
:1081200080F310887047EFF309800E4B1A682038EF
:108130001060F0C044464D4656465F46F0C008B554
:1081400072B60BF083F962B60CBC11680868103087
:10815000F0C8A046A946B246BB4680F3098820383D
:10816000F0C81847B4470020044880470448004737
:10817000FEE7FEE7FEE7FEE7FEE7FEE759B5000192
:10818000C180000130B50B460146002020220124A9
:1081900009E00D46D5409D4205D31D469540491B3B
:1081A0002546954040191546521E002DF1DC30BD84
:1081B00070B500242546002801DA01244042002938
:1081C00001DA01254942FFF7DDFFAC4200D0404211
:1081D000002C00D0494270BDF0B51FB40646002007
:1081E00082B005464024019100901BE0019922468F
:1081F0000F46304600F02DFE049A059B801A9941E7
:1082000010D310461946224600F013FE361A8F414D
:108210000197224601200021009F00F00AFE381835
:108220004D4100902046641E0028DFDC019B009831
:108230002946324607B0F0BD01464139192900D818
:10824000203070470549064A08685043054A80189F
:108250000860400870470149086070470C480020DA
:108260006D4EC6413930000003460B439B0703D0D7
:1082700009E008C9121F08C0042AFAD203E00B78EB
:108280000370401C491C521EF9D27047D2B201E063
:108290000270401C491EFBD270470022F6E710B561
:1082A00013460A4604461946FFF7F0FF204610BD64
:1082B000421C0178401C0029FBD1801A704710B580
:1082C000002200E0521C835C8C5CA34201D1002B95
:1082D000F8D1D8B2E1B2401A10BDC9B203E00378B8
:1082E0008B4203D0401C521EF9D20020704730B59B
:1082F00004460020034600E05B1C934203D2E05C8E
:10830000CD5C401BF8D030BD03460A780270401C9B
:10831000491C002AF9D11846704730B5054600209F
:10832000034600E05B1C934205D2EC5CC85C201A5B
:1083300001D1002CF6D130BD0FB400B58DB009903D
:108340000B9010A900200091C0430A9000200C90CF
:1083500006480690064807906A4609A80F9900F05B
:10836000B1FD0DB008BC04B018470000E58E000157
:10837000058F0001FFB5087889B01546FF2805D0A4
:10838000491C2D2804D00022002407E000240BE023
:108390000122F9E70A235C430419491C0878FF28E5
:1083A000F8D1002A00D06442002004902A780146C7
:1083B0002D2A01D02B2A0FD16D1C2D2A02D000228C
:1083C000049209E00122FBE700260A2233466D1CD5
:1083D00000F0F2FC381871412F78FF2FF4D10C9A7D
:1083E000A218069202460A4304D0FF23069A91334C
:1083F000DA4205DA002109980A4606C00DB0F0BD40
:108400000024B74AB54D2646079200F011FC0290B1
:1084100006980391002801DA474200E00746390533
:108420000020AF4A001C51410191009012E0F80772
:1084300007D022462B463046079900F0D9FA064667
:10844000079122462B461046194600F0D1FA044601
:108450000D467F10002FEAD10698019B0028009A54
:108460000399029806DA00F02BFB3246079B00F0D6
:1084700027FB05E000F0BCFA3246079B00F0B8FA93
:10848000049A002A02D00122D2075140099A03C25D
:10849000B4E7FFB591B0002009900025ED432E20F0
:1084A0009E685C681F460190B9696D1C12988847E8
:1084B0000090396A88470028F6D10098401C0AD0FD
:1084C0000D20C0018443002E12DD00982B2809D016
:1084D0002D280DD103E00020C04315B0F0BD0120D0
:1084E00080020443B9696D1C12988847761E00907B
:1084F00003A9600501D52D2000E02B206A461073EA
:10850000491C0CA80F9102900AE0B9696D1C1298E1
:10851000884700900120400204431398761E0560AE
:10852000002E02DD00983028EFD001990098884293
:1085300046D18020044308E00998401E099001209C
:10854000400204431399681C0860B9696D1C761ECB
:108550001298884700903028EED031E00199884287
:1085600005D1200603D480200443761E1EE0009827
:1085700003F0D8FA002826D001204002044307A9BE
:108580000F980331761E88420BD200980F9930382D
:1085900008700F98401C0F90200607D50998401EC0
:1085A00003E0200602D40998401C0990A00502D5DA
:1085B0001399681C0860B9696D1C1298884700906F
:1085C000002ECBDC59E0002E57DD0098652801D045
:1085D000452852D1A00550D5032000028443B96933
:1085E0006D1C761E129888470090002E0CDD2B28FB
:1085F00004D02D2808D1FF2001300443B9696D1C37
:1086000012988847761E0090E00501D52D2100E0E4
:108610002B21029801700298401C0290019025E0E5
:108620000120400204430EA902980131761E8842BF
:108630000ED20098029930380006000E087003D15F
:108640000299019881420AD90298401C029006E0E2
:10865000E00501D5234801E0224840420990B9696C
:108660006D1C12988847009013980560002E04DD59
:10867000009803F057FA0028D2D1F9691298884778
:108680000F99FF200870029903AA087000200A9031
:108690000B900CA90AA8099BFFF76CFEA00502D459
:1086A0000120C04319E72420044209D0E00713D178
:1086B00038680B9A0A99031D3B60006806C00BE0FE
:1086C0000B990A9800F05CFB0146E00704D138687A
:1086D000021D3A60006801602846FEE60000144072
:1086E0000000F03FF1D8FFFFF7B582B00F4600263B
:1086F000029C03F003F90090006801902578641C47
:10870000002D05D000F0CAFB0068405DC007F5D120
:108710002B2D02D02D2D1CD0641E0098002101604D
:1087200039462046049A00F0FFFB0146002F04D092
:108730003868A04201D10298386000980068022889
:108740000BD00098019A0260700506D5484205B02A
:10875000F0BD012080020643DFE70846F7E7F8B5E1
:1087600002464A40D40F42004B0052085B089A422E
:1087700002D20246084611464A0023D0C30D4A00E1
:10878000DDB2120EAD1A202D35DA49020126490A52
:10879000F6058A19002C00D0524220214F1B1146A9
:1087A000B9402A411018C20D9A4221D0002C17D08E
:1087B000012D08DCDA05801AD20F8019D207DBB24E
:1087C00000F060FCF8BDDA05801A012340001B06AA
:1087D000C01880185A428018CA0F1043490007E099
:1087E0004908C2071143DA05801A80194008801829
:1087F00000F040FCF8BD61000122511A001BF7E7B0
:108800000122D2075140AAE70122D2075040A6E731
:10881000024670B54A40D30FDB0740002DD04A0016
:108820002AD0010E140E000212020919400A520A3F
:108830008418E50104465443000A120A2E045043EA
:10884000A4194219200CC543AA18120C0125AD0326
:10885000521C521912047F39240400D0521C1043B8
:1088600001D44000491EC2B20C06C0092018401CA9
:108870004008802A02D003E0002070BD400840007C
:10888000002900DA0020184370BD0000F0B507464B
:108890000846584087B0C00F049048000E46590063
:1088A00040084908BC1A884105D2384631461E4660
:1088B00017460B4602465800400810434CD0300D76
:1088C000039040055900400D490D0590401A029053
:1088D000402872DA18030121000B090508430190B2
:1088E00004980092002805D0019952420020884146
:1088F00000920190029840210A1A0199009800F014
:1089000098FA05460C466B4607CB00F0B3FAC0193F
:108910007141039A0E0D0023D71756401A467A402C
:10892000164344D0049A002A2DD0029A012A039AB1
:1089300015DC1205C01A914101263605001C714153
:10894000D20F059ED2070093019202962A46234633
:1089500000F0DEFB07B0F0BD38463146FAE71605F9
:10896000224A0F46B218C01AB74101210905001C5E
:108970004F4100187F41114618187941E20F10430A
:108980006D19644113E0E2076D0815436408C207DE
:108990001443039A01261205C01A91413605001CA2
:1089A0007141CE07400830434908C01851412A465A
:1089B000234600F0A0FBCDE7FFE70498012240002A
:1089C000C117121A00238B4104983146C417381A74
:1089D000A141EEE730B40124E407634030BC55E721
:1089E00030B40124E407614030BC4FE70000E0FFF1
:1089F000F0B51FB488B00B99099800244840099934
:108A0000C00F490049080991C0070B99009049001F
:108A100049080B9109990898A64608431CD00B9960
:108A20000A98084318D0099801244000420D4800D4
:108A3000410D099824050003000B204309900B9871
:108A40000003000B20430B9050181C4940180022D3
:108A500001901446104605E0002001460DB0F0BD1F
:108A6000032801DA034600E003239C46C11A0AAE3C
:108A70000AE05F0008ADED5B4F00F75B7D43002728
:108A8000AA187C41491C5B1E6145F2DD410004AB24
:108A90005A522104120C0A43240C401C0828DFDB24
:108AA000019802900099704601910090059B049AEC
:108AB0000799069800F02CFBD0E700000DFCFFFFA3
:108AC000F0B50C465C4085B0E40FE40703944C001D
:108AD000002664085900944649080246029622433B
:108AE00021D062460A431ED06200570D4A000E0391
:108AF0002303550D012402462C492405781B1B0B2A
:108B0000360B401823432643614600901C46501AFA
:108B1000B44103D30098401C009002E092180098E2
:108B20005B41002803DA0020014605B0F0BD0020BB
:108B3000012109050746864611E064461D46141BBF
:108B4000B54106D36546521BB341744607430C43F7
:108B5000A646CD0740084908284392185B410546C0
:108B60000D43EAD11046184313D0604619465040D1
:108B70007140084306D06046101AB34106D2012264
:108B8000002306E000220123DB0702E00122D2439A
:108B90005310009874460105381C6141029C039DE6
:108BA0000019694100F0A7FABFE70000FD030000CB
:108BB00070B54B005B0803430BD04B005C0D0026E7
:108BC00033466542B341D417AD1AA34102DB0020FE
:108BD000014670BD12053018514170BD10B500221C
:108BE0009623114600F04EFA10BD00000EB5C217D4
:108BF000C10F5040CA0740180021054B0293019253
:108C000000910A460B4600F083FA03B000BD000055
:108C1000330400000EB505490291002100910A4677
:108C20000B46019100F074FA03B000BD330400005C
:108C30000EB5054A0292002200921346019200F0FE
:108C400067FA03B000BD000033040000C20F41000A
:108C500040020123400ADB05D207090EC0187F2914
:108C600001DA00207047962903DC9623591AC84080
:108C700001E096398840002AF4D040427047000055
:108C800070B5CD0F4A0009030123090B1B051943D9
:108C90000B4BED070024520D9A4201DA002070BD03
:108CA000074B34339A4203DC9A1A00F0D2F802E000
:108CB0000449511888402C43F1D0404270BD000057
:108CC000FF030000CDFBFFFF4A0009030123090B4E
:108CD0001B0519430A4B10B5520D9A4202DA0020C7
:108CE000014610BD064B34339A4203DC9A1A00F059
:108CF000B0F810BD034BD21800F09BF810BD000077
:108D0000FF030000CDFBFFFFC20FD2074000400869
:108D10000BD0C10D0723DB01C91840020905400A29
:108D20001143C208400711437047002001467047B5
:108D300010B5002904DB0124E40740428C412146A0
:108D4000002B04DB1C460123DB075242A3418B426C
:108D500000D1824210BD000010B5002904DB0124BF
:108D6000E40740428C412146002B04DB1C460123D2
:108D7000DB075242A341994200D1904210BD00004E
:108D8000CB0FDB07490010B5490802460A4307D05C
:108D90000A0D07240903E401090B121B002A01DC58
:108DA000002010BDC900440F0C43C100E018D205DB
:108DB000801800F05FF910BDF0B51FB486B0002038
:108DC0000090019002900698069980B2049007984E
:108DD000090C02040014114307900027089D09980C
:108DE00006913E463C4603900398A9B20204000C4B
:108DF000039004982D0C154348430021224600F0AF
:108E000018F8C719714110340E46402CECDB384677
:108E1000029A00F00EF8009A019B801800905941C8
:108E200002980191103002904028CCDB00980BB0E2
:108E3000F0BD10B5202A04DB0146203A9140002005
:108E400010BD914020239C1A0346E34019439040F3
:108E500010BD10B5202A04DB0846203AD04000217E
:108E600010BD0B46D340D0402024A21A91400843A5
:108E7000194610BD10B5202A06DBCB170846203A4C
:108E80001041C1170B4306E00B461341D04020248C
:108E9000A21A91400843194610BD000000487047CF
:108EA000604D010110B50446FFF7F8FF0068005D52
:108EB000C007C00F10BD0000026813785118016090
:108EC0001846704710B5D1600449516104491162D8
:108ED00000211161114600F08FF910BDB98E00011B
:108EE000A58E00014268002A08D001680B78491C51
:108EF000002B03D0521E06C0184670470121C160E6
:108F0000881E70474268002A0BD0C3680168002B96
:108F100007D183688B4204D0491E521C06C0002032
:108F200070470020C0437047F7B582B0029C00270D
:108F30002078641C15460197302802D0002D15D0EA
:108F400015E020780127641C782804D0582802D026
:108F5000002D09D00BE0002D01D0102D07D10027E6
:108F600010252078641C02E0082500E00A25002670
:108F7000009610E00099012769430818020C294661
:108F800080B2714300908E183804864201D30120CC
:108F900001902078641C294600F01EF90028E9DAC7
:108FA0000398002805D0002F01D0641E00E0029C29
:108FB00004600198002806D002F0A0FC02210160A4
:108FC000C81E05B0F0BD009930040843F9E7000061
:108FD0000FB400B589B00CA900910B990023CB60A8
:108FE000204B214A06930792042201921F4A0292C3
:108FF0001F4A089202466B460020FFF74AFA09B062
:1090000008BC04B0184770B586B006460020C043BF
:109010000190002015460C460091029104903246C2
:10902000694604A8FFF7D4FF024604982118002DD2
:1090300005D0002801D0084600E0204628600498AA
:1090400000280DD0002A02DD0098884208D0081BB5
:109050000190009432466946029404A8FFF7B8FFD5
:1090600006B070BDE58E0001058F0001FFFFFF7F98
:10907000A58E0001002904DA401C490001D14008F6
:109080004000704770B40024050C05D11024000482
:1090900002D1002921D01124050E01D1000208348B
:1090A000050F01D10001241D850F01D18000A41CF2
:1090B000002801DB4000641C002908D020252E1B5D
:1090C0000D46F540A14000D0012129430843010687
:1090D0001B1B000ADB1D02D5002070BC7047DB059E
:1090E000181880180029F8DA401C4900F5D170BC26
:1090F00040084000704710B5002B08DA0024401CDF
:10910000614192185B411A4301D14008400010BDF3
:10911000F0B51FB482B005460C0003D0084602F03B
:10912000D5FB02E002F0D2FB20300246009021463F
:109130002846FFF77EFE049B059A04460F46184317
:109140001143084314D0184610431BD00098402107
:109150000A1A18460599FFF77CFE05460E46009A46
:1091600005990498FFF765FE084305D0012004E047
:109170002046394607B0F0BD0020C11705430E4315
:109180002C43374300990E986305401A7905E40A89
:1091900000220C43FD0A0A3002D500200146E9E70F
:1091A0000105101969410C9C0D9D00196941FFF7DB
:1091B000A2FFDFE7064C0125064E05E0E36807CC79
:1091C0002B430C3C98471034B442F7D3FEF77CFF96
:1091D0003C5201015C5201013A2800D23038202370
:1091E00002469A43412A01D310463738884201D3B8
:1091F0000020C04370470000F3B58DB000200A90F6
:1092000001200B90002608460C300C46099062693C
:10921000012109989047051E2ED0252D2DD0216AB9
:109220008847002818D06269012109989047216A6F
:1092300088470028F7D1411E62690998904700E0ED
:10924000761CA1690D988847216A88470028F7D1C4
:10925000E1690D988847DAE7A1690D9888470746C4
:10926000A84201D1761CD2E7E1690D9888477F1C9E
:1092700002D10A98002877D049E1002762693D466B
:109280003946099890472A280CD16269012109982A
:109290009047012506E00A214F433F18303FEBD4A9
:1092A0001020054362690121099890470146303931
:1092B0000A2903D29B498F42DEDCECE7E90600D4A1
:1092C000994F6C280AD04C2810D0682824D06A28DE
:1092D0002ED074280CD07A280AD00DE062690121C2
:1092E000099890476C2823D004211CE020200543D6
:1092F0006269012109989047A760656065284FD091
:1093000026DC582839D01ADC452849D012DC25281B
:1093100034D04128B0D143E06269012109989047D7
:10932000682802D008210D43E6E70120C002DEE7ED
:109330000220DCE7462833D047282CD130E05B28D8
:1093400070D061282CD063286CD0642823D161E0D0
:109350006F284FD009DC662822D0672820D06928E2
:1093600026D06E2817D12EE0CDE070284DD073287E
:109370006FD075284ED078280DD154E0A1690D9892
:1093800088470546252800D16CE7E1690D98884794
:109390006D1C00D16DE7BAE00A224CE00A2252E0CF
:1093A000012023466A46C0430D99FFF772F8A3E0F7
:1093B0002846402108436060A807234601D50022C3
:1093C00039E000223FE0E80700D020E72068011DD7
:1093D00021600068290501D5067018E7290701D525
:1093E000068014E7A90703D5F117066041600EE770
:1093F00006600CE72846402108436060A807234622
:1094000001D5082217E008221DE0484928460840F7
:10941000606016E02846402108436060A8072346A4
:10942000BCD5B9E715E02846402108436060A8078D
:1094300007D5234610220120C0430D99C046C046DF
:109440005AE0234610220120C0430D99C046C04671
:1094500052E000210C910B460091632802D05B285A
:1094600007D043E0E80601D40120A060012000906D
:109470003CE062690121099890475E2805D10120EE
:109480000C9001466269099890472169002906D12C
:109490000B4601AA8F00491CD3510829FADB00288A
:1094A00035D0216900290ED1C117C90E09184A11FA
:1094B000930001AA9A1849094901411A0120136829
:1094C00088400343136062690121099890475D2831
:1094D000E5D10C98002808D0002001AB81005A5833
:1094E000401CD2435A500828F8DB01AB0120224629
:1094F000C0430D99C046C04600280ADA401C06D178
:109500000B98002803D00020C0430FB0F0BD0A988C
:10951000FBE7E90702D10A99491C0A913618002095
:109520000B9074E6CCCCCC0CFFFFFF7FF1F7FFFF74
:1095300070B58D180478401CA207920F01D10278F3
:10954000401C231106D10378401C03E006780E70FE
:10955000401C491C521EF9D1002B15D002780C2654
:109560008A1A3440401C0C2C03D0A401121B9B1CF3
:1095700008E004782402121B401CF8E714780C70F1
:10958000491C521C5B1EF9D5A942D3D3002070BDE3
:1095900003B40148019001BD232A000003B401482F
:1095A000019001BD6D56000003B40148019001BD5A
:1095B0006560000003B40148019001BDAF7F000069
:1095C00003B40148019001BDB551000003B4014846
:1095D000019001BDD37E000003B40148019001BD9C
:1095E000697E000003B40148019001BDC37F000003
:1095F00003B40148019001BDE954000003B40148DF
:10960000019001BD9957000003B40148019001BDCC
:10961000ED57000003B40148019001BD1D7C00001E
:1096200003B40148019001BD0D2A000003B40148B4
:10963000019001BDAB52000003B40148019001BD8F
:10964000F58F000003B40148019001BDE1FE000068
:1096500003B40148019001BD250E010003B4014887
:10966000019001BDB143000003B40148019001BD68
:1096700085290000C943416070470268702392B297
:109680009A430A430260704770B5044602F024F81A
:10969000002818D08069002815D0FFF79FFA0546EA
:1096A0002046FFF79BFA2946FFF7AEF8FFF72CFBA1
:1096B000064A074BFFF704FA0022064BFFF7E6F8CD
:1096C000FFF75EFB70BD044DEAE700001F85EB511C
:1096D000B81E01400000394000803B4470B50D4683
:1096E0000646002401F0F8FF002816D0C1690029C1
:1096F00013D0026A002A10D08BB290B289B292B213
:10970000102D0CD0202D0AD0302D17D0402D15D083
:10971000502D13D0602D11D022E0002070BD891A89
:10972000B01AAF2292005043FEF742FD0446963431
:109730000FD47D20C000844211DC11E0191AAF2241
:10974000301A12015043FEF733FD4B21C900441873
:1097500001D5002404E0E1200001844200DD04463C
:10976000204670BD70B5104CA0421BD1851401215C
:10977000284601F063FE0021284601F05FFE01212A
:10978000284601F04FFE09486061002020606060BB
:109790001F21A16006492161A06160622062A06270
:1097A0000448E06170BD000000080240080A0200A1
:1097B0000000FC0F2E6D00000029016802D001227C
:1097C000114301E049084900016070470422002963
:1097D000816902D0114381617047914381610848DA
:1097E0000649C1620749016307494163074981632B
:1097F0000749C1630849074808607047220078009C
:1098000000080240E700E1009F00BF04190C0516A4
:1098100070206E286E2B00004008024002220029B2
:10982000016801D0114300E0914301607047C068B6
:1098300080B270470246526800200A4200D00120E0
:1098400070470000044A9068C90640094001C90EEB
:1098500001439160704700000008024070B5054662
:1098600049480C464EC88CB0039602930192009171
:109870004EC8079606930592049142680168806875
:10988000099208910A90414A00996846914217D17D
:10989000282104F043FA0A99884211D1022D1ADBDB
:1098A0000020646802460B900BA92046FEF71CFFBF
:1098B00005460B98A04209D00078002806D101E0A7
:1098C00033A004E0012D0AD0022D08D03EA004F000
:1098D00023FB0CB070BD0198012809D00125019827
:1098E000A84207D1294647A004F0B0FA0CB070BDD9
:1098F0000225F4E7012D6C4614D01834012D13D045
:1099000047482268824206D16068002803D00721B8
:10991000890388420AD9294642A0636804F096FA6E
:109920000CB070BD0834E9E74C48EAE74CA004F0FD
:10993000F3FA6168206804F0F1F9A268824206D067
:1099400003462946544804F081FA54A0BFE729464B
:109950005FA06368E26804F079FA6846019503F055
:10996000FDFD002801D06AA0B1E76EA004F0D4FA92
:10997000C82009F061FCBFF34F8F72497048C8607E
:10998000BFF34F8FFEE700000040000111C011CA75
:1099900061707073773A20626F6F74736574746965
:1099A0006E67207265636F726420696E76616C69A0
:1099B000642C2072656675736520746F20737769F7
:1099C0007463680D0A00000075736167653A206171
:1099D00070707377205B317C325D20286E6F206160
:1099E0007267203D2073776974636820746F2074F8
:1099F0006865206F746865722062616E6B290D0A5C
:109A00000000000061707073773A20616C726561CC
:109A10006479206F6E20415050256C750D0A00004E
:109A20000040020161707073773A2062616E6B25AD
:109A30006C75207265636F726420696E76616C6903
:109A4000642028616464723D30782530386C582079
:109A500073697A653D256C75290D0A000080000147
:109A600061707073773A20766572696679696E679E
:109A70002074617267657420696D61676520637227
:109A8000632028666577207365636F6E6473292E83
:109A90002E2E0D0A00000000A851010120202020D8
:109AA00020202072756E20424C45204F5441207476
:109AB0006F20777269746520612076616C6964201B
:109AC000696D6167652066697273740D0A00000034
:109AD00061707073773A2062616E6B256C752069D6
:109AE0006D616765206F6B20287665722030782560
:109AF00030386C582C20256C752042292C20737727
:109B000069746368696E672E2E2E0D0A00000000CE
:109B100061707073773A20666C6173682066616962
:109B20006C0D0A0061707073773A20646F6E652C5B
:109B300020726573657474696E672E2E2E0D0A008F
:109B40000400FA0500ED00E010B50B488CB01EC80B
:109B500003940293019200911EC807940693059204
:109B600004914268016880680A90099208916846E9
:109B700003F022FD0CB010BD00400001F0B58DB027
:109B80000E46032807DA54A004F0C6F95AA004F0E0
:109B9000C3F95F480FE00024B76822460BA9384696
:109BA0000B94FEF7A1FD05460B98B84202D0007851
:109BB000002804D057A004F0AFF90DB0F0BD5A4B07
:109BC00087CB039702920191009087CB079706926B
:109BD000059104909A68596818680A920991534A45
:109BE000009908906846914205D1282104F096F822
:109BF0000A9988420DD0009401940294039404942D
:109C00000594069407940894099449A00A9404F0D2
:109C100083F955A17068FEF752FB002804D07068E4
:109C20000178622908D02BE0012D03D0022D01D04C
:109C30004FA0C0E701953AE04178312902D032299E
:109C400002D01DE002AC00E006AC51A1801CFEF782
:109C500036FB002816D070684FA1801CFEF72FFB42
:109C6000002819D070684EA1801CFEF728FB002840
:109C70001AD070684BA1801CFEF721FB002815D07C
:109C800049A098E74E48854204D04E48854201D00D
:109C90004DA090E725600AE007208003854201D9A6
:109CA00058A088E7656002E0A56000E0E5602A460C
:109CB0005DA0716804F0CAF8684603F04FFC002804
:109CC00001D062A077E766A004F026F9684603F0A9
:109CD00073FC0DB0F0BD000075736167653A2062DA
:109CE00073736574203C6669656C643E203C7661E4
:109CF0006C3E0D0A0000000020206669656C643A25
:109D000020616374697665203C317C323E0D0A0027
:109D1000F051010162737365743A206261642076C8
:109D2000616C75650D0A00000040000111C011CA88
:109D300062737365743A206578697374696E67201D
:109D40007265636F726420696E76616C69642C2041
:109D500072656275696C642066726F6D20736372E0
:109D6000617463680D0A00006163746976650000C0
:109D700062737365743A20616374697665206D75EA
:109D800073742062652031206F7220320D0A00004A
:109D9000616464720000000073697A65000000006D
:109DA000637263007665720062737365743A20753E
:109DB0006E6B6E6F776E206669656C640D0A0000CD
:109DC000008000010040020162737365743A2061F3
:109DD000646472206D757374206265204341494943
:109DE000435F415050315F42415345206F722043E1
:109DF000414949435F415050325F424153450D0A4A
:109E00000000000062737365743A2073697A6520FC
:109E100065786365656473207468652062616E6B44
:109E20002073697A650D0A0062737365743A2025A0
:109E300073203D2030782530386C582C207772699B
:109E400074696E672E2E2E0D0A0000006273736512
:109E5000743A20666C617368206661696C0D0A0053
:109E600062737365743A206F6B2028766572696639
:109E7000696564290D0A000000B583B00021032044
:109E80000B46012201910090920203A1034809F0C0
:109E900049FE03B000BD0000434C4900A5A20001EB
:109EA00010B5022805DB48680DA1FEF708FA002866
:109EB00005D00D480078002804D00CA103E007F07D
:109EC0009FF910BD0BA110A003F0C0FF124C13A00E
:109ED000218903F0BBFF1CA0E16803F0B7FF10BDB0
:109EE0006A736F6E000000009847002076616C690D
:109EF0006400000064656661756C7420286E6F7480
:109F00002073617665642900706172616D733A2017
:109F100025730D0A00000000B45E002020206C654F
:109F200064203D2025752020286C65643120626CFA
:109F3000696E6B2068616C6620706572696F642C55
:109F4000206D73290D0A0000202070776D203D20C0
:109F5000256C7520202870776D20647574792C200D
:109F60002525290D0A000000F3B595B015980D467A
:109F7000032807DA6F4803F0CFFF6FA003F0CCFF90
:109F800079A023E07FA16868FEF799F9002810D036
:109F90000020AE680246009069463046FEF7A4FBFA
:109FA00004460098B04202D0007800287BD077A009
:109FB0000CE000240226B00014902858FEF778F92F
:109FC0000746E019801C502804D975A003F0A4FFAF
:109FD00017B0F0BD002C03D0202069460855641C42
:109FE00014983A46295868460019FEF73DF9159825
:109FF000E419761C8642DEDB002069460855451EC2
:10A000006E462C4605F0B2FC304603F0DDFD06003E
:10A0100023D003F0BEFD00281FD069A1304603F015
:10A0200081FD074603F0ACFD002800D07D6965A1E5
:10A03000304603F077FD074603F0A2FD002800D06C
:10A040007C69002D13DA002C22DA5FA003F064FF94
:10A05000304603F03DFD17B0F0BD65A003F05CFF96
:10A06000002EF8D0304603F033FD17B0F0BD29467E
:10A0700066483239814209D3654A322165A003F02E
:10A08000E5FE304603F024FD17B0F0BD002C0BDBDD
:10A09000642C09DD642164A003F0D8FE304603F08F
:10A0A00017FD17B0F0BD14E0304603F011FD002D90
:10A0B00001DB62480581002C01DB6048C46007F0C9
:10A0C000F3F8002801D05EA080E707F099F817B0F8
:10A0D000F0BD3BA16868FEF7F2F8002807D039A16F
:10A0E0006868FEF7ECF800280DD05CA06EE720460B
:10A0F00046493238884203D3454A322145A015E00B
:10A100004E48048109E0642C05D9642146A003F07F
:10A110009DFE17B0F0BD4948C46007F0C5F800289F
:10A1200001D055A052E7224659A0696803F08EFE7F
:10A1300017B0F0BD6451010120206C6564203D2002
:10A140006C65643120626C696E6B2068616C66209E
:10A15000706572696F642035302E2E3130303030AA
:10A16000206D730D0A000000202070776D203D20C7
:10A1700070776D206475747920302E2E3130302048
:10A18000250D0A006A736F6E000000006170707325
:10A1900065743A206261642076616C75650D0A0011
:10A1A000617070736574206A736F6E3A206C696EAB
:10A1B0006520746F6F206C6F6E670D0A00000000E1
:10A1C0006C65640070776D00617070736574206AEF
:10A1D000736F6E3A206E6F206B6E6F776E206B65BB
:10A1E0007920286C65642C2070776D290D0A000099
:10A1F000617070736574206A736F6E3A207061725B
:10A200007365206661696C0D0A000000DF2600009E
:10A21000102700006C65642072616E6765202575EB
:10A220002E2E25750D0A000070776D2072616E6705
:10A230006520302E2E25750D0A000000B45E00202A
:10A24000617070736574206A736F6E3A20666C611A
:10A250007368206661696C0D0A000000756E6B6E94
:10A260006F776E20706172616D20286C65642C20A0
:10A2700070776D290D0A00006170707365743A2063
:10A28000666C617368206661696C0D0A00000000ED
:10A290002573203D20256C752C2073617665640D37
:10A2A0000A000000002498B0F8A527461594661E01
:10A2B00028461294FDF7FCFF81B2284603F046FBC6
:10A2C000FE4800258078002839D06421684603F0D4
:10A2D0009DFA002816D06846007802F037FE002864
:10A2E0000ED0F6490020887003F00EFBF4A5284636
:10A2F000FDF7DEFF81B2284603F028FB03F014FBD4
:10A30000002518E0643502F071FDF748854212D34C
:10A31000EA490020887002F069FD02F05DFD03F05B
:10A32000F3FAF2A00190FDF7C3FF81B2019803F0A8
:10A330000DFB03F0F9FAE14880780028C5D100212F
:10A34000C943684603F062FA0028B9D0159800287E
:10A3500005D000211591694609788142B0D0129844
:10A3600001281FD0022826D0684600781B287DD0FF
:10A3700009287CD00D287BD00A287AD0082879D0EB
:10A380007F2877D0014620395F2999D23F2C72D29D
:10A39000E1490855641CA4B20121684603F0D6FACD
:10A3A00027468DE7684600785B2802D0002012908F
:10A3B00086E70220FBE700201290684600784128DB
:10A3C00016D04228EDD1002EEBDB761E57D4BB48C9
:10A3D0004078801BC01DC117490F0918C908C90062
:10A3E000401A8101CD4809184038FDF78DFF49E03A
:10A3F000B248711C02789142D3DA4078761C801BF7
:10A40000C01DC117490F0918C908C900401A8101A8
:10A41000C24809184038FDF777FFBF480290FDF7A2
:10A4200047FF85B2BEA42046FDF742FF81B2204619
:10A4300003F08CFA0024002F0BD9BCA00190FDF78B
:10A4400037FF81B2019803F081FA641CA4B2BC42C8
:10A45000F3D3B3A42046FDF72BFF81B2204603F0CF
:10A4600075FA002D34D02946029805E036E038E030
:10A47000E2E0E3E081E18EE103F068FA28E0A6493A
:10A4800000200870A4480290FDF712FF85B2A4A432
:10A490002046FDF70DFF81B2204603F057FA002455
:10A4A000002F0BD9A1A00190FDF702FF81B2019806
:10A4B00003F04CFA641CA4B2BC42F3D398A4204627
:10A4C000FDF7F6FE81B2204603F040FA002DCAD116
:10A4D0002F469148FDF7ECFE84B2F1E60120129080
:10A4E000EEE603F011FA8C4800252F46019003F0A8
:10A4F00044FC1390224620210198FDF7EEFE00282F
:10A5000060D1019908551399149000295AD91498CB
:10A5100003F036FC224616900199FDF7FEFE002856
:10A5200019D1002F0AD102A81699FDF7EDFE02A855
:10A53000FDF7BEFE85B20DE06D1EADB2A54206D997
:10A540002A4602A81699FDF7E8FE0028F4D100215A
:10A5500002A841557F1C14981399401C14908842FE
:10A56000D5D3002F64D0012F1AD0A5422BD902AF2A
:10A570003F2C5DD2AC425BD23819012103F0E6F9E1
:10A580000198395D0155641CA4B2F1E73819012125
:10A5900003F0DCF90198395D0155641CA4B200E0B8
:10A5A00002AF3F2C44D2AC42F0D301992020085591
:10A5B000641C5EA5A4B22846FDF77AFE81B2284647
:10A5C00003F0C4F934E05AA52846FDF771FE81B2C4
:10A5D000284603F0BBF91398002500281CD928460B
:10A5E00003F0CEFB074622460199FDF796FE0028B0
:10A5F0000ED13846FDF75CFE81B2384603F0A6F96D
:10A600004CA73846FDF754FE81B2384603F09EF958
:10A6100013986D1C8542E2D345A52846FDF748FEF8
:10A6200081B2284603F092F92146019803F024FCF8
:10A63000274603F079F943E60A2000E00D20159043
:10A6400003F062F93AA52846FDF732FE81B22846AA
:10A6500003F07CF93049002008550D462878002881
:10A6600077D0164C207800280AD06078C01D4007AB
:10A67000C10D2A4808182946FDF721FE002868D098
:10A680006078810125480818294656E00D0A434C98
:10A69000492072656164792E20547970652027689D
:10A6A000656C702720666F7220636F6D6D616E64DC
:10A6B000732E0D0A63616969632D3E0044470020D3
:10A6C0000D0A5B6F74615D2061626F727465642C4A
:10A6D000206261636B20746F20434C490D0A6361F3
:10A6E0006969632D3E000000102700000D0A5B6FB2
:10A6F00074615D2069646C652074696D656F757443
:10A700002C206261636B20746F20434C490D0A63F7
:10A71000616969632D3E0000D05000201051002077
:10A720000D63616969632D3E000000002000000098
:10A730000D0A0000202000000BE0FDF7E5FD607829
:10A74000401C4007400F60702078082801D2401C50
:10A750002070002003F0DAFB134803F01DFB13A464
:10A760002046FDF7A5FD81B2204603F0EFF803F087
:10A77000DBF800242746661EA2E5002CFCD0641EF0
:10A780000CA5A4B22846FDF793FD81B2284603F03C
:10A79000DDF8274694E508A52846FDF789FD81B236
:10A7A000284603F0D3F88BE5D05000206361696937
:10A7B000632D3E00082008000700000010B50C467D
:10A7C000022812DB0EA16068FDF779FD002809D090
:10A7D0000CA16068FDF773FD002804D00AA003F007
:10A7E0009BFB10BD012001F075FF01F06DFF0028FB
:10A7F00001D003A100E003A10AA003F027FB10BDD4
:10A800006F6E00006F66660075736167653A20625F
:10A810006C656C6F67205B6F6E7C6F66665D0D0AA2
:10A8200000000000626C65206C6F673A2025730D94
:10A830000A000000F8B502F0DFF9074602F0D8F987
:10A840000546254A25A128A003F000FB02F002FAE4
:10A8500001462CA003F0FAFA2F48874203D12FA01B
:10A8600003F05AFB15E000F037FF044602F024FA2B
:10A8700006460A213846FDF79BFC0A460146002C95
:10A8800001D0A06900E00020009033462BA003F027
:10A89000DDFA02F02DFA014632A003F0D7FA35486E
:10A8A000854203D134A003F037FB03E029463AA0E8
:10A8B00003F0CCFA09F002FA7D21C900FDF762FC31
:10A8C000014639A003F0C2FA08F0F2FD01463AA0B1
:10A8D00003F0BCFAF8BD00001500010056312E301F
:10A8E000302E3231000000006669726D776172654A
:10A8F0003A202573202830782530386C58290D0AE5
:10A90000000000006375722062616E6B3A20415056
:10A910005025750D0A000000FF7F00006368697014
:10A920002074656D703A2041444320726561642053
:10A9300074696D656F75740D0A0000006368697055
:10A940002074656D703A2025642E256420432028EC
:10A950006164633D2575207472696D3D256C7529B0
:10A960000D0A00007664643A202575206D560D0AA4
:10A9700000000000FFFF000066616E2072706D3AFB
:10A98000206E2F6120286E6F20746163686F6D6583
:10A99000746572290D0A000066616E2072706D3A4E
:10A9A0002025750D0A000000757074696D653A20E8
:10A9B000256C7520730D0A006672656520686561F7
:10A9C000703A20257520420D0A00000002F0D6FBE7
:10A9D00000280DD007A003F09FFAC82008F02CFC37
:10A9E000BFF34F8F11491048C860BFF34F8FFEE788
:10A9F0000FA0F0E7666163746F72793A20666C614C
:10AA00007368207772697465206661696C65642C6F
:10AA100020726573657474696E6720616E79776101
:10AA2000792E2E2E0D0A00000400FA0500ED00E03C
:10AA3000666163746F72792064656661756C7473A6
:10AA400020726573746F7265642C2072657365740F
:10AA500074696E672E2E2E0D0A00000070B5194D18
:10AA60000E46022819DB00240C2060432958706828
:10AA7000FDF725FC002807D0641C102CF4D312A08D
:10AA8000716803F0E3F970BD0C204443601942681B
:10AA9000295916A003F0DAF970BD17A003F03CFAAB
:10AAA000002420460C21484341194A6829580FA028
:10AAB00003F0CCF9641C102CF3D312A003F02CFA91
:10AAC00070BD0000184C0101756E6B6E6F776E20C3
:10AAD000636F6D6D616E643A2025732028747279FE
:10AAE000202768656C7027290D0A00002020252D7D
:10AAF00038732025730D0A00636F6D6D616E64738A
:10AB00003A0D0A006B6579733A20544142203D208A
:10AB1000636F6D706C6574652C2055502F444F57D2
:10AB20004E203D20686973746F72790D0A00000031
:10AB300070B50C46032823DB60680178312902D008
:10AB4000322906D01CE04078002819D1184E012582
:10AB500004E04078002813D1164E402516A1A068C5
:10AB6000FDF7ADFB00280FD014A1A068FDF7A7FBEF
:10AB700000280ED012A1A068FDF7A1FB00280DD07F
:10AB800011A003F0C9F970BD2946304600F05AFB08
:10AB900008E02946304600F051FB03E029463046E4
:10ABA00000F022FB11A0A268616803F04FF970BDAC
:10ABB000000C0140000801406F6E00006F666600E7
:10ABC000746F67676C65000075736167653A206C28
:10ABD0006564203C317C323E203C6F6E7C6F666643
:10ABE0007C746F67676C653E0D0A00006C656420BD
:10ABF000257320257320646F6E650D0A0000000028
:10AC000010B5034803F088F901F0CEFE10BD000036
:10AC1000644D010106A003F07FF9C82008F00CFB89
:10AC2000BFF34F8F07490648C860BFF34F8FFEE759
:10AC3000726573657474696E672E2E2E0D0A00009E
:10AC40000400FA0500ED00E010B509F037F87D21A9
:10AC50000446C900FDF796FA0246214610A003F00B
:10AC6000F5F808F01BFA014614A003F0EFF808F01D
:10AC700025FC044608F01CFC024605212346090376
:10AC800011A003F0E3F81DA003F046F927490020C6
:10AC90000870084608F0F0FA244803F03DF910BDAA
:10ACA000757074696D653A20256C75207469636BE5
:10ACB000732028256C752073290D0A007461736B4D
:10ACC000733A2025750D0A00686561703A20746F2B
:10ACD00074616C20257520422C20667265652025E4
:10ACE0007520422C206D696E206576657220667233
:10ACF000656520257520420D0A0000006E616D65B6
:10AD0000202020202020202020202020207374615B
:10AD1000746520207072696F2020737461636B28E2
:10AD2000772920206E756D0D0A000000F04E00207E
:10AD300010B506A003F0F0F8E12149020BA003F0E2
:10AD400085F816A003F0E8F810BD00007573617275
:10AD500074313A2054583D5042362052583D5042AA
:10AD6000372028414634290D0A00000062617564CD
:10AD70003A20256C752C203820646174612062694A
:10AD800074732C206E6F207061726974792C20317D
:10AD90002073746F70206269740D0A00666C6F779F
:10ADA00020636F6E74726F6C3A206E6F6E653B201D
:10ADB00074783A20444D41204348312028706F6C0C
:10ADC0006C6564293B2072783A205258444E4520E5
:10ADD0006972712071756575650D0A0010B5E12401
:10ADE0006402204602F058FD214602A003F02EF82E
:10ADF00010BD000075736172742072657365743ADA
:10AE000020256C7520384E312C20727820717565A4
:10AE1000756520666C75736865640D0A0000000036
:10AE200010B506A108A003F011F80DA003F074F806
:10AE30001948016819A003F009F810BD56312E30E9
:10AE4000302E3231000000006669726D77617265E4
:10AE50002076657273696F6E3A2025730D0A0000C3
:10AE60006D636D2D6464632D626C653A20424C45C0
:10AE700028726474737329202B20467265655254BE
:10AE80004F53202B205541525428444D4129202B0B
:10AE900020434C490D0A0000004000205379737490
:10AEA000656D436F7265436C6F636B203D20256C4D
:10AEB0007520487A0D0A00004860704701681A4AF8
:10AEC000114001600021016041608160C160174A4A
:10AED0001749904204D148680F22104348607047D8
:10AEE000144A904204D14868F022104348607047E9
:10AEF000114A904205D148680F221202104348605F
:10AF000070470E4A904205D148680F221203104341
:10AF1000486070470A4A9042FBD148680F221204E9
:10AF20001043486070470000FEFF00000800024028
:10AF3000000002401C000240300002404400024079
:10AF4000580002400029016802D00122114301E0AB
:10AF5000014A114001607047FEFF00000246096887
:10AF60000020114200D001207047000030B4036877
:10AF70000D4A0C6A13408A684D6922430C692C43C0
:10AF800022438C692243CC6922434C6A22438C6A57
:10AF900022431A430260CA6842600A6882604968B4
:10AFA000C16030BC704700000F80FFFF002B01D054
:10AFB000106170470020106170470000014948612E
:10AFC0007047000000040140054B002219685B69CE
:10AFD0000140034202D0002900D0012210467047F0
:10AFE0000004014010B4837919490268002B28D06D
:10AFF0000B6893430B604A6803689A434A6002797E
:10B00000521813680468234313608A6803689A43DC
:10B010008A60CA6803689A43CA604279102A06D0D7
:10B0200051180A68006802430A6010BC70478A68B9
:10B0300003681A438A60CA6800680243CA6010BC89
:10B0400070470079401801689143016010BC704757
:10B05000000401400B680022002B56D0F0B40124FC
:10B060000B68944023424AD04B68022B01D0122B2C
:10B0700016D113070AD5456A5307DB0E0F269E40EB
:10B08000B5434E699E402E43466209E0056A530768
:10B09000DB0E0F269E40B5434E699E402E4306624E
:10B0A0004B68012B05D0112B03D0022B01D0122BA2
:10B0B00006D14568DB06DB0FA54393402B43436075
:10B0C0000568530003279F400E79BD43B607B60FAE
:10B0D0009E402E430660C5688E68BD439E402E4349
:10B0E000C66085680126A543CC6894402C438460E3
:10B0F000C46A9E400D69B4439D402543C5620B68F8
:10B10000521CD340ABD1F0BC704770470549016079
:10B11000002242600F218260416101210261C16011
:10B1200070470000FF3F00008162704781617047F7
:10B1300042694A404261704782B0EFF30884FCF7ED
:10B14000D5FF400701D5EFF309840AA000F084FB86
:10B15000E06800900CA0A3686268216800F07CFBA6
:10B16000E069009014A0A3696269216900F074FB92
:10B17000FEE700000A2A2A2A2048617264466175A7
:10B180006C74202A2A2A0A00523020203D253038AB
:10B190006C5820523120203D2530386C58205232D6
:10B1A00020203D2530386C5820523320203D25305A
:10B1B000386C580A00000000523132203D253038EA
:10B1C0006C58204C5220203D2530386C582050437C
:10B1D00020203D2530386C5820785053523D253082
:10B1E000386C580A0000000010B5FFF7A1FF10BD31
:10B1F00030B505460E4887B00C46854202D1012184
:10B20000042004E00B48854210D10121082000F001
:10B2100021F90948844209D86846FFF777FF0120E1
:10B220000190694600942846FFF714FF07B030BD2F
:10B2300000080140000C0140FF3F000010B5FFF77F
:10B2400073FF10BD10B5FFF771FF10BD10B40021E2
:10B250004156FF23CAB29207D40E4278A340920708
:10B26000120EA24000290BDA0907090F08398C08D1
:10B270001049A4006118CC699C431443CC6107E0D9
:10B280008C080D49A40061180C689C4314430C60A1
:10B29000827801210078002A04D0C006C00E8140C7
:10B2A000064803E0C006C00E81400548016010BC9E
:10B2B0007047000000ED00E000E400E000E100E085
:10B2C00080E100E0F7B5FFB004460025A5B00520F9
:10B2D000EFF31087FF210090453102A8FCF7DDFF56
:10B2E000EFF31086FF21453153A8FCF7D6FF53A892
:10B2F000013001909822224953A8FCF7B5FF0120A4
:10B3000080F310880198804786F3108801221D4938
:10B31000120303265300360388420AD194421AD0FE
:10B320009C4201D1151116E0B44210D101256D02E5
:10B3300011E0154988420AD1944201D115460AE02C
:10B340009C4201D11D4606E03546AC4203D0009830
:10B350007FB028B0F0BD06ACFF22013441320B496A
:10B3600002A8FCF781FF012080F310882846A69AE6
:10B37000A599A04787F310887FB028B0F0BD0000E2
:10B38000E8400101C440130085601300A83F01019B
:10B3900010B5EFF31084012181F31088FF21090615
:10B3A000401803490968884784F3108810BD0000DD
:10B3B0000440002010B50848064901600749416073
:10B3C00007498160C922920006490748FCF74CFFF3
:10B3D00010BD0000F14800200440002085490020F5
:10B3E000594800208C4101015048002010B5EFF36E
:10B3F0001084012383F31088FF231B06C018034B1E
:10B400005B68984784F3108810BD0000044000205A
:10B41000034AD16A102399430143D1627047000067
:10B4200000100240044A0029516901D0014300E0A4
:10B43000814351617047000000100240044A002916
:10B44000916A01D0014300E081439162704700009E
:10B4500000100240044A0029916901D0014300E034
:10B4600081439161704700000010024001220549AC
:10B4700012060128086802D0904308607047104304
:10B48000FBE700000010024030B4164A5168042364
:10B490001940154B01D0042901D0036001E0134984
:10B4A00001605168124B8906890F5B5C0168D940C5
:10B4B000416053680F4C5B055B0FE35C0D46DD405C
:10B4C000856053689B045B0FE35CD940C160D16A1F
:10B4D000C90601D5084901E07D21C903016130BCDD
:10B4E00070470000001002400090D0030048E801BF
:10B4F000804101018441010100093D0070470000C5
:10B5000010B5FCF709FE044608F0DEFB002803D066
:10B5100001200349000748602046FCF701FE10BDEA
:10B5200000ED00E010B50A4C2069411C01D0002854
:10B530000AD10120064934220003FFF7C3FE206927
:10B54000411C03D0002801D0024810BD002010BDCE
:10B550001C48002045480020F0B5564C85B0E069F5
:10B5600021040843E0618120534D000628635348BD
:10B57000686153482862534803220168920391434B
:10B580000160514934228014FFF79CFE4E4B4F4E10
:10B5900018694F4F411C29D0002827D0A9691A7873
:10B5A00049094901D206D20E0A43AA612168EA1369
:10B5B0009143216021687F221202914300020843D7
:10B5C00020606068304360606068B84360606068B5
:10B5D000211508436060206A3E4908402062206AC5
:10B5E000D96809020843206205B0F0BD61682046B1
:10B5F000314361606168B943616061680127BF02DE
:10B6000039436160002104917D21C900039100212B
:10B6100000917F214024002502950191026861027A
:10B620008A4302600E11234908687F221202904368
:10B63000220202430A600520FCF750FD0120FCF7BE
:10B640004DFD1C48406B800704D4284603996D1CAF
:10B650008842F3D91748C06B80B2B04201D9811B30
:10B6600000E0311AB94202D2E2B28FB20292B04285
:10B6700001D3019400E00094019A00988018C0055D
:10B68000000EA04203D0044604988142CBD809485A
:10B6900001687F2212029143029A12020A43026059
:10B6A000416849084900416041684907FCD405B038
:10B6B000F0BD000000100240007000400F080000C4
:10B6C00018000200001001401C480020000001008A
:10B6D00000070000FF00F8FF10B50A4C2069411C6C
:10B6E00001D000280AD10120064934220003FFF7C7
:10B6F000E9FD2069411C03D0002801D0014810BD9C
:10B70000002010BD1C48002010B502F09BF810BDB1
:10B7100010B40B06CC065B0FE40E0121A140012BF7
:10B7200007D0022B07D01430002A026805D00A4344
:10B7300004E00C30F8E71030F6E78A43026010BCF2
:10B74000704700000029818903D001225203114370
:10B7500001E0024A1140818170470000FFDF0000D4
:10B76000002A828A01D00A4300E08A43828270471D
:10B770000246128800200A4200D00120704770B4AF
:10B780000A06530FCE060125F60E2A460024B240C3
:10B79000012B0FD0022B10D0838A1340090A008896
:10B7A0008D402840002B02D0002800D001242046E4
:10B7B00070BC704783891340F0E7038AEDE700000F
:10B7C00070B50446008A86B00D461B490840E988DA
:10B7D00001432182A08919492A890840A988114377
:10B7E0006A8902431143A181A08A15490840A989A9
:10B7F0000143A1826846FFF747FE1248844201D107
:10B80000039800E002982968192289005043FCF748
:10B81000B9FC06466421FCF7B5FC05012809642142
:10B820004843301A00013230FCF7ACFC0007000F2F
:10B830002843208106B070BDFFCF0000F3E900006F
:10B84000FFFC0000003801408088C005C00D704733
:10B85000C905C90D818070470FB410B503A9044B09
:10B86000044A029800F066F910BC08BC04B01847FE
:10B870000DE40001C40100200FB410B504A9074B6A
:10B8800002AA039800F056F9044602A9002000F02D
:10B89000F8FC204610BC08BC04B0184783C2000165
:10B8A0007CB51546024600201C4600290BD0491ED7
:10B8B00000920191044B6A462146284600F03AF96D
:10B8C000009A002111707CBD6DC200012021020C84
:10B8D00001D010211046020A01D010460839020991
:10B8E00001D01046091F820801D01046891E420867
:10B8F00001D0881E7047081A704700000048704742
:10B900001848002030B5002805D0164C021F2068CA
:10B910000023014605E0084630BD904203D80346A7
:10B9200040680028F9D1002B00D05968002B0AD0BC
:10B930001C68D51AA54204D11268A4181A461C60C6
:10B9400002E05A6000E02260002807D01468851ADF
:10B95000A54203D105686419146040685060184618
:10B9600030BD000010480020F1B50E4C0F480C4EC1
:10B97000001B0D4FC508ED0000221146009804F091
:10B980000DF8002803D13068002801D00020F8BD50
:10B990003C6000202560606001203060ECE7000022
:10B9A00014480020DCAF002010480020D8B100204F
:10B9B000F0B51FB486B00998089A030D0021024320
:10B9C00014D05148514A18185043051411980128B1
:10B9D00010981AD0281A401C00264D4F4D49009649
:10B9E00001910490002812DA444211E011980124D8
:10B9F00049A3012801D11098C1430698119A846087
:10BA00000360C26041600BB0F0BD4042E4E7044611
:10BA1000210500203F4A001C51410391029012E091
:10BA2000E00707D032463B4601990098FCF7E0FF5B
:10BA30000191009032463B4610461946FCF7D8FF6C
:10BA400006460F466410002CEAD10498039B002898
:10BA5000029A0999089806DAFCF7CAFF019B009A36
:10BA6000FCF7C6FF05E0FDF72BF8019B009AFDF7F8
:10BA700027F804460E460022284BFDF76DF903D83F
:10BA80000020C043014607E00022254B20463146F6
:10BA9000FCF7FCFEFDF718F9102409E0002C0ADB86
:10BAA0000A220023FCF798FB079B30321A55641ECC
:10BAB00002460A43F2D11122641C079B121B1C1977
:10BAC000119B012B03D0012308430ED10AE0084348
:10BAD00004D0112010900020119077E71098151ACB
:10BAE0006D1E0BE01098824202DD00236D1C03E006
:10BAF000824201DA00236D1E002BEED006981199C8
:10BB00008260C16030C07EE701FCFFFF104D000085
:10BB1000000014400000F03F300000000000F0433F
:10BB20000000E03F30380A2801D201207047002091
:10BB300070470000FFB597B00646002518E225289B
:10BB400077D100242746FD49049400E00443761C85
:10BB500032780120203A90400842F7D130782A28E4
:10BB60000ED00222307801463039092916D80499BE
:10BB70000A235943303940181443761C0490F1E7E6
:10BB8000189802C804911890002904DA0120400393
:10BB900004434842049002200443761C30782E2847
:10BBA00014D1042004437078761C2A2809D11898EF
:10BBB000761C80C8189009E00A214F43303FC7190E
:10BBC000761C3078014630390929F5D930786C284F
:10BBD00010D006DC4C281AD068280ED06A2817D15D
:10BBE00004E0742813D07A2812D110E00120400517
:10BBF00004430CE00121090501E0032109050C4380
:10BC00007178814203D1012000052418761C761C2E
:10BC10003078119066280BD013DC58287DD009DCD1
:10BC200000287BD04528F6D04628F4D047281AD1E2
:10BC3000A5E118E0632835D0642870D0652812D1BA
:10BC40009DE170286CD008DC6728F1D069287BD092
:10BC50006E280DD06F2806D1BAE073282ED0752833
:10BC600071D0782859D01A9A199990476D1C7EE1A5
:10BC70006002400F022809D003280DD0042818982C
:10BC800001680DD00D60001D189070E11898EA173A
:10BC900001680D604A60F6E7189801680D80F2E7C8
:10BCA0000D70F0E718986A4601781172001D18901F
:10BCB0000020507202A80090012005E0189802C8E8
:10BCC000189000200091C04361070DD5002101E0CC
:10BCD0000199491C0191B94212DA8142F8DB009ABC
:10BCE000515C0029F4D10BE0002101E00199491CCD
:10BCF00001918142FADB019A0099895C0029F5D112
:10BD0000019904981A9B471A21463846199A00F05F
:10BD100097FA0199401945180BE04FE02CE113E028
:10BD20004EE0009800990078491C00911A9A1999E0
:10BD300090470198401E0190401CF2D121463846A0
:10BD40001A9B199A10E137E00A2000210090019116
:10BD50006002410F022907D0189A01CA1892C2172F
:10BD60009446032908D00AE01898C01DC108C900EC
:10BD700005C91891944607E000B2C21794460429F9
:10BD800002D140B2C1178C4600226146944506DAC2
:10BD90000A460021404291418C462D2102E02105B6
:10BDA00004D52B216A461173012103E0E10701D07C
:10BDB0002021F7E7029155E00A200AE0102008E070
:10BDC000102000900021042004430191082703E083
:10BDD00008200021019100906002410F022907D044
:10BDE000189A01CA189200229446032908D008E044
:10BDF0001898C01DC108C90005C91891944603E0F0
:10BE000080B2042900D1C0B200210291210729D5B6
:10BE10001199702906D0009A1021019B4A401A43BB
:10BE200005D00EE040216A461173012108E0614609
:10BE3000014306D030216A461173119951730221D2
:10BE40000291009A0821019B4A401A430AD1614697
:10BE5000014301D1610705D530216A4611730121E3
:10BE60007F1E02911199582904D035A10E910DA978
:10BE70000D910DE037A1F9E76146019B009AFCF7AF
:10BE8000ABF90E9B8C469B5C0D9A521E0D92137063
:10BE900061460143F0D10D9805A9081A20300190A0
:10BEA000600703D501200004844300E001270198C6
:10BEB000874201DD381A00E0002001990090411806
:10BEC000029809180498401A0490E00306D4214609
:10BED0001A9B199A049800F0B3F94519002706E057
:10BEE00003A81A9AC05D199990476D1C7F1C02988F
:10BEF0008742F5DBE0030CD521461A9B199A04987A
:10BF000000F09EF9451904E01A9A302019999047DB
:10BF10006D1C0099481E00900029F5DC08E00D9882
:10BF20000D990078491C0D911A9A199990476D1C2A
:10BF30000199481E01900029F1DC63E10928010004
:10BF4000303132333435363738396162636465668F
:10BF50000000000030313233343536373839414251
:10BF6000434445460000000000F05AF94519761C8C
:10BF70003078002800D0E2E528461BB0F0BD60070D
:10BF800000D406271898C01DC108C90048680A686F
:10BF90000831C30FDB071891190001D09CA108E0FC
:10BFA000210501D59BA104E0E10701D09AA100E0A1
:10BFB0009AA1430011985B08109165280CD006DC0B
:10BFC000452809D046281DD0472841D141E06628A0
:10BFD00018D067283CD13CE00021112F01DB112053
:10BFE00000E0781C0191009008A911A8FFF7E0FC7F
:10BFF000139905910021119A15927F1C12980197AF
:10C00000009150E00120C00703900120019008A991
:10C01000009711A8FFF7CCFC139A149905920022FF
:10C02000119B009212981593059A0192002901D054
:10C03000104602E0791C40180190381A01D5019889
:10C0400004E04042401E0090781C0190C01B02900A
:10C0500043E0012F00DA01270021112F01DD11201B
:10C0600000E038460191009008A911A8FFF7A0FC54
:10C0700013990591119A0021129815920091019738
:10C0800021070CD40599B94201DB019900E0019127
:10C09000012904DD159A491E515C302906D0B842A9
:10C0A00001DA011D05DA0121029115E00199491E0D
:10C0B000EDE7002805DC0099411800910199091A63
:10C0C00003E0019A411C914200DD01910099401A60
:10C0D000401C02900120C0070390200706D402995B
:10C0E0000198814202DB0020C04302900020694693
:10C0F000C87707AF012103980337C907884224D0C6
:10C10000022011902B201290039800280CDA404254
:10C1100003902D20129007E00A210398FCF732F8D3
:10C1200030317F1E039039701199481E11900029FB
:10C13000F2DC03980028EFD1791E1298087030784D
:10C14000202108404530BF1E387006A8C01BC01D06
:10C15000039010980078002800D001200199411820
:10C160000298C0170918039809180498401A401E2D
:10C170000490E00306D421461A9B199A049800F013
:10C180005FF8451910980078002803D01A9A199979
:10C1900090476D1CE00324D521461A9B199A0498F8
:10C1A00000F04EF845191CE00098002807DB0099C4
:10C1B0000598884203DD1598405C199901E01999AA
:10C1C00030201A9A904700986D1C401C00900298ED
:10C1D000401E0290002804D11A9A2E2019999047E7
:10C1E0006D1C0199481E01900029DDDC05E03878BE
:10C1F0001A9A7F1C199990476D1C0399481E039049
:10C200000029F4DC21461A9B199A0498ACE6000038
:10C210002D0000002B0000002000000000000000A6
:10C22000F8B5044600251E461746880404D405E0E8
:10C2300039462020B0476D1C641EF9D52846F8BD4C
:10C24000FFB50446002581B01E46C80301D530273E
:10C2500000E02027880404D505E038460399B0475C
:10C260006D1C641EF9D5284605B0F0BD4A68002A49
:10C2700006D00A68531C0B6010704868401E486066
:10C2800070470A68531C0B6010707047002903D078
:10C29000002801D0884201D1002070478268002A1E
:10C2A00008D05268002A03D011604A60806841605B
:10C2B000012070478160496000200860F8E7FFB501
:10C2C00081B007000A9814460D4605D0002D03D012
:10C2D000002C01D0A74202D1002005B0F0BD0126FC
:10C2E0007602002802D0E068304307E0284604992F
:10C2F00001F000FD051EF0D0E068B0430646A089BD
:10C30000800505D4206A002802D00499496888472E
:10C31000E660214638462562FFF7B8FF05B0F0BD5C
:10C3200000B599B060216846FBF7B7FF042008AA62
:10C33000D07012A0006801900B2010AAD0700246A5
:10C3400010A109A8FBF790FF002010AA107101218D
:10C350005171D071917190731175D082A0201083AA
:10C360009176B42090831920C001D08308480090B2
:10C37000684603F0F3FD19B000BD000003160A186B
:10C38000000000000AFFFFFF4E6174696F6E7300CA
:10C3900095C300017047000010B540210848FEF722
:10C3A00051FF08490020087000F08EF9002802D0E3
:10C3B00005A0FFF751FAF72003F044FF10BD00007D
:10C3C00000080140374700205B424C455D20636F09
:10C3D0006E6E65637465640D0A00000010B503F0AD
:10C3E000E1FD00F07FF940210648FEF727FF0649EE
:10C3F0000020087000F068F9002802D003A0FFF7C1
:10C400002BFA10BD00080140374700205B424C4525
:10C410005D20646973636F6E6E65637465642C2060
:10C420006164766572746973696E6720726573748E
:10C4300061727465640D0A0010B58CB0002400941C
:10C440000194029403940494059406940794089428
:10C4500009940A94FFF766F8002804D0014601A861
:10C46000FDF796F807E012A001886A46918041889E
:10C47000D180808810816946CC704C810A208870F8
:10C4800012220A7303A80CA10130FBF7EDFE0C2069
:10C490006946088418204884FF208C84F530C884BD
:10C4A0000A480885684603F01BFE0CB010BD00006A
:10C4B000010203040506000043414949432D4D4351
:10C4C0004D2D3230323630393032000088130000C2
:10C4D00000B583B00D4900910D49002001910290F3
:10C4E00069460872684603F0FFFEFFF7A5FF00F0FB
:10C4F00033FAFFF715FF074803F09CFC064803F0EA
:10C5000099FC03F04FFD03B000BD00001DC5000104
:10C51000C1D3000191CA0001A9D10001017801290C
:10C5200028D070B50025144E144C022912D00329CE
:10C530000FD103F037FD00F0D5F840213046FEF76B
:10C540007DFE257000F0C0F8002802D00C48FFF7EF
:10C5500083F970BD40213046FEF774FE257000F06F
:10C56000B3F8002802D00748FFF776F9F72003F068
:10C5700069FE70BD70470000000801403747002089
:10C580000CC40001C8C30001F8B50646244F0020C2
:10C59000388178810124481E0D463E2814D80A4669
:10C5A00031462048FBF760FE1E49002048551E48D2
:10C5B00001F0ACFC1B4801F0EFFB0446002001F049
:10C5C000A5FC388900280CD1002C12D017A00090AF
:10C5D000FBF76EFE84B2224619480099FBF744FE31
:10C5E0003C81B878002819D016A0FFF735F900244F
:10C5F0000CE019A0EBE7315D084620385F2800D336
:10C600002E2117A0FFF728F9641CA4B2AC4201D276
:10C610003F2CF0D3398913A0FFF71EF9F8BD0000B5
:10C620004E47002010550020E1DE0001756E6B6E54
:10C630006F776E20636F6D6D616E640D0A00000090
:10C640008B5800205B424C455D20636C6920657807
:10C6500065633A20220000006F6B0D0A00000000A5
:10C660002563000022202D3E202575422072737024
:10C670000D0A000030B40C49098E182902D3891E16
:10C680008AB200E01422094C094D63892189ED1812
:10C69000C91A89B2914200D911465A1862810180A3
:10C6A000284630BC70470000C04D00204E47002097
:10C6B0008B5800200348002101708180C1804170A7
:10C6C000704700004E470020014880787047000006
:10C6D0004E470020002800D0012001498870704793
:10C6E0004E47002010B50549002008708880488119
:10C6F00000F008FF00F070FB10BD00004E47002066
:10C70000F3B583B00498002400287AD95B480290DE
:10C710005B4A03981178005D002904D001290BD0F1
:10C7200002291AD122E0CA286CD15649087001208A
:10C7300090800521D18017E0524B91885854491CB4
:10C7400088B2908005285DD102984178037808026C
:10C75000FF211843E131884203D9002010709080F6
:10C7600084E0C01DD080022010707FE0444A454B19
:10C7700091885854491C88B29080D188884275D1DC
:10C7800002980022417800780D0205433E48844615
:10C79000281D86B23D48002E14D93D4F6146895C64
:10C7A000090248400021030402D54000784000E01F
:10C7B0004000491CC9B280B20829F4D3521C92B27D
:10C7C000B242EBD32F4E71198A794B79110219437A
:10C7D000884247D17778B07801902948761D8078D3
:10C7E000002806D03346009539462AA0019A05F064
:10C7F000E7FC112F2AD006DC012F09D0102F31D1F0
:10C8000024E039E032E0122F20D0202F2AD124E07A
:10C8100001273F2D11D82A4631461F48FBF724FD3A
:10C820001D49002048551D4801F070FB1A4801F0D1
:10C83000B3FA0746002001F069FB68460770012340
:10C840006A460320019900F02BF80BE02B46324694
:10C850003846019900F08EFB04E02A4631460198E3
:10C8600000F004FA0648002101708180641C0498DD
:10C87000A4B2844200D24BE705B0F0BD935500202E
:10C880004E4700209055002091550020FFFF0000EA
:10C89000211000005258000050550020892101014C
:10C8A000FFB5D81D80B283B01D460190FB2803D987
:10C8B0000020C04307B0F0BD214CCA20207003986F
:10C8C00060700498A070280AE5702071002D04D0D3
:10C8D0002A46601D0599FBF7C7FC281D83B2194F36
:10C8E00019480024002B13D9184E395D090248401D
:10C8F0000021020402D54000704000E04000491CC5
:10C90000C9B280B20829F4D3641CA4B29C42ECD30F
:10C910000B4949194871000A88710D488078002830
:10C9200006D000950BA0059B049A039905F048FCDE
:10C930000348019900F0EEFD002007B0F0BD0000B3
:10C940009057002091570020FFFF000021100000A9
:10C950004E4700205458000000B587B000200190D9
:10C960000090039004906A46069010730C4902915F
:10C9700005219170032313701023D3705070107130
:10C980000123537190715073064805907D20917377
:10C9900000011082104604F06DF907B000BD0000E0
:10C9A00040E2010000B00301014901208870704796
:10C9B0004447002010B5024803F004FF002010BDDA
:10C9C000644E00202F48007900285AD1F8B56D2018
:10C9D0002C230322072140010BF4AED0A0210446F2
:10C9E000017029480027C178617027710321E18017
:10C9F0006772012666710721244D2177A979617735
:10CA0000687B002803D0E780032060710EE0E8799E
:10CA100000280BD0A879022800D166772671E6801D
:10CA20002046A979203041708670077015488079BA
:10CA3000022804D0032815D004281BD116E004F0E6
:10CA40000BF900280BD00520E0806771688A6061CF
:10CA5000688AA06120460A3003F02CFF0AE00949E9
:10CA600003208871288B6061288B02E0E88B60616D
:10CA7000E88BA06103480671467120460BF498D0FC
:10CA8000F8BD7047C04D0020444E0020B04E00203D
:10CA900010B584B00A230322072110480BF44CD0B0
:10CAA0001B210170002141701424448003228280E4
:10CAB000C1800B4A02810BF47BD068460480094890
:10CAC0000190684603F0D8FB68460481064803904D
:10CAD00002A804F0CBFF04B010BD00001B0D000045
:10CAE000FF010000C04A0101D9E00001FFB585B097
:10CAF000054602A800901C462846069904F004F951
:10CB00006846007A002866D006980090280A334AC2
:10CB1000019403900E2826D0314800240178002982
:10CB200051D92F48E1000818828803998A4240D1E0
:10CB3000009A81689646019A284694460A79120618
:10CB4000120E36D00968254BD700083FCE1937881A
:10CB50007668BFB2874201D09F4226D16346032246
:10CB60007146B04725E01F49681809282BD800985E
:10CB70001D49844608792E4600062346000E1ED025
:10CB8000C4000F68083C3C1927886468BFB2B742EC
:10CB900001D0974204D1032261462846A0470EE007
:10CBA000401E0006000EEBD109E0521E1206120EC6
:10CBB000CAD10B48641C0078E4B2A042B1D86846E0
:10CBC000007A002807D00948426C002A02D0284683
:10CBD00006999047002009B0F0BD0000FFFF00005B
:10CBE0006C4D0020EEF1FFFF10460101C04D00200A
:10CBF00000487047FFFF000070B5124D0121284624
:10CC0000FCF70CFE142006F017FB702002F0BEFDAE
:10CC1000702002F0BBFD044600212846FCF7FEFD13
:10CC2000094844800948844201D1401070BD204623
:10CC3000FCF72AFD0649FBF7EBFDFCF707F800B20D
:10CC400070BD00000008024094470020FFFF000074
:10CC50000000204110B500F089F90349884201D154
:10CC6000022010BD012010BD00400201F0B50746B2
:10CC700000208DB015460E46002A04D0012D04D1A7
:10CC80003178FF2901D10B4E07250024002D08D94A
:10CC90000146325D684602F0AFFD641CA4B2AC42AE
:10CCA000F6D303466A4639462120FFF7F9FD0DB059
:10CCB000F0BD0000D84C01010148408870470000D9
:10CCC0009447002070B506460020074D04460146F3
:10CCD0002A5D064802F090FD641CA4B2072CF6D32E
:10CCE0003080024870BD0000D84C0101825E0020F7
:10CCF00010B5602002F04AFD0449884201D10020AD
:10CD000010BD6021FCF7EAFC80B210BDFFFF0000FF
:10CD100010B503F01DFD04480169002901D004206D
:10CD20008847002010BD0000D04E002070B5224C76
:10CD3000606B224DC00722D0A06B21497E2209687A
:10CD40005143401A2988491E29804B21C9004018A7
:10CD50001C49884213D300202880206A40084000E4
:10CD60002062194908680204930F184A01D09043C1
:10CD700000E0104308601648407F03F021FA29883C
:10CD800001200029216B07D00143216305220321E3
:10CD900010480BF493D10DE0FF221202914321635E
:10CDA000216B0522920211432163216B0143216310
:10CDB00003F0A0FF002070BD0010024034470020A7
:10CDC0008C000020B10400000010014000C00000F1
:10CDD000204E0020010F0000034800210170C161B6
:10CDE00001624162C16270475C4700200248002135
:10CDF0004171C180704700005C470020054A51899D
:10CE00000180002901D0012090700020508102484B
:10CE1000704700005C470020725E0020F7B5414972
:10CE200082B04A6303980024002879D93E483F4FD6
:10CE300000903C4A02985179005D002904D00129F4
:10CE40000CD002291BD128E0CA2864D138490870C7
:10CE50000121D1800520108151715CE0344BD188D3
:10CE60005854491C88B2D080052854D10098417884
:10CE700003780802FF211843E131884203D90020DA
:10CE80005071D08047E0C01D80B21081052802D0CB
:10CE9000022050713FE00020FBE7224A244DD18858
:10CEA0006854491C88B2D0801189884233D10098D7
:10CEB000204D41780278080210430346001D81B2DC
:10CEC0004A1E1D4896B2002914D02978090248400C
:10CED00000216D1C020402D54000784000E04000B3
:10CEE000491CC9B280B20829F4D33146761EB6B2C5
:10CEF0000029EAD10E4AD1188D794E7929023143A1
:10CF0000884204D191785078521D00F033F80548DA
:10CF100000214171C180641C0398A4B2844288D36B
:10CF200005B0F0BD5C4700208E5C002021100000A1
:10CF30008B5C00208C5C0020FFFF000010B5024AD3
:10CF4000FFF76CFF10BD0000D10D010101B5054ACE
:10CF500001216846FFF762FF0349002208790A7140
:10CF600008BD0000DD1101015C470020004870474A
:10CF700000800001F8B514464F4A0D46102815D020
:10CF8000112871D0122870D013280ED1FFF724FF7A
:10CF90001446D36900221321284604F0CFF84749EC
:10CFA000606B884201D101202071F8BD00910C2BEB
:10CFB00004D000230122102128466EE02378E17876
:10CFC0001846637809061B021843A3781B0418430C
:10CFD00008430502E0782D0A000623790543184628
:10CFE0006379E1791B021843A37909061B041843EE
:10CFF00008430602E079360A000606430820211895
:10D000000B7818464B781B0218438B78C9781B04A1
:10D010001843090608430702E07A3F0A000607435F
:10D020001078002806D0D36902221021009804F05D
:10D0300085F8F8BD22482349234C884202D0A042FB
:10D040000BD10C462149281F88420FD3002303220D
:10D050001021009804F072F8F8BD0023022210217C
:10D06000009804F06BF8F8BD1AE01FE01248407811
:10D07000002804D1FEF79EF90F49012048700E48A0
:10D08000012101700021C16101624162C1620C3065
:10D09000F0C00B460A461021009804F04FF8F8BD86
:10D0A0001A462146284603F0A5FEF8BD1A46214639
:10D0B000284603F049FFF8BD5C470020DD1101015F
:10D0C000008000010080000100400201FDBF01005E
:10D0D00010B50E4CE078002816D006F0EFFD216B5D
:10D0E000401AA178002903D0FF212D31884203D2B4
:10D0F0007D210901884207D3BFF34F8F05490448BA
:10D10000C860BFF34F8FFEE710BD00005C470020F2
:10D110000400FA0500ED00E000487047B45E00200E
:10D12000F8B5342211491248FBF79EF8104C114F04
:10D1300020680125104EB8420BD16068012808D143
:10D140002046302100F0EAFD216B884201D1357084
:10D15000F8BD34210648FBF7A0F8FF202760F53022
:10D16000656020810020E0603070F8BD0060000143
:10D17000B45E00207ADA12CA9847002010B5342134
:10D180000748FBF78AF8064806490160012141601B
:10D19000FF21F53101810021C16004F085F810BD47
:10D1A000B45E00207ADA12CA10B584B014230322C8
:10D1B000072112480AF4C0D41B21017000214170DC
:10D1C0004724448003228280C1800D4AC2600D4AF8
:10D1D00002610D2202720AF4EBD4684604800A4808
:10D1E0000190684603F048F86846048107480390B8
:10D1F00002A804F03BFC04B010BD00001B0D0000B1
:10D20000E04A0101D04A0101C84A01017529010122
:10D2100000207047F8B5184D184FE879002801D064
:10D220002E7B00E0FE780322331D072114480AF408
:10D2300083D4A921044601701248C178617000218D
:10D240006180E8791049002803D02A7B896C201D71
:10D2500002E0FA78201D091DFBF706F8608802211C
:10D260008019608007480279062A00D00171417157
:10D2700020460AF49DD4F8BDB04E0020904E002008
:10D28000A60D0000C04D0020704E0020F8B51F26EE
:10D2900023230322072128480AF44ED40446AA2057
:10D2A000264F2070F878264D6070E8786080EA7824
:10D2B0002449201DFAF7D8FF6288B01AC1B2201D98
:10D2C0001018214A0326032910D92B79002B0DD0E1
:10D2D0000670192343705389091F1B0AC370937A80
:10D2E00083706388C9B21B1D6380001D02291AD98F
:10D2F0006B79002B17D0137B891E8B4200D2194605
:10D30000CDB2691C0170117BA94201D1092100E055
:10D31000082141702A460D49801CFAF7A5FF608854
:10D32000AD1C401960803879062800D03E717E71AE
:10D3300020460AF43DD4F8BDA60D0000C04D0020E3
:10D34000B04E0020944E0020444E0020514E00204C
:10D3500070B53A230322072116480AF4EDD3A4211D
:10D36000154D04460170E8786070A97913480022D1
:10D37000022910D0032913D0042916D0628022710B
:10D38000807902F04DFB0520287104206871204649
:10D390000AF40ED470BD018A642359436180EEE71C
:10D3A000C18A642359436180E9E7818B642359432F
:10D3B0006180E4E7A10D0000C04D0020B04E0020C8
:10D3C00070470000FFB50F4683B000210091019126
:10D3D00016466946FCF7E2F8040030D10521C9027F
:10D3E0006846FCF7E1F8002828D121496846FCF797
:10D3F000DBF8002822D11F496846FCF7D5F8002841
:10D400001CD11D496846FCF7CFF8002816D1292108
:10D4100009026846FCF7C8F800280FD1174968468A
:10D42000FCF7C2F8002809D115496846FCF7BCF89A
:10D43000002803D100988088C10B03D00624204621
:10D4400007B0F0BD00050099000D0D186888B042C6
:10D4500000D207242988B819884201D90D24EEE7A3
:10D46000A8193A46001D0699FAF7FEFE6F80E6E716
:10D470000128000003280000022800000229000003
:10D48000032900001DF48CD700F010F8FFF720FEF0
:10D49000012005F0D1FEF5E710B503490020087022
:10D4A00000F004F810BD0000484700201248002199
:10D4B000007800281FD070B5104D86B0287800285D
:10D4C00017D1A8886C88A04213D00D4E6A4680B24E
:10D4D000A04209D0335C5354401CC005491CC00D08
:10D4E00089B2A8801429F2D301202870104605F0D3
:10D4F00045FA06B070BD7047374700204847002006
:10D50000105300200249002048808880087070472E
:10D5100048470020F0B484460D480078002814D015
:10D520000022002911D90B480B4D878843881C46DF
:10D530005B1CDB05DB0DBB4207D06646B65C521CAC
:10D540002E5592B243808A42F0D3F0BC704700005F
:10D5500037470020484700201053002070B5134D76
:10D5600004462878002803D1FDF724FF0120287005
:10D570000F4820602821204600F0D0FB0D4DA0620E
:10D580002846FDF705FF00280DD12C22214628460C
:10D59000FDF72CFF002806D12C2229462046FAF759
:10D5A000A6FE002800D0012070BD00009A47002090
:10D5B00011C011CA0040000110B5044600681949A5
:10D5C000884208D12046282100F0A8FBA16A8842A1
:10D5D00001D115A200E016A21B491CA000F036FCE8
:10D5E00021A0216800F032FC26A0616800F02EFC2A
:10D5F0002AA02369E268A16800F028FC33A06169D1
:10D6000000F024FC37A0236AE269A16900F01EFC47
:10D610002EA0616A00F01AFC3EA0A16A00F016FC80
:10D6200010BD000011C011CA76616C696400000071
:10D63000494E56414C49442028626164206D61671F
:10D6400069632F637263290000400001626F6F7489
:10D6500073657474696E6720402030782530386CAB
:10D66000583A2025730D0A0020206D6167696320F8
:10D670002020202020203D2030782530386C580D87
:10D680000A00000020206163746976655F62616E44
:10D690006B203D20256C750D0A0000002020626182
:10D6A0006E6B313A20616464723D30782530386C9D
:10D6B000582073697A653D256C75206372633D302F
:10D6C000782530386C580D0A0000000020202020FA
:10D6D00020202020207665723D30782530386C5827
:10D6E0000D0A0000202062616E6B323A2061646492
:10D6F000723D30782530386C582073697A653D2545
:10D700006C75206372633D30782530386C580D0A93
:10D71000000000002020637263333220202020208C
:10D7200020203D2030782530386C580D0A0000004C
:10D7300030B58DB001210820FDF78CFE0121880352
:10D74000FDF788FE02A8FDF7E1FC402002900220D0
:10D75000284D0424039002A907942846FDF77AFC7B
:10D7600080210794029102A92846FDF773FCE1206D
:10D7700040020890002069468884C884088588850E
:10D780000C2048851C4D08A92846FEF719F80121F0
:10D790000846FDF747FE194C2046FDF78FFB012395
:10D7A000224617490220FDF701FC0122802128466C
:10D7B000FDF7D6FF00220121402005F0BFFE114CED
:10D7C0002060012005F0A8FE606001220E49284675
:10D7D000FDF79EFF1C206946087003204870012059
:10D7E00088706846FDF732FD01212846FDF7AAFF43
:10D7F0000DB030BD000C014000380140080002406F
:10D8000000000240384700202505000070B505469D
:10D810000B480468002C0ED0481C0ED008467D2111
:10D82000C9004843FAF7AEFC02462946204605F0F7
:10D83000ECFF012800D0002070BD0020C043F3E7BA
:10D840003847002010B582B00020104C00900E49DF
:10D850002046FDF794FF002814D02046FDF7F4FF82
:10D86000694608710A480068002804D00A46002367
:10D8700001A905F083FF0098002803D00120054985
:10D880000007486002B010BD2505000000380140C7
:10D890003847002000ED00E030B5184D85B0044653
:10D8A00040212846FDF764FF0028F9D000212846D2
:10D8B000FDF748FF0020694600948880C8800881F1
:10D8C00088810C2048812846FDF77AFF0C4C20689F
:10D8D000002807D006F0E2F9022803D100212068D1
:10D8E00005F04EFE012207492846FDF711FF0121F0
:10D8F0002846FDF727FF05B030BD00000038014085
:10D90000384700202505000010B5064C6068002847
:10D9100007D006F0C3F9022803D1C11E606806F0E3
:10D9200015F810BD3847002010B5074C6068002876
:10D9300009D006F0B3F9022805D100231A4619468A
:10D94000606805F054FE10BD3847002000283FD025
:10D9500000293DD0F0B51F4E0C4605468BB0002186
:10D960003046FDF7EFFA1C4F02203946FDF7A4FAC6
:10D970001A48009010200290002080210591049008
:10D9800003210195039409030690079008900991DB
:10D990000A9069463046FDF7E9FA01213046FDF765
:10D9A000D1FA39460220FDF7D9FA0028F9D0002132
:10D9B0003046FDF7C7FA39460220FDF77DFA084CDC
:10D9C00040212046FDF7D4FE0028F9D00BB0F0BD71
:10D9D0007047000008000240000002400438014087
:10D9E0000038014010B4002807D00368002B04D091
:10D9F00042688168914201D206E0002010BC704765
:10DA0000491C8160002804D0914202D25C5C202C29
:10DA1000F6D99142F2D1491E816010BC70470000D6
:10DA2000F8B50C4605461046194600F013F80646B0
:10DA300000200090064B324621462846FEF73FFC68
:10DA40000028304602D100F043F80020F8BD000065
:10DA5000A447002070B505460E46124800F0A2F813
:10DA600004001CD0E6610820A561E0600E4A0F4B5F
:10DA700028463146FBF770F902D80D4860610EE088
:10DA800000220C4B28463146FBF752F902D8012000
:10DA9000C00703E028463146FBF7F2F860612046F4
:10DAA00070BD0000A44700200000C0FFFFFFDF4161
:10DAB000FFFFFF7F0000E0C110B5044800F072F8DE
:10DAC000002801D04021C16010BD0000A447002003
:10DAD000002824D0F8B5124E04460027A0892568F6
:10DAE000C0050DD4A068002804D0FFF7F1FFA0897D
:10DAF000C00505D42069002802D0716888472761D5
:10DB0000A089800505D4206A002802D07168884762
:10DB100027627168204688472C00DFD1F8BD704726
:10DB2000A447002010B5002201F088FD10BD0000C0
:10DB300030B4124A0E4D0F4B0F4C0028136013D017
:10DB40000168002900D0116054604068002800D0AE
:10DB50005060002090601068984203D15068A04245
:10DB600000D1956030BC70479560546030BC704700
:10DB7000D12D010169B9000105B90001A4470020B8
:10DB8000002803D0007B082801D000207047012026
:10DB90007047002803D0007B402801D00020704748
:10DBA0000120704710B501682820884700280AD056
:10DBB0000021016041608160C1600161416181615A
:10DBC000C1610162416210BD70B500260446354650
:10DBD000002808D0FAF76CFB411C2B463246204641
:10DBE00000F004F870BD002070BD0000FFB50024F7
:10DBF00089B0064600940194344802940394049436
:10DC000005940694046015464460002E5AD00029FD
:10DC10003FD0024600960191D16890681269049045
:10DC2000069205912A48FFF7BDFF0790002830D0E3
:10DC300000986F46002802D00298002801D00020EA
:10DC40000DE00198042809D9032222A10098FAF7CF
:10DC500064FB002802D10298C01C02903846FFF7EE
:10DC6000C1FE0146079803F085FC00280ED00C98F1
:10DC7000002814D06846FFF7B5FE0299019881424A
:10DC800004D202990098405C002808D00798FFF75A
:10DC90001FFF0199029888420AD204460BE0002D2A
:10DCA00003D0029900984018286007980DB0F0BD85
:10DCB000081E00D0441E002D01D0301928600348F2
:10DCC0000660446000200DB0F0BD00009C470020BD
:10DCD000A4470020EFBBBF0010B5024A002103F0AB
:10DCE00067FF10BDA44700200149496808470000AC
:10DCF000A4470020002810D070B50E460446FAF75D
:10DD0000D7FA401C336805469847061E04D02A46B9
:10DD10002146FAF7A9FA304670BD7047002230B4A8
:10DD2000D243491E0FD3094C03785A400023401CAC
:10DD30005508D20700D022465B1C6A40DBB2082B94
:10DD4000F6D3491EF0D230BCD04370472083B8EDE3
:10DD500002468B880020022B01D00D207047C98815
:10DD6000002A05D00029F9D00129F7D08120704779
:10DD70000029FCD00229F9D170471020704700001B
:10DD8000102804D20C21484302490858704700204B
:10DD900070470000184C010170B588B000246A4635
:10DDA000234616E0401C01782029FBD00929F9D030
:10DDB0000906090E12D0A1005050641C00E0401C5E
:10DDC000017800290AD0202901D00929F7D1037050
:10DDD000401C0178002901D0082CE4DB002C14D071
:10DDE000104E002528460C21484331580098FAF778
:10DDF00066FA00280CD06D1C102DF3D30AA00099F0
:10DE000000F024F8012008B070BD002008B070BDFB
:10DE10000C204543A8198268694620469047002097
:10DE200008B070BD184C0101756E6B6E6F776E2077
:10DE3000636F6D6D616E643A20257320287472796A
:10DE4000202768656C7027290D0A00000FB410B5F3
:10DE500003AB60210648029AFDF722FD0549002028
:10DE6000C877034800F058F810BC08BC04B0184745
:10DE700070500020B0500020F3B581B00D460198DD
:10DE8000FAF716FA144C86B22046FAF711FA81B264
:10DE90002046FFF75BFD0024002D0BD90F4F3846BD
:10DEA000FAF706FA81B23846FFF750FD641CA4B2B7
:10DEB000AC42F3D3084C2046FAF7FAF981B2204677
:10DEC000FFF744FD002E03D031460198FFF73EFDD9
:10DED000304603B0F0BD000020A700012CA70001D0
:10DEE00030B40125074B084CAD0203E06254491CD5
:10DEF0001981401C0278002A02D01989A942F5D361
:10DF000030BC70474E4700208B5800200149086004
:10DF1000704700004047002010B5074909680029F4
:10DF200001D0884710BD0446FAF7C2F981B22046F5
:10DF3000FFF70CFD10BD000040470020F0B51FB4F6
:10DF400005460398144646000198760847007F0866
:10DF5000334628463946FAF7FFFE02D228463946AC
:10DF600001E0204631463322D243FAF721FE06462D
:10DF70000F4622462846039B0199FAF72BFD4900DC
:10DF800049083B463246FAF7D3FE02D8012005B0D5
:10DF9000F0BD002005B0F0BD02460020802901D967
:10DFA0008D207047062A06D0072A07D0082AF8D104
:10DFB0000729F5D170470829F2D170470629EFD318
:10DFC00070477047704770B5C468054660680028A0
:10DFD00003D00020002802D00CE00120FAE7201D29
:10DFE000FBF7E8FA09F498D46068002808D000200C
:10DFF0000028F4D00020E860204609F48DD470BDDC
:10E000000120F5E730B40446A2890920521C93B2DE
:10E01000E48900222546D540ED0707D05D1C8D42DE
:10E0200002D130BC104670479B1C9BB2521CD2B22E
:10E03000092AEFD330BC7047FFB585B00E9D04466A
:10E040002F8801201E4600213A46CA40D20704D03C
:10E050004B0003225B1C9A401043491CC9B209299A
:10E06000F2D3049030461E210840218A184A00232A
:10E070000191009302920390132304AA1549069874
:10E08000FBF79EFA009000281FD10121142009F40B
:10E09000CDD40746E06006980188B9812988F981C6
:10E0A000F00701D00120C003079908433880208A77
:10E0B000788014206082204600F060F8381DFBF75D
:10E0C00085FA208A002109F407D6009809B0F0BD2E
:10E0D000D04401010A18000000487047684501015A
:10E0E000FFB5087881B00C46092836D2142003F019
:10E0F00089FC0746217800F0EFF800282BD06178E2
:10E100002078FFF749FF060028D17D68002D0ED04A
:10E1100020782979814207D12946381DFBF75CFA1E
:10E12000284609F4F9D302E02D68002DF1D160787A
:10E130000121083009F47AD40546207828716078E6
:10E1400068716278A11CA81DFAF78EF82946381D5F
:10E15000FBF748FA02E0822600E081260223064807
:10E16000039A049909F4E8D421780170467009F4FF
:10E170001FD5002005B0F0BD0114000010B5044605
:10E18000142003F03FFC0449216003216181123017
:10E1900060600120208110BD78450101F8B5174667
:10E1A0000C46104609F486D5012831D1142003F01D
:10E1B00029FC0546017C00F08FF80646297C227870
:10E1C0001448914214D1697C637809023A46891D4A
:10E1D0009B1D09F4B1D405460680002028716078A3
:10E1E00068806278A11C681DFAF73EF8284609E0AD
:10E1F000697C062309023A46891D09F49DD40680EC
:10E200008021017109F4D4D40021384609F464D581
:10E210000020F8BD140C0000F8B50F460024097862
:10E220001846254609291DD20B007B441B79DB18B3
:10E230009F440407101313130A160D00052414A598
:10E2400010E00A2414A50DE0082416A50AE007240E
:10E2500017A507E00A2418A504E0052419A501E084
:10E2600006241AA50146A31C1A4809F465D40646DB
:10E27000387830707470002C04D022462946B01CC7
:10E28000F9F7F2FF304609F493D40020F8BD0000FE
:10E290004E53494E470000004E532D424C452D3100
:10E2A0002E300000123456FFFE9ABCDE0000000043
:10E2B000025E044000000300312E302E302E302D3F
:10E2C0004C450000312E302E30000000FFEEDDCC3A
:10E2D000BBAA00000314000010B48289C489521C38
:10E2E00093B200222046D040C00706D0914202D10E
:10E2F0005B1C9BB205E09B1C9BB2521C52B2092ACC
:10E30000F0DB092A02D010BC1846704710BC002070
:10E310007047000070B5050005D0134E3068854287
:10E3200003D1002070BD72B6FEE704F03DFF6C69BA
:10E3300004F046FF7068844202D0B068844201D184
:10E34000022070BD0948844204D1A86A0028F7D190
:10E35000032070BD0648844203D0002C01D0012068
:10E3600070BD042070BD0000B4470020C45F0020D1
:10E37000B05F0020002802D00368002B01D10020EC
:10E380007047F8B50D4641680446002902D0A068E0
:10E39000884211D21B4EB5420ED8A2686D1C50198E
:10E3A000814201D39818F8BD2169002904D116498A
:10E3B000884203D9B04202D90020F8BD4600226A43
:10E3C0000027002A05D0314618469047050012D094
:10E3D0000CE0A1693046884705000CD0A26821688E
:10E3E000521CF9F741FFE1692068884766602560A3
:10E3F000A0684019F8BDE16920688847676000207F
:10E400002760F8BDFFFFFF7FFFFFFF3F70B50D4D99
:10E4100004460A2809D10D212846FDF719FA802162
:10E420002846FDF7A5F90028F9D0E1B22846FDF706
:10E430000FFA80212846FDF79BF90028F9D02046E5
:10E4400070BD000000380140F0B50878324F334D00
:10E45000334E801E83B00C46062859D20100794401
:10E46000097949188F4402255434543A01203070F8
:10E47000A0786876A078C00705D02A492A48FBF71B
:10E4800087F8387AA874B28A002A06D0FF20F530BF
:10E4900070800321254809F411D6F169002937D08D
:10E4A00000200090019005206A4610706846884759
:10E4B0002EE000246C7601F0FDFDF169002927D0E3
:10E4C000009406206A4601941070684688471FE051
:10E4D0001722A11C1648F9F7C7FE19E0B878000109
:10E4E000C0194030807D002812D11C22A11C114887
:10E4F000F9F7BAFE0F48A18A0182E18A4182218B95
:10E500008182618BC1820B49608A0883207F687495
:10E51000002003B0F0BD0000C04D0020044D0020DD
:10E52000204D0020C94D0020174D0020040F000091
:10E53000FE4C0020E44C0020F0B518460D46014684
:10E5400085B022230322744809F4F6D2012104463F
:10E55000417028780B286ED2010079440979491856
:10E560008F4405CDCDCD6F6ABB23CDCD6C0001208E
:10E57000207060706948817921710179A170C17939
:10E5800061714179E170017AA171417AE171817A19
:10E590002172C16900294ED00020009002206A46F5
:10E5A0001070684601948847A9E007202070012078
:10E5B000607068461DF452D0019F009EF9F742FE3C
:10E5C000801960820025F9F73DFE811960190090DD
:10E5D0008170F9F737FEC11900986D1CEDB2017515
:10E5E000082DF0D30825F9F72DFEB9194018611947
:10E5F0006D1CEDB28870102DF5D31020207748489F
:10E600008178090108184030807D012877D11C22CB
:10E61000A11C4448F9F728FE4248A18A0182E18AF8
:10E620004182218B8182618BC1823E49608A08834D
:10E630003D48217F417462E0052000E00A202070FF
:10E640005DE0042222706878012804D0002802D0FE
:10E65000022833D053E00120304D6070287C002820
:10E6600010D002A81CF4FAD7F9F7ECFD2F49F9F7FE
:10E6700089FD2F480818029940182E49F9F782FDA4
:10E68000009101E0E8680090E969002907D00020C6
:10E69000029003206A46107202A803928847102154
:10E6A000A01CF9F7FAFD0098A0700098000AE0702D
:10E6B0000098010C2171000E607120E01748C169BB
:10E6C000002905D00020009001906846027088471C
:10E6D00020460C3809F462D214E00620164D207052
:10E6E000E878012811D01021A01CF9F7D6FDA988DF
:10E6F0006182E988A1822989E18200202076204672
:10E7000009F456D2002005B0F0BD10220B49A01C20
:10E71000F9F7AAFDEBE70000140E0000204D0020E1
:10E72000C04D0020E44C0020044D0020A0BB0D0093
:10E73000A08601003F420F00444E0020CF4D002034
:10E7400000B5084883B0026C002A08D00020009071
:10E75000029005206B461870684601919047002092
:10E7600003B000BDC04D002010B584B0FF2B19D000
:10E77000144C226C002A08D0002000900290062041
:10E780006B461870684601919047032009F492D2B5
:10E79000032814D1A26F002A11D003210A4809F4DA
:10E7A0008DD40CE009480123007F032201020848B0
:10E7B000083109F4C1D10721017009F4F9D1002011
:10E7C00004B010BDC04D0020090E0000204E0020F6
:10E7D000050E0000FFB5180A4C4E83B00C46B07011
:10E7E000FF287DD00102342303224948083109F46F
:10E7F000A3D10546B07800270101891940318872FC
:10E80000B07821880001801940300181B078617AA8
:10E81000000180194030C172B0786289000181190D
:10E8200040318A81A289CA81E0890882207C01283E
:10E8300002D0002807D00BE0B17801200901891926
:10E840004031887504E0B078000180194030877548
:10E8500020883080607A307221460A312D48FAF7DC
:10E8600097FE02F0F9F900281BD0607A012804D144
:10E8700003221146284809F4AFD102F0F5F9052822
:10E880000FD201007944097949188F44060606021F
:10E89000060001202821485505E005212820415582
:10E8A00001E0282047550321059809F415D21720C7
:10E8B0003086B17809018919403148821748C0680B
:10E8C000002803D00321164809F458D31548028DB7
:10E8D000002A03D00321144809F4F0D3306C00E07F
:10E8E0000EE0002808D002206946009708700295C3
:10E8F0000194316C68468847284609F459D101E0F3
:10E9000001F050FB002007B0F0BD0000C04D00201A
:10E91000020E0000C94D0020150D0000D04E002051
:10E92000030F0000444E0020020F000030B5180A0B
:10E93000144D00010C46401983B0FF214030817214
:10E9400001F004FC002803D10221032009F4C4D102
:10E950002A6C002A08D0002000900290032069460B
:10E96000087068460194904710210748F9F795FC14
:10E9700006480068002802D0092008F497D7002034
:10E9800003B030BDC04D0020DF4D0020100C002032
:10E9900000B5084883B0C169002907D00020009065
:10E9A000019009206A46107068468847002003B02D
:10E9B00000BD0000204D0020FFB591B00D46122390
:10E9C00003224348149909F4B7D00021044601708A
:10E9D00040480078002862D03E48407C002833D070
:10E9E0003C216846F9F759FC01F028FF002841D086
:10E9F00004A90F913749461EF0B23A228969504363
:10EA000041186846091DF9F72FFC6846008B2988D4
:10EA1000884206D10822A91C0F98F9F768FC002843
:10EA20000BD0207800280BD008A8407C60741022FE
:10EA30006946601CF9F718FC1CE001202070F3E720
:10EA40003006000ED6D12AE023482988008B884260
:10EA500025D10822A91C2148F9F749FC002809D131
:10EA6000012020701E481022407C60741A49601CEE
:10EA7000F9F7FAFB2078002811D01648C16900295F
:10EA800007D000200090019007206A461070684669
:10EA90008847204609F48CD0002015B0F0BD0D4801
:10EAA000C169002907D000200090019008206A4623
:10EAB000107068468847022303220A48149909F413
:10EAC0003BD0012101700621417009F471D0E0E7CB
:10EAD000180E0000204D0020E44C0020F44C0020D3
:10EAE000044D0020040E000070B50C4609781B4848
:10EAF0001B4D1E46002904D0012912D002292BD11A
:10EB00001AE01C23314609F417D0064620783070ED
:10EB1000287B70802A7B1349301DF9F7A5FB30460E
:10EB200007E00A23314609F407D02178017069898A
:10EB3000418009F43DD00FE00A23314608F4FCD7A8
:10EB400021780170298C4180698C8180A98CC180D9
:10EB5000E98C018109F42CD0002070BD0B0E00005F
:10EB6000444E0020514E002010B5087800F058FFA8
:10EB7000002010BD05480A8842861A0A12011018A2
:10EB8000098840308182002070470000C04D00207D
:10EB900030B5180AC043000683B00D46000E21D0E0
:10EBA000190A0902E120062303220001083108F4B2
:10EBB000C3D704460120207002206080FF2041302E
:10EBC000A0800B48026C002A08D00020009004208E
:10EBD000694608706846019502949047204608F4FB
:10EBE000E7D701E001F0DEF9002003B030BD0000FE
:10EBF000C04D002000B5084883B0026C002A08D040
:10EC000000200090029008206B4618706846019121
:10EC10009047002003B000BDC04D002070B51846DD
:10EC20000C46014602230A4808F486D705460949DE
:10EC3000A07808736288211D0748F9F715FB0020AA
:10EC4000687020782870284608F4B2D7002070BD7C
:10EC50000D0E0000444E0020514E00204A780B4813
:10EC6000002A05D02030012A08D0022A09D00AE063
:10EC70000279012A07D10978C17004E00978017589
:10EC800001E009784175002070470000C04D002068
:10EC900070B54878002806D0FF25124C01280BD00B
:10ECA000022816D01BE010480179062917D1072148
:10ECB000017101F0E5F812E0207DFF280FD001F08E
:10ECC000DDF90A4825750169002908D00020884728
:10ECD00005E0607DFF2802D001F0B2F965750020E3
:10ECE00070BD0000E04D0020C04D0020D04E00203F
:10ECF00010B5032B06D010220548891DF9F7B4FA88
:10ED0000002010BD0348017A034801F04DFEF7E7EB
:10ED1000DF4D0020C04D0020C94D0020F0B50D464C
:10ED20000878E34EE14934464978002720348DB015
:10ED3000A1287AD012DCDF490C911B2876D006DCA2
:10ED4000012819D003287CD017286DD14FE128283D
:10ED50006ED091286DD0A02866D152E10246A23A29
:10ED6000092A61D213007B441B79DB189F44FE5CA7
:10ED7000FDFD5CFDFCFDFD006878002854D10120FC
:10ED800002F0A4FE01F04EFE342303220721CA48FC
:10ED900008F4D2D603210170C84904468A7842702B
:10EDA0000122C276FB224284C54AC284C54A8284BB
:10EDB0000A88028487768A888280CA88C2800A8903
:10EDC0002281487A8009032805D1887805221042DB
:10EDD00001D10120A076A07E04221043A076BA487B
:10EDE0006080C878012825D0204610210A30F9F724
:10EDF00054FA316C002907D001206A460097107040
:10EE00006846019502948847012000F009FE2046DB
:10EE100008F4CED6012303220721AC4808F48CD68F
:10EE20001A21017008F4C4D633E11EE1CAE008E0FB
:10EE300069E049E0204610220A300C99F9F714FAEB
:10EE4000D7E70097019702970397049705970697CE
:10EE50000797089709970A970B9701F0FDFE00287E
:10EE600005D0684601F03EFD0AA801F00BFD01F057
:10EE7000F3FE00280CD068468079002808D108A845
:10EE8000807B002804D00121684601F071F900E17F
:10EE90008A4C6946A0880880E0884880208988805C
:10EEA0008F71102202A80C99F9F7DEF9E078012899
:10EEB00004D00697079708970997E4E7102206A859
:10EEC0000C99F9F7D1F9DEE7E07B002813D1112383
:10EED000032207217E4808F42FD6054628202870F3
:10EEE0007648C078012808D01021681CF9F7D5F9B8
:10EEF000284608F45DD6E773CBE01022681C0C9915
:10EF0000F9F7B2F9F4E7012002F0E0FD0121032056
:10EF100008F4E2D66F48012444841F200490674817
:10EF20000178490601D57F2104918178052211429B
:10EF300004D0FF2204998132114304910088C00556
:10EF400004D503210498490208430490082162482B
:10EF50000191029003210B2304AA00970394C90294
:10EF60005E48FAF72DFB02E079E04AE089E00028EC
:10EF700046D15B4806218786FF20059059480191BC
:10EF80000290082305AA0097039457495748FAF7B7
:10EF900017FB00287DD100F05DFF002879D1022108
:10EFA000032008F499D6B079012808D001F022F89E
:10EFB0003E484078C0076CD001F064FB69E000F087
:10EFC000F1FF66E001F048FEE77300F043FF002820
:10EFD0005FD10221032008F47FD6B0790128EED05A
:10EFE00001F008F831484078C007E5D151E0687871
:10EFF00000284ED0F179481EF0713D4801F0A4FC84
:10F0000047E07179491E052906D8A72802D1307931
:10F01000002806D100F034FF2878A42801D0A728C2
:10F0200037D17079042806D0062804D0082808D0E3
:10F030000C282ED10CE02F480168002929D0B07986
:10F0400004E01A480169002923D00120884720E004
:10F050001648016900291CD00320884719E0377140
:10F06000FF20F0702075607513E0207DFF2802D02E
:10F070006878002802D001F001F80AE0C8079BD1A7
:10F0800007E0607DFF2802D06878002804D000F0F7
:10F09000D7FF00200DB0F0BDA07D0028F9D0880773
:10F0A000F7D5E17D144801F05BFAF2E7D04E00207D
:10F0B000C04D0020CF4D0020040D0000444E002024
:10F0C0000502000048080000A08C0000190D000097
:10F0D000230D0000B00B00204C490101D20B002091
:10F0E000680B0020A4490101011800009C0B0020BE
:10F0F000C94D0020704E0020F84D002070B500254D
:10F100000C462846401C0628FCDB254E2246307E55
:10F1100031461A32C96906282AD203007B441B797A
:10F12000DB189F4424020910171E0622A01CF9F7C1
:10F13000DEF800281BD01BE0237E092001F0B0F888
:10F14000002814D114E0237E212001F0A9F8002822
:10F150000DD10DE0237E162001F0A2F8002806D183
:10F1600006E0237E192001F09BF8002800D001253D
:10F170000C48807D002811D17169002901D02046FA
:10F180008847002D0AD03169002901D00220884724
:10F1900001F0FAFA217AA01C01F0E2F9002070BD1A
:10F1A000D04E0020E04D002010B50A78000A000281
:10F1B00010434A78FF231B02120298431A4010435F
:10F1C0008A781B02120498431A401043C97800023F
:10F1D000000A09060843F9F73EF8002010BD10B5F3
:10F1E000104608F467D5002010BD0020401C0628FA
:10F1F000FCDB002070470000F8B51C4617460D46A2
:10F20000104608F457D5002811D1472002F0FAFB28
:10F21000064604233A460321064808F48DD4210A01
:10F2200001702988B288891A418008F4C1D400206D
:10F23000F8BD00000D470000F8B517460C46472002
:10F2400002F0E0FB21780646122901D013291BD1D8
:10F25000B06805460C351229C288018916D00623EC
:10F260000F4808F469D4698841806178017108F415
:10F270009FD4B068002803D008F44ED30020B060BB
:10F280000021384608F428D50020F8BD042305489D
:10F2900008F452D46988018061788170E7E7000042
:10F2A000094700000747000000B5084883B0026C1A
:10F2B000002A08D000200090029009206B461870A8
:10F2C000684601919047002003B000BDC04D00206A
:10F2D00030B5104D83B0088828861C0A20014019DB
:10F2E0000A88403042822A6C0025002A07D0009507
:10F2F00007206B46029518706846019190470648B2
:10F30000A1004058002801D04030C574002003B04F
:10F3100030BD0000C04D0020580B0020FFB581B06B
:10F32000002000900E46039808F4C4D4002802D0B0
:10F3300001284CD04DE0142002F064FB07463188D0
:10F34000FEF760FE05462448092D36D27C68002C65
:10F350001ED02179A94203D02468002CF9D117E0EE
:10F36000002C15D06379039A9B1D049908F4E4D30B
:10F37000054630882880002028716079688062798D
:10F38000A11D681DF8F770FF284608F411D420E08D
:10F390003D740498010A7974384602F02BFB01464B
:10F3A00001230E48039A08F4C7D3057008F400D46B
:10F3B0000121039808F490D40BE00623039A0499E2
:10F3C00008F4BAD33188018080210171DDE7022081
:10F3D0000090009805B0F0BD140C0000021400006D
:10F3E000FFB585B00E46079808F464D4002802D013
:10F3F000022009B0F0BD472002F004FB029000207B
:10F40000694608700898070A308803F000FA00245B
:10F41000694605468C8000281ED102981622016A92
:10F420006846007803465043024610328A5A520416
:10F43000920F1FD10A5C401C085C1E490002101884
:10F44000884217D102AA03A9184603F0F3F80298DC
:10F450006946C05D88800224A31D1748079A089951
:10F4600008F46AD30746308838803D717C80002DCF
:10F4700015D019E03946029802F0BCFA014604237F
:10F480000E48079A08F458D30770694609784180F6
:10F4900008F48ED30121079808F41ED407E0224611
:10F4A00001A9781DF8F7E0FE384608F481D3002062
:10F4B00009B0F0BD02290000140C00000447000050
:10F4C000FFB58BB00C46472002F09CFA0025694638
:10F4D00005900D740E9804A9070A208803F097F987
:10F4E000060061D105981622016A6846007C5043E7
:10F4F000024610328A5A5204920F3AD10A5C401CDA
:10F50000085C304900021018884232D102950395F8
:10F51000208800F0DFF802A9002300911A4608A90C
:10F52000FAF766F86846008C012109030840C043D9
:10F53000C004C0172146401CFEF70AFC0606360E22
:10F5400032D168460997007C0190A57907AA6946DF
:10F5500003F070F86846028806A80799F8F784FE59
:10F5600006A909980A460D5468460188019803F0D7
:10F570009FF83946059802F03DFAA1880D9A891D39
:10F580008BB20146104808F4D7D20546A288A11DC7
:10F59000801DF8F769FE2F706846007C6880A0889F
:10F5A000A880284608F404D3042308480D9A0E992D
:10F5B00008F4C2D221880180867008F4F9D20020B4
:10F5C0000FB0F0BD022900000A470000160C000031
:10F5D000F0B589B00446FAF711F805460026154F34
:10F5E0001BE006A92046F9F7D9FF002302AA01A9CA
:10F5F00006A80096FAF708F868460089B84203D1D1
:10F6000069460979022911D00B49884203D168461D
:10F610000079022807D0641CA4B2A888A04202D8AE
:10F62000E888A042DDD2002009B0F0BD204609B034
:10F63000F0BD00000229000003280000F7B50028F3
:10F6400045D00199002942D08668002A01D10CE0FA
:10F650003668002E3BD0316A002938D00198F8F77F
:10F660002EFE0028F4D12CE03668002E2FD0019C0D
:10F67000356A002CF8D0002DF6D0AC4224D020788A
:10F68000F8F7DAFD07462878F8F7D6FD87420DD15E
:10F690002078002813D06078641C6D1CF8F7CCFD2E
:10F6A00007462878F8F7C8FD8742F1D02078F8F7A8
:10F6B000C3FD04462878F8F7BFFD8442D4D1002E5C
:10F6C00005D0306A002802D0304603B0F0BD0020DB
:10F6D00003B0F0BDF0B589B00446F9F78FFF0546D9
:10F6E0000026104F14E006A92046F9F757FF002323
:10F6F00002AA01A906A80096F9F786FF68460089C4
:10F70000B84203D1641CA0B209B0F0BD641EA4B21B
:10F71000A888A04202D8E888A042E4D2002009B01C
:10F72000F0BD00000328000070B5164C20780028BA
:10F7300027D101210803FBF775FE0020FBF768FEC7
:10F740000120FBF793FE104D2846FAF70BF8032132
:10F750002846FAF777F801212846FAF737F8012109
:10F7600021702846FAF75AF8142003F065FD70203E
:10F7700000F00CF8702000F009F800212846FAF794
:10F780004DF870BD944700200008024070B5054652
:10F79000164CFFF7C9FF2946154D2846F9F76DFFAE
:10F7A00001212846FAF708F801212846FAF742F81D
:10F7B000002807D1641E13D001212846FAF73AF831
:10F7C0000028F7D001212846F9F754FF2846FAF718
:10F7D0002EF8044600212846F9F7EEFF204670BDBA
:10F7E00000212846F9F7E8FF024870BDA086010015
:10F7F00000080240FFFF0000F7B504270225494E2C
:10F8000086B01446082A74D2100078440079001893
:10F81000874484030D3A3D5363704348019001AB24
:10F8200000970799069800F08BF809B0F0BD3F4F9C
:10F8300001213846F9F7F2FF142003F0FDFC702097
:10F84000FFF7A4FF7020FFF7A1FF04460021384610
:10F85000F9F7E4FF3648B442448001D1354808E066
:10F860002046F9F711FF3449F8F7D2FFF9F7EEF91E
:10F8700000B2694688812A4603AB0095079906982D
:10F8800000F05EF809B0F0BDFDF7B2F90AE06020C3
:10F89000FFF77CFFB04201D1002003E06021F9F7BF
:10F8A0001DFF80B26946088102AB22460095079988
:10F8B000069800F045F809B0F0BD04F0FFF97D218D
:10F8C000C900F8F75FFC019001AB22460097079949
:10F8D000069800F035F809B0F0BD03F0E9FD01909D
:10F8E00001AB224600970799069800F029F809B065
:10F8F000F0BD13E0FDF73AFB1049884201D1022028
:10F9000000E00120694608740120009004AB224603
:10F910000799069800F014F809B0F0BD079809B0EF
:10F92000F0BD0000FFFF00001500010000080240CC
:10F9300094470020FF7F00000000204100400201AA
:10F9400030B4029C42540546491C88B22C54401CD9
:10F95000002180B2002C07D95A5C2A54401C491C53
:10F96000C9B280B2A142F7D330BC704710B5084C81
:10F9700082B02078002808D10648009006480190FF
:10F980006846FEF7D5F80120207002B010BD0000D7
:10F99000B047002005250101DD310101F8B50B302C
:10F9A000C608F600104D19E02068B04215D3B042E9
:10F9B0000BD96368871B201D0093F8F755FCA0192D
:10F9C000009B07604360286004E060682860201D99
:10F9D000F8F74AFC201D2660F8BD251D2C68002C78
:10F9E000E2D10020F8BD000010480020FF25F535C9
:10F9F0000A4E6F00FDF790FB0489322C00D22C4692
:10FA000001213046FBF7F0FB7D212046C900484329
:10FA10003946F8F7B7FB03F00FFCEBE7000C0140A9
:10FA200010B5A0230949022809D0002203280AD0D2
:10FA3000042808D00B704A7000F0A2F810BD0B70BB
:10FA400080204870F8E7E0200870F4E711400020BB
:10FA5000F8B52A492020486029480121C163294975
:10FA600005228A610021C16327490B20086100F04B
:10FA700087F82748254A026326494163264B83635A
:10FA8000264CC4632748264D0560274E466027490B
:10FA900081602749C16027490161274941612749A0
:10FAA000816127490163284826494160274FC76083
:10FAB000274F07610262274A42628362C46205637C
:10FAC0004663254A8263254AC2632648244A026067
:10FAD000184A4260244A82600163244981632448B1
:10FAE000244A41688918244A914206D223498268EF
:10FAF0000A63C2684A6300698863F8BD0010014068
:10FB0000C027024040250240402702400259F80029
:10FB100040280240025B8500025A8000025D850099
:10FB2000025F80508028024002000878020A080024
:10FB3000026EAC500259FC000200C800127013148F
:10FB400002700314026E2800C0280240025D050006
:10FB5000125B0500025B8400020A0600026E2C5054
:10FB600002C3BF00002902401200AC00125D050074
:10FB7000104000206F2895FFAF590F00C0260240AB
:10FB800030B415481549037D154AFF2B06D1407D39
:10FB9000FF2803D113484078C0070CD01248134BFC
:10FBA00004789C604078D86111480861114B8B62E1
:10FBB000106030BC7047104B0B6110484861104C0E
:10FBC0008C61104D8D62C8620F48086313600F4846
:10FBD0005060946030BC7047E04D00200028024027
:10FBE00040280240D04E0020114000200027024053
:10FBF000127E0200127E0300027E020002C2A000FA
:10FC000012C70000027E030012C7800002C2E0009B
:10FC100082B0224920480863FDF78AFD20A0FBF747
:10FC20001BFE2AA0FBF718FE31A134A0FBF714FE3F
:10FC30003848016838A0FBF70FFE3EA142A0FBF751
:10FC40000BFE4AA0FBF708FEFCF742FCFCF732FD76
:10FC500001215148FBF7CCFA40215048FBF7C8FA84
:10FC6000FDF75EFA01F03AF802200024020200904B
:10FC700023464BA101944B4803F054FF0120009010
:10FC80000023802248A10194484803F04BFFFAF773
:10FC9000F3F803F0ABFBFEE700800081007000404A
:10FCA0000A3D3D3D3D3D3D3D3D3D3D3D3D3D3D3DB7
:10FCB0003D3D3D3D3D3D3D3D3D3D3D3D3D3D3D3D74
:10FCC0003D3D3D3D3D3D3D3D3D0A0000206D636DA8
:10FCD0002D6464632D626C653A20424C45202B20D4
:10FCE0004672656552544F53202B20434C490A00FD
:10FCF00056312E30302E323100000000204669721D
:10FD00006D776172652076657273696F6E202573F9
:10FD10000A000000004000202053797374656D4391
:10FD20006F7265436C6F636B203D20256C752048B6
:10FD30007A0A000043414949432D4D434D2D32304D
:10FD4000323630393032000020424C4520656E6139
:10FD5000626C65642C206164766572746973696E87
:10FD60006720617320222573220A00003D3D3D3D3E
:10FD70003D3D3D3D3D3D3D3D3D3D3D3D3D3D3D3DB3
:10FD80003D3D3D3D3D3D3D3D3D3D3D3D3D3D3D3DA3
:10FD90003D3D3D3D0A000000000C014000080140CF
:10FDA000424C450085D400014C454400EDF900016A
:10FDB00010B50124E4022046FBF706F9002805D01F
:10FDC0002046FBF7FBF80D490220087001242403AC
:10FDD0002046FBF7F9F800280AD02046FBF7EEF89A
:10FDE000BFF34F8F07490648C860BFF34F8FFEE748
:10FDF00005484068002800D0804710BD80000020E2
:10FE00000400FA0500ED00E04040002006480068CC
:10FE1000002800D08047BFF34F8F05490348C860D2
:10FE2000BFF34F8FFEE70000404000200400FA05BA
:10FE300000ED00E0064A11780A2907D289008918E6
:10FE400048601078401C10700120704700207047F7
:10FE5000404D002010B5084C084AE1791378002085
:10FE6000994207D28800801840688047E079401C9A
:10FE7000E071012010BD0000C04D0020404D002069
:10FE8000F8B5324D0526297928468079304C082965
:10FE90000CD20A007A4412799218974403080D1381
:10FEA00013191C2A052801D0FCF78CFDF8BD022887
:10FEB00008D0FDF7AFF9F8BD607B002802D1E079EA
:10FEC000002802D0FDF744FAF8BDFDF7DFF9F8BDD0
:10FED00006202871F8BD0223032207211D4807F4DC
:10FEE0002BD6A5210170E9784170072129716E7127
:10FEF00028E0022303220721174807F41DD60746EE
:10FF0000A7203870E9787970062068710020287180
:10FF1000032007F4CFD6032812D0A879012804D0F3
:10FF2000022802D003280BD104E0207D002801D054
:10FF3000032003E0A07E002802D00420A87100E086
:10FF4000AE71384607F434D6F8BD0000C04D00202D
:10FF5000B04E0020A20D0000A30D000010B5002837
:10FF600004D0014660220C48F8F77EF90B490C4892
:10FF7000CA781C2A04D9427B002A01D11C22CA70EB
:10FF8000C1781F2901D91F21C170017BE22901D944
:10FF9000E221017310BD0000704E0020904E002041
:10FFA000B04E002011490122087907280CD0887929
:10FFB000002809D0012801D0052806D10C48827BF1
:10FFC000002A03D002200CE08A717047027D002ACB
:10FFD00001D0032005E0807E002801D0042000E04D
:10FFE0000520887110B5FCF7EDFC10BDC04D002058
:10FFF000B04E002070B5104C0525A079062809D216
:020000040101F8
:1000000001007944097949188F4402020404040369
:10001000A57170BDA571022303220721074807F4CB
:100020008BD5A5210170E17841700721217165719F
:1000300007F4BED570BD0000C04D0020A20D000029
:1000400010B50B4C607DFF2810D00223032207213E
:10005000084807F471D5A7210170617D4170064AF7
:1000600000215171FF21617507F4A2D510BD000078
:10007000E04D0020A30D0000C04D002010B50A4C3B
:10008000207DFF280ED0022303220721074807F412
:1000900053D5A7210170217D4170054A002151717E
:1000A00007F486D510BD0000E04D0020A30D000030
:1000B000C04D002010B508480223807803220102B9
:1000C0000648083107F438D5012101701321417029
:1000D00007F46ED510BD0000C04D0020040E0000D6
:1000E00010B584B0002804D001462A220E48F8F743
:1000F000BBF80EA00FC86C460FC40B4B002069461E
:100100001C180A5C247922430A54401CC0B20628F9
:10011000F6D310220A48F8F7A7F80A490A48F9F76F
:1001200037FA04B010BD0000444E00205019219051
:100130001F04D5624FA489AB90D0CF2300000000EC
:10014000CF4D0020484E0020FC0000200020074B2F
:1001500001460A01D2184032927AFF2A01D0401C8F
:10016000C0B2491CC9B20329F3D37047C04D002067
:10017000F8B507460B46282043430D4603220721C6
:100180000E489B1C07F4D8D4912101700024064628
:100190004570002D0ED9204628214843C119002260
:1001A000CA7180192822801CF8F75EF8641CE4B23A
:1001B000AC42F0D3304607F4FBD4F8BD910D0000FB
:1001C000F8B57D262025F600184B194C194903284F
:1001D00012D00A6A01273A430A620A6A9207FCD5DA
:1001E0000A6AAA430A6201281AD002281AD01E609D
:1001F000F9F710FA2060F8BD0F480F2782683F0218
:100200003A438260086A042210430862086A0007C1
:10021000FCD5086A284308623D2000011E60E9E71A
:10022000064800E006481860E2E700008C00002065
:10023000900000200010024000100140D103000097
:100240005704000010B504460848042380780322B0
:1002500001020748891D07F46FD406494C8001212B
:1002600001700021418007F4A3D410BDC04D0020CF
:10027000010C0000F00B0020084A11780A290AD26C
:10028000C9004368891800688B6048601078401C7A
:100290001070012070470020704700006C4D002056
:1002A000FFB581B01C00064618D01078411CA14251
:1002B00014D8032C12D3401EC5B25078971CB042FC
:1002C00006D12A4638460299F8F711F8002808D0D6
:1002D0007A19601B801E0406240EE6D1002005B0AA
:1002E000F0BD012005B0F0BDF0B504466F4E70487A
:1002F00083B06D4FB168C1626E490163F16A81627A
:10030000F16B4163B16B816331467C2240313846E9
:10031000F7F7AAFF00257D60FD607D626648B86240
:100320007D64BD64FD643D666448B86664483862B7
:10033000644865490570032008706448F914016039
:100340000904016089140160F06861490746401E94
:100350000088604B884200D01F60366E701E008897
:10036000884200D05E60012000030090694601953C
:100370000D710820487101278F716846FAF732FE27
:1003800084215548F7F789FF2A215448F7F785FF5C
:1003900060215348F7F781FF52484F490561456195
:1003A0008561C561056245628562C562FF264E486A
:1003B000CE70067546750020020152184032401C6E
:1003C000C0B296720328F7D3206808646068486456
:1003D00046486189C187217A4548032901D8417778
:1003E00000E0457701212020FBF71CF8414A4249F3
:1003F000042001F099FA4249404808600A46414900
:10040000052001F091FA404A4049072001F08CFA9A
:1004100040493F4808600A463F49082001F084FAF5
:100420003E4A3F49092001F07FFA3E4805633E48B5
:10043000414907703D4805703D4805703D480860DA
:1004400001203E49C00208803D494F2008703D49C7
:10045000082008703C480721067046708670C170FD
:10046000057145718571C57111483849C1613849B7
:10047000016238494162002002F0E4FC3649032061
:1004800007F46ED40021032007F426D4002001F0E5
:100490001DFB012303220721304807F44DD30770C9
:1004A00007F486D303B0F0BDC0090020008000012E
:1004B000C00000200DFE00010D4700205D2F01014E
:1004C000B1FD0001C6000020D800002000E100E0DE
:1004D000FEE7000040400020C04D0020444E0020B8
:1004E000704E0020C04E0020E04D0020004E002045
:1004F000204E00208040002080800100194601012C
:10050000C0400020C08001000041002000DB01004D
:10051000814100204041002040DB0100C046002016
:10052000C06102000070004060000020C90000208F
:10053000610000200090D0036C00002068000020C3
:100540006300002064000020080100206D190101F3
:10055000951A0101351A0101AC4A0101020D000092
:10056000F8B5404D0646687D3F4C0F46FF281CD02D
:100570002046C268002A03D003213C4807F49ED5D8
:100580003A23032207213A4807F4D6D2A421017066
:10059000697D0446417037480022017800291ED049
:1005A0000121A170A28002701BE06D2002230322B2
:1005B0000721400107F4C0D2A22101702E49C97859
:1005C000417007F4F5D2EF7531462C48F8F7E0FF9B
:1005D0000120A8756078022108436070F8BDA27000
:1005E000A2800120E07019214901E1802248218187
:1005F000038CE381438C2382838C6382C38CA3822C
:10060000FF23E2824133184D23836D786D070DD5AA
:100610000525E5706181A181018CE184418C2185F2
:10062000818C6185C08CA085E285238638200755A2
:10063000204631463230F8F7ABFFE078810703D52A
:100640000220FFF7EDF906E0400701D5032000E0A6
:100650000120FFF7E5F90A490C204871204607F40C
:10066000A7D2F8BDE04D0020D04E0020030F0000BF
:10067000A10D0000404E0020444E0020F84D002007
:10068000C04D0020F8B52C4E2C4D317D01276878E7
:10069000FF2941D0C1073ED0B843687028490020E7
:1006A00008703A2303220721264807F445D204465E
:1006B000A4202070307D60702878A0706878800653
:1006C000800F20716888E080A8882081E888E08118
:1006D00028892082E7700120FFF7A2F96878400797
:1006E0000AD5E07802210843E07068886081A88814
:1006F000A0810320FFF794F96878000703D5E0781C
:100700000C210843E0701049082048710020B075A2
:10071000204607F44DD2F8BD384368706D2002239F
:1007200003220721400107F407D2A12101700749E4
:10073000C9784170EDE70000E04D0020D04E002068
:10074000404E0020A10D0000C04D0020444E00206E
:1007500010B50A4C607DFF280ED00223032207212A
:10076000074807F4E9D1A5210170617D4170054A70
:100770000D21517107F41CD210BD0000E04D002086
:10078000A20D0000C04D002070B50B4C207DFF284D
:1007900011D00A4D687909280DD0022303220721C0
:1007A000074807F4C9D1A5210170217D41700921B5
:1007B000697107F4FDD170BDE04D0020C04D0020EF
:1007C000A20D000010B504464088A1880246491CCD
:1007D00019234A43DB019A420FDC06280DD32288F5
:1007E00090420AD3E2887D23DB009A4205D84B0071
:1007F000C9184843D100884201DD002010BD0D48D2
:100800000E238078032201020B48083107F494D1AB
:10081000092101702188418061888180A188C1807F
:10082000E188018100214181491E818107F4C0D105
:10083000012010BDC04D00200E0E000010B5084A6A
:10084000084B906901888478994206D1917CA14235
:1008500004D20024FAF79CFD00E00024204610BDDD
:10086000204D0020341200000B4610B504493A22F6
:100870008969504341181846091DF7F7F5FC10BD6A
:10088000204D002010B590B004463C216846F7F793
:1008900004FDFFF7D3FF401EC0B26946FFF7E4FF37
:1008A00008A8807CA0710CA920460331F8F770FEDF
:1008B00010B010BD10B590B004463C216846F7F763
:1008C000ECFCFFF7BBFF401EC0B26946FFF7CCFF50
:1008D00008A8007CA0710AA920460231F8F758FE4A
:1008E00010B010BD10B590B004463C216846F7F733
:1008F000D4FCFFF7A3FF401EC0B26946FFF7B4FF68
:100900000AA920460231F8F743FE08A8007CA0712E
:10091000204606A9102208300231F7F7A5FC084846
:10092000C17820461830012904D01021F7F7B5FC12
:1009300010B010BD10220349F7F796FC10B010BD9F
:10094000444E0020CF4D002070B590B00D460646B5
:10095000FFF774FF002D23D0854221D818230322EE
:100960000721104807F4E8D0044617202070012022
:1009700060703146A01CF8F70BFE3C216846F7F783
:100980008CFC6D1EE8B26946FFF76EFF204606A993
:10099000102208300231F7F767FC204607F408D12F
:1009A00010B070BD140D0000F3B58FB00C463C21A3
:1009B0006846F7F772FCFFF741FF012C1AD00028B8
:1009C00016D0154D0AAE0236441EE0B23A22A9698D
:1009D000504341186846091DF7F746FC0622314688
:1009E0000F98F7F784FC00280DD02006000EEBD1FD
:1009F00011B0F0BD0949421ECA7101460F98FFF7B8
:100A0000A3FF11B0F0BD06A9102205480231F7F787
:100A10002BFC11B0F0BD0000204D0020C04D002087
:100A2000DF4D002070B5284C82B020688003FCD5D3
:100A3000264D687FFFF7C4FB606A606A0126304379
:100A40006062606AB04360622148C08F0A2811D991
:100A5000E16932071143E1611E494A6832434A6045
:100A60001E491D4A0A6003224A6088601C480860CB
:100A70001C48086068461AF4F1D51B4900980860C4
:100A8000687FFF252D02032811D000F027F9206B85
:100A9000A8432063206B3F21490208432063206B59
:100AA0003043206301220321104807F407D3104884
:100AB0000168A94301600F490868FF2212049043AE
:100AC000086002B070BD000000100240204E0020FF
:100AD000004E0020401002405555000000300040FC
:100AE000AAAA0000CCCC000048400020010F000062
:100AF00000E400E008E400E0F0B5D7B054A81AF430
:100B0000ADD54A490024886AC96A54990122411A1C
:100B100009010909D206914204D95499081A000121
:100B200000094142424E40290CDC7088002809D05F
:100B3000401E7080142203213E4807F4BFD20020DB
:100B400057B0F0BD3C48FF21569029316846F7F771
:100B5000A4FB707CB569002832D0FFF76FFE6946B0
:100B60008870B17C6F4688420BD23A2148430246D6
:100B7000291D381DF7F778FB69468878401C887076
:100B800008E03A21401E4843024629463E31381DBE
:100B9000F7F76AFB694688783A214843C0190A4644
:100BA00036385699F7F760FB244869460880B069E3
:100BB000FAF7EEFBFF2227326946B069FAF716FC16
:100BC000FF20F53070804A944B944C944D944E9491
:100BD0004F9450945194529417485394418D40AA85
:100BE0001185818D5185C08D9085154C48AA257C35
:100BF0009573102213494CA8F7F736FB1248C078BA
:100C0000012804D11022114950A8F7F72DFB012625
:100C10000F48002DC67306D1A07C002803D0012107
:100C20004AA8FFF7A5FA0B48067088E7C080024083
:100C3000204D0020040F0000E44C0020341200007E
:100C4000044D0020FE4C0020444E0020CF4D0020DB
:100C5000E04D0020404E002002480078002800D0DF
:100C600001207047204D00200148007970470000A6
:100C7000204D002070B517493CC80E4684B0403660
:100C80003CC64368026880684B65134C0A658865FA
:100C9000607C002818D0002569460D72FAF78AFB9F
:100CA000FFF7CCFD69460872E1690126002906D0EC
:100CB00068460095067002A8019068468847684615
:100CC000007A002802D0267004B070BD257004B0F0
:100CD00070BD0000E44C0020204D0020044908684D
:100CE000401C0860012801D0012070470020704797
:100CF0002440002003490868002802D0401E0860F4
:100D00000120704724400020F8B50C462849294BA3
:100D10004118294F294A0026069D002908D001299B
:100D200022D0274940180A282FD301202870F8BD67
:100D300020780A2838D2214980000958214A914256
:100D400003D11E490E501E502EE0B9422CD1032271
:100D5000082311461C4806F4EFD62178017061681B
:100D6000416006F425D71FE020780A281CD28000B5
:100D70001158B94218D11958115020781349626896
:100D80004018032107F49AD10EE0C0B20A280BD212
:100D900084001159002907D0B94205D0094FB94242
:100DA00002D016511E5188472E700020F8BD000059
:100DB000FBF0FFFFBC4C002073300101944C00207D
:100DC000F9F0FFFF71300101060F0000070F00006E
:100DD000102909D810B50C460A4601460348F7F712
:100DE00043FA0348448110BD70470000725E002042
:100DF0005C470020F7B5524F387800280AD03846B3
:100E0000C369042A08D201221121009800F096F942
:100E100003B0F0BD002313E00C780D1D20464C7884
:100E2000240220438C7824042043CC7824062043D9
:100E3000CC780002000A24062043141F984206D0F2
:100E400002221121009800F079F903B0F0BD386951
:100E50001E19864206D903221121009800F06EF96E
:100E600003B0F0BDFE61786AB0420FD2796AF868CB
:100E70004018FAF78DFA002801D0052207E001207A
:100E8000796A000308187862B042EFD30022002A82
:100E90003CD1F86A002822D02A49042808D2002C24
:100EA0001BD02B780B54401C641E6D1CF862F4E7B9
:100EB0003E46042811D1316AF068224B40180422C2
:100EC0001946FAF793FA002801D0052203E0306AA8
:100ED000001D002230620020F062002A16D1042C8E
:100EE0001DD33A6AF868A608B6008018294632462B
:100EF000FAF77CFA002801D0052203E0386A80194D
:100F000000223862AD19A41B002A08D01121FB6908
:100F1000009800F013F9FBF75FFF03B0F0BD002C61
:100F200005D0224629460748F7F79EF9FC620022C1
:100F30001121FB69009800F001F903B0F0BD000039
:100F40005C47002084470020F7B56E4D8CB02878B0
:100F50000E4600280AD02846C369042A08D0012278
:100F600012210C9800F0EAF80FB0F0BD002312E057
:100F70003278F17810467278090612021043B2787E
:100F80001204104308430402F078240A00060443C4
:100F90002869834206D0022212210C9800F0CEF874
:100FA0000FB0F0BDE86A0026002815D0042806D24C
:100FB000554AFF211154401CE8620428FAD32B6AD9
:100FC000E86851490422C018FAF710FA00287DD1C8
:100FD000286AEE62001D28622969E868FCF79EFE17
:100FE000A04202D16969884209D004221221EB692A
:100FF0000C9800F0A3F8FBF7EFFE0FB0F0BDE86827
:10100000001D00F089F8E9680A460832904203D3CF
:101010002A698918814209D806221221EB690C98A5
:1010200000F08CF8FBF7D8FE0FB0F0BD374C6F46E0
:101030000FCC0FC70FCC0FC7A268616820680A9257
:101040000890334F0098203C0991B84206D12821DE
:101050002046FCF763FE0A9988420AD00096019662
:1010600002960396049605960696079608960996A4
:101070000A960097274AE968914201D1012000E0D1
:10108000022001909142684601D1083000E01830FA
:1010900001602969416069698160A969C16028218D
:1010A0006846FCF73BFE0A902046FAF771F90028E3
:1010B0000FD12C2269462046FAF798F9002808D16A
:1010C0002C2221466846F7F712F900E001E00028DB
:1010D00009D005221221EB690C9800F02FF8FBF7DC
:1010E0007BFE0FB0F0BDAE70002212212B690C9870
:1010F00000F024F802F0E2FD28630120E8700FB050
:10110000F0BD00005C470020844700200040000143
:1011100011C011CA008000010378C27819464378D3
:1011200012061B0219438378C0781B04194311432C
:101130000902090A000608437047000070B586B02E
:101140006C4621746274A374190AE174190C217538
:10115000190E61751E494C6B002C30D0CA216A46AD
:1011600011701F21517090700620D07000201071F6
:1011700004A9501DF8F70CFA16480923164D00AAC9
:1011800001321178090248400021521C060402D5A0
:101190004000684000E04000491CC9B280B2082904
:1011A000F4D319465B1E9BB20029EAD16946C87286
:1011B000000A08730D216846A04706B070BD0146BD
:1011C000062304AA1F20FBF76BFB06B070BD0000CE
:1011D0005C470020FFFF00002110000070B50C46A6
:1011E0000546FCF791FB21462846FCF7AFFBFCF7D0
:1011F0009BFB02490120887070BD00005C47002005
:1012000070B5FEF7B3FBFCF757FC04002FD01A4D66
:101210002889F7F7FFFC02460B4618A12046FCF789
:10122000FFFBE868F7F7F6FC02460B4614A12046E0
:10123000FCF7F6FB13480078F7F7ECFC02460B4688
:1012400011A12046FCF7ECFB2046FCF745FD0546C6
:101250002046FCF73DFC002D09D02846FCF75CFE3B
:101260000BA0FCF759FE2846FCF73EFD70BD09A017
:10127000FCF752FE70BD0000B45E00206C65640097
:1012800070776D009847002076616C6964000000FB
:101290000D0A00006A736F6E3A20616C6C6F6320F8
:1012A0006661696C0D0A000070B5134C0125607809
:1012B000002802D1FAF77EF8657010483021FCF75B
:1012C0002DFD0E490E4E08633046FAF761F80028EE
:1012D0000DD1342209493046FAF788F8002806D1A2
:1012E000342231460548F7F702F8002801D00120E2
:1012F00070BD2570002070BD98470020B45E0020AE
:1013000000600001F3B583B004980021066880688E
:10131000009137187D1C305C2C4622287ED1049821
:10132000406807E05C2A04D15B1C834277D2491CE9
:10133000641C641CA31B834202D22278222AF1D1AE
:10134000A21B82426BD22078222868D1E01B401A6F
:101350000499401C09698847009000285ED0A54286
:1013600070D229785C2903D00170401C6D1CD8E034
:101370000223611B012952DB6A78662A15D008DC3A
:10138000222A22D02F2A20D05C2A1ED0622A46D1BF
:1013900008E06E2A0DD0722A0FD0742A11D0752A57
:1013A0003DD115E00821017010E00C210170401CB6
:1013B000B6E00A210170401CB2E00D210170401C12
:1013C000AEE009210170401CAAE00270401CA7E0B9
:1013D0000022944606296FDBAF1C1346F95C0E46CB
:1013E000303E092E02D8303A8A180BE00E46413EB4
:1013F000052E01D8373A04E00E46613E052E1FD86F
:10140000573A8A18032B00D212015B1C042BE5D338
:1014100037218902531A55498B4201E09CE094E040
:101420007BD91B23DB02D31A8B423FD80C23A91D87
:101430009E46631A062B70DB0B785C2B6DD102E0A5
:101440000022E5E770E04B78752B66D1891C01918D
:1014500000210E46019B9B5D1F46303F092F02D89D
:10146000303959180BE01F46413F052F01D8373955
:1014700004E01F46613F052F16D857395918032E2F
:1014800000D20901761C042EE4D337239B02CE1A26
:1014900001239B029E4240D292058905120B890DC1
:1014A0000A439901521803E00021EEE706218E4617
:1014B000802A02D2012315E02FE00121C9028A42CD
:1014C00003D20223C0218C460CE0012109048A4288
:1014D00002D20323E02104E025498A421DD80423D7
:1014E000F0218C46591E0906090E0AD0164680279F
:1014F0003E43BF273E404654491E92090906090E45
:10150000F4D1012B03D961460A43027002E051066F
:10151000490E0170C018734600E00023002B14D060
:10152000ED18A54200D21CE700210170039810219C
:10153000C160039900980861049804990068201A12
:10154000401C8860012005B0F0BD0098002803D041
:101550000498416900988847002D04D004980068D9
:10156000291A04988160002005B0F0BDFF03000037
:10157000FFFF1000F0B591B00C0006467ED0216848
:1015800000297BD0A0686368021D9A4206D808181B
:101590000422DBA1F6F7C1FE002833D0A068626800
:1015A000411D914207D8216805220818D6A1F6F7F7
:1015B000B4FE00282ED0A0686268011D914207D8B1
:1015C000216804220818D2A1F6F7A7FE002829D026
:1015D0006268A168914203D22068405C22282BD027
:1015E00091427AD22068405C2D2802D030380928F8
:1015F00073D800200146109020682E22002807D0C2
:101600006B464DE00420F060A068001DA060012042
:1016100011B0F0BD0120F060A068401DA060012065
:1016200011B0F0BD0220F06001207061A068001DC3
:10163000A060012011B0F0BD21463046FFF762FEE8
:1016400011B0F0BD25682818085C342820D00DDCC6
:1016500005462B3D092D28D22F007F443F79FF19E5
:10166000BF441623161823161616160038280FD056
:1016700008DC35280CD036280AD000E074E0372882
:1016800013D105E0392803D0452801D065280CD1B5
:10169000585400E05A54491C3F2906D2002C04D06B
:1016A000A06867684518BD42CCD30020585410A9E3
:1016B000184601F0CFFC0F4605461099684688424F
:1016C00052D0F761944A954B28463946B561F7F7F1
:1016D00043FB03D8924870610FE019E00022914B60
:1016E00028463946F7F724FB02D80120C00703E05B
:1016F00028463946F7F7C4FA70610820F060109A5E
:10170000A1686846101A0818A060012011B0F0BD49
:101710007D20C000914203D223685B5C5B2B06D026
:10172000914279D22268515C7B2967D074E000270E
:10173000E1683D4681426FD2491CE1602168A068A2
:10174000095C5B2968D1401CA0602046FCF74AF97F
:101750006168A068884203D22268125C5D2A38D092
:10176000884202D3401EA06056E0401EA060204682
:1017700010300090FCF716FA002839D0002F23D043
:10178000286045600546A068401CA0602046FCF724
:1017900029F921462846FFF7EDFE00282AD02046E9
:1017A000FCF720F9002C25D06168A068884203D29C
:1017B0002168095C2C290AD0626890421AD22168FB
:1017C000085C5D2816D104E007463D46DBE700983B
:1017D000D0E7E068401EE060002F00D07D60202050
:1017E000B760F060A068401CA060012011B0F0BD9F
:1017F000002F11D03846FCF76BF90DE00027E168A7
:101800003D46814208D2491CE1606168A068884277
:1018100002D2115C7B2902D0002011B0F0BD401C27
:10182000A0602046FCF7DEF86168A068884203D219
:101830002268125C7D2A4CD0884293D2401EA06060
:10184000204610300090FCF7ADF9002855D0002F4D
:101850004ED0286045600546002CCBD0A06861685A
:10186000401C8842C6D2A0602046FCF7BBF8214647
:101870002846FFF747FD0028BCD02046FCF7B2F809
:1018800028692862002028616168A0688842B1D276
:101890002168095C3A29ADD1401CA0602046FCF7C4
:1018A000A1F821462846FFF765FE0028A2D0204671
:1018B000FCF798F86168A068884203D22168095C47
:1018C0002C2918D06268904294D22168085C7D2847
:1018D00090D1E068401EE060002F00D07D60402085
:1018E000B760F060A068401CA060012011B0F0BD9E
:1018F00007463D46B0E70098A5E7002F8CD079E772
:101900006E756C6C0000000066616C736500000011
:1019100074727565000000000000C0FFFFFFDF412A
:10192000FFFFFF7F0000E0C1102819D230B40D4C3A
:1019300083001B199D6989032D0B2D03090D0D4390
:101940009D619969084D920992052940920A1143B7
:1019500099610122616982401143616130BC704725
:101960007047000000200240FF0FC0FFF3B505469E
:1019700081B00026408800F003F901000AD01C4F16
:101980006A88002014234343DB195B8A934203D106
:1019900042262AE0402628E0401CC0B20A28F1D3A3
:1019A000002E22D1002414206043C019408AFF2851
:1019B00006D0641CE4B20A2CF5D30A2C14D014E02F
:1019C00028460830009014206043C0190E686B78D8
:1019D000AA880746A91DB0470600EED1688878821C
:1019E0000298398A0180E8E74B26304603B0F0BD03
:1019F000784B002002885004400CD20B01D0090221
:101A00000843704710B40024094A214614234B436D
:101A10009B185B8A834204D1142041438818C46810
:101A200003E0491CC9B20A29F0D3204610BC704714
:101A3000784B002030B4FF23040AC5B20A490020C5
:101A4000142242435218128AAA4204D1142250434B
:101A50004018438A03E0401CC0B20A28F0D3200299
:101A600030BC184370470000784B0020084A1178BA
:101A70000A290AD2C9004368891800688B60486047
:101A80001078401C10700120704700207047000043
:101A9000404C002030B4FF23040AC5B20A4900209C
:101AA000142242435218528AAA4204D114225043AB
:101AB0004018038A03E0401CC0B20A28F0D3200279
:101AC00030BC184370470000784B0020F1B582B05D
:101AD0000299294E0020002900D13070002502987B
:101AE000002804D0012834D002283ED10FE0294636
:101AF00014225143214A284609308C182082C0B252
:101B000006F448D1207C214606F42AD12DE028464F
:101B100014214843194900234718B87C00903078B5
:101B20001C4600280DD9E0008019828800998A425D
:101B300002D1806880470346641C3078E4B2A0423A
:101B4000F1D8002B02D0596838468847387C06F413
:101B500045D11422094B6A430021D018FF24C160EB
:101B6000448299504160018141816D1CEDB20A2D82
:101B7000B5D303B0F0BD0000404C0020784B0020EE
:101B800070B50146094DCEB20020297804460029DF
:101B90000BD9E10049198A88B24201D1886880478F
:101BA000641C2978E4B2A142F3D870BD404C0020F7
:101BB000F7B500248AB000940194029403940E4671
:101BC00004940594069407940894FF27013711683C
:101BD000154638468847059601970090AA686968B7
:101BE0002868069000980892079100283CD0694622
:101BF0000A9800F0CDF8002830D00098002806D0D0
:101C000002994018F6F754FB029940180290AA680E
:101C1000002A07D002990098491C904706001DD061
:101C2000009418E002982968401C8847060015D0E7
:101C300002980199401C814201D20A4601E0029AB1
:101C4000521C30460099F6F70FFB0298345469682D
:101C500000988847009430460DB0F0BD00980028E9
:101C600002D069688847009400200DB0F0BD0000E4
:101C7000F8B500240A460546002910D0002D10D0E2
:101C800001460078002826D008780C283BD015DCC7
:101C9000082838D0092836D00A2815D133E000208A
:101CA000F8BD03211046FCF765FB0028F8D022217F
:101CB00001704170002181700120F8BD0D2822D0F3
:101CC000222820D05C281ED0202800D2641D48780D
:101CD000491C0028D8D1481B0719F91C1046FCF7ED
:101CE00049FB061EE9D0002C0FD022203070287846
:101CF000741C002834D0C0B21F2813D9222811D058
:101D00005C2837D10EE0641CE1E7222434703A46A7
:101D10002946701CF6F7A8FAF0194470002181706A
:101D20000120F8BD5C2020702A78641C0C2A23D086
:101D300006DC082A1DD0092A24D00A2A06D11DE073
:101D40000D2A1DD0222A12D05C2A13D00EA12046C3
:101D5000F9F792FD241D6878641C6D1C0028CAD117
:101D60002221F0194170002181700120F8BD22204C
:101D700000E062202070EEE76620FBE76E20F9E7C6
:101D80007220F7E77420F5E77525303478000000FD
:101D9000002801D0002901D100207047F0B5054688
:101DA000007B8BB00C4610287ED008DC012819D0AF
:101DB000022821D0042809D0082876D128E020283C
:101DC00074D0402873D080287DD19BE00521204627
:101DD000FCF7D0FA002803D0DCA1F7F721FC0120A2
:101DE0000BB0F0BD06212046FCF7C4FA0028F7D05E
:101DF000D8A1F7F7CDFB08E005212046FCF7BAFA99
:101E00000028EDD0D5A1F7F70BFC01200BB0F0BDF9
:101E100007910024AF69EE6900942E200194039489
:101E200004940594029406940894314609940A9007
:101E3000002F01D0012000E0002001434800C949E3
:101E40004008081AC00F14D1012170004905C8428A
:101E500001D1002F0DD06869F6F7C8FE3A46334627
:101E6000F6F766FF0BD1C0A168466A69F9F704FD71
:101E700026E0BEA16846F9F7FFFC054621E03A4698
:101E80003346BCA16846F9F7F7FC054608AABBA192
:101E90006846F6F751FA01280CD13A4633460999BB
:101EA0000898FCF74BF803E03EE00CE041E094E0DA
:101EB000002806D13A463346B1A16846F9F7DCFC62
:101EC00005461A2D02D300200BB0F0BD691C0798FF
:101ED000FCF750FA0028F7D0002D0BD92E236A46C4
:101EE000115D0A9EB14201D1035500E00155641C09
:101EF000AC42F5D300210155079880684119079835
:101F0000816082E728690028DED0F6F7D1F9401C0D
:101F1000064601462046FCF72DFA0028D4D032466A
:101F20002969F6F7A1F970E72869FFF7A1FE0BB060
:101F3000F0BDAD6801212046FCF71CFA0028F6D060
:101F40005B210170A068401CA060E068401CE0605C
:101F5000002D34D0002621462846FFF719FF00281F
:101F600013D0002C09D02068002806D0A1684018A2
:101F7000F6F79EF9A1684118A160286800281BD0D7
:101F80006069002804D0022703E030460BB0F0BDA2
:101F90000127791C2046FCF7EDF90028F5D02C210B
:101FA00001706169401C002902D020210170401C91
:101FB0000670A068C019A0602D68002DCBD1022149
:101FC0002046FCF7D7F90028E0D05D210170002100
:101FD0004170E068401EE06017E76069AD68002866
:101FE00001D0022700E00127791C2046FCF7C2F946
:101FF0000028CBD07B210170E168401C491CE160C6
:1020000062690A21002A00D00170A068C019A0608E
:10201000002D78D000276069002814D02046E168A0
:10202000FCF7A8F9002825D0E2680021002A06D98B
:1020300009220270E368401C491C8B42F9D8E16810
:10204000A0684018A0602146286AFFF711FE00280A
:1020500010D0002C09D02068002806D0A1684018B4
:10206000F6F726F9A1684118A1606069002804D03C
:10207000022603E038460BB0F0BD0126314620466B
:10208000FCF778F90028F5D03A2101706169401C0D
:10209000002901D009210170A06821468019A060A3
:1020A0002846FFF775FE0028E4D0002C09D02068F0
:1020B000002806D0A1684018F6F7FAF8A168411880
:1020C000A1606069002800D001202968002900D0A3
:1020D00001214618711C2046FCF74CF90028C9D094
:1020E0002968002902D02C210170401C6169002957
:1020F00002D00A210170401C0770A0688019A060FE
:102100002D68002D87D16069002802D0E168491C44
:1021100000E002212046FCF72DF90028ABD06169D0
:1021200000290BD0E2680021012A07D009220270A1
:10213000E368401C491C5B1E8B42F8D87D2101706E
:1021400000214170E068401EE0605EE66E756C6CD8
:102150000000000066616C736500000074727565B4
:10216000000000000000F07F256400006E756C6CBC
:102170000000000025312E3135670000256C670016
:1021800025312E313767000070B5054600780028EC
:1021900013D00A4E2846F6F78BF884B20D2C00D9DE
:1021A0000D2471782346481C70702A460220FAF7E5
:1021B00077FB2D1928780028ECD170BD4E47002000
:1021C000F8B5069E1F46182E01D9182500E03546A1
:1021D00013460A4601460CA00096F9F73DFB002481
:1021E000002D07D9395D11A0F9F736FB641CA4B2A4
:1021F000AC42F7D3AE4202D90EA0F9F72DFB0FA0E7
:10220000F9F72AFBF8BD00005B424C452025735DC1
:1022100020747970653D30782530325820736571AF
:102220003D2575206C656E3D2575000020253032FA
:1022300058000000202E2E2E000000000D0A000085
:10224000F8B5134E0F46756904463068001D00F05E
:1022500011FF601C07D1002F05D031680D48091D02
:1022600000F095FFF8BD30682C1944603168AC422D
:1022700004D2B068091D00F071FFF8BD7068091D37
:1022800000F06CFF306B8442F7D23463F8BD00007D
:10229000B4470020C45F0020F8B5856B164604469D
:1022A0000027026C002A11D0002E19D0E068F5F743
:1022B000DBFF216CE068401AE0602268904202D2A5
:1022C0006068401AE060022E17D019E020680028EC
:1022D00016D1606801F062FD0746002060600FE0E3
:1022E000A068F5F7C1FF216CA0684018A060616884
:1022F000884205D32068A06002E0002D00D06D1E4A
:102300006D1CA5633846F8BD114D124E124FE8689A
:10231000002817D000F048FFF068C468201D00F0C6
:10232000A9FE2869401E2861E868401EE86000F0A8
:1023300047FF206B00F052FF204600F04FFFE86897
:102340000028E7D138680128E1D900F069FFDEE70D
:10235000B4470020B05F0020E85E002030B412498E
:1023600000E011460A688242FBD34B685C18844245
:1023700003D1406818184860084643681C18944206
:102380000CD10A4C2468A24206D052689A184260C6
:102390000A681268026002E0046000E002608142A4
:1023A00000D0086030BC704700480020F047002093
:1023B000F7B582B0039800260068002859D003982A
:1023C000416802464968083241600092914201D159
:1023D000496841604068C068019003984168496855
:1023E0004160009A914201D149684160CF68242040
:1023F00002997043441804983D46002F01D11E49AC
:102400000D682560294634316160E96A2161296BD4
:10241000E161696CA1600023E96CA3616161052839
:1024200013D015490A68954201D1237311E0207336
:1024300003280ED1886B401C8863A86A002801D04D
:102440000220207301F04CFD03E02846FBF762FFF9
:102450002073286B00210278A52A04D14278401C01
:10246000491CA52AFAD0880820840198761C874246
:10247000B3D1304605B0F0BDB44700200348006832
:10248000401C72B600D0FEE7FEE7000008480020BE
:10249000F8B5054600F088FE2E4640360524345730
:1024A000002C0FDD2F462437686A00280AD03846F2
:1024B00001F0E4FC002801D000F046FF641E64B285
:1024C000002CF1DC0027FF43777100F079FE00F06B
:1024D0006BFE04243457002C10DD28461030009089
:1024E000286900280AD0009801F0C8FC002801D013
:1024F00000F02AFF641E64B2002CF1DC377100F09A
:102500005FFEF8BDF8B50446002500F097FF374E92
:1025100000273068364A002801D0F0681BE005210A
:1025200034480903430705D0C01DC008314BC00023
:10253000C31AC91A41180839C908C9005760106080
:1025400031604F600B1A0F6043600160B36001207F
:10255000C0077360F06004423FD1002C3DD020469C
:102560000830410708D04107490F0823591A0818B5
:10257000410701D072B6FEE700282ED0716888426C
:102580002BD81B49146801E0214614466268824238
:1025900002D22268002AF7D1326894421DD00D6819
:1025A00022680A60616808350A1A102A09D92118B8
:1025B0004B0701D072B6FEE74A6060600846FFF73D
:1025C000CDFE61687068401A7060B268904200D2B7
:1025D000B060F06827600143616001F081FC68072A
:1025E00001D072B6FEE72846F8BD0000F047002093
:1025F00000480020D85F002004490868002803D064
:102600000868026D521C026508687047B4470020D4
:1026100010B40124031F24061C601B1F1960191F1E
:10262000034B0B6014390A6010BC4038704700003F
:102630007D24010170B5064614460D464720FFF77C
:10264000E1F90369002B0DD01879B04207D1587910
:102650002880981D2060002B04D0002070BD1B68CE
:10266000002BF1D10020288020600A2070BD0000DE
:1026700070B516460C46104605F41CD3002813D13D
:102680004720FFF7BFF9054606233246194607489B
:1026900005F452D2A988628889180180A1884180F6
:1026A000A179017105F484D2002070BD180C0000DE
:1026B000F7B506460D464720FFF7A4F9046907461B
:1026C000002C14D02079B0420BD16079A8420CD0F4
:1026D000384621461030F6F77FFF204605F41CD11E
:1026E00005E02468002CEDD101E0002C0AD1284639
:1026F0000121083005F49AD10446014638461030CD
:10270000F6F770FF267165712A46A01D0299F5F74C
:10271000ABFD002003B0F0BDF8B5C5680124287FEB
:102720000F4601281ADD0E4E20461622504302465F
:10273000296A10328A5A5204920F0BD10A5C401C4B
:10274000085C00021018B04204D1E1B20022384601
:1027500000F03EF9287F641CA042E5DCF8BD0000D3
:1027600002290000F8B5C5680124287F0F4601281A
:102770001ADD0E4E2046162250430246296A1032B8
:102780008A5A5204920F0BD10A5C401C085C00026A
:102790001018B04204D1E1B20022384600F018F916
:1027A000287F641CA042E5DCF8BD0000022900007F
:1027B00070B5C46805462069002803D000200028B1
:1027C00002D00EE00120FAE7264610363046F6F732
:1027D000F1FE05F4A1D02069002808D000210029CD
:1027E000F4D00020E860204605F496D070BD0121A9
:1027F000F5E710B504464720FFF704F98279002178
:10280000A24202D98088001981B2084610BD70B575
:1028100004460D464720FFF7F5F8014680888022E0
:10282000A04206D889794118A14202D9201A2870FD
:102830000022104670BDFFB585B00E9D0646297872
:1028400001208840401E049018460E210840328A1C
:1028500069681F4640300192002303900093029163
:102860002B7804AAA9680698F6F7E0FE00900028E5
:102870002AD10121282005F4D9D00446AA68696824
:10288000286862622162E061F46006980188A18094
:10289000217FA171F80701D00120C00307990843E7
:1028A0002080308A608047207082304600F0AAF88D
:1028B00020461030F6F78AFE217F206A00F008F8E3
:1028C000308A002105F408D2009809B0F0BD00005C
:1028D000F3B583B00020019004980125012845DD5F
:1028E0001621039A69438818028A5204920F39D13B
:1028F000039A4078515C000209181D48814231D189
:1029000001A80290EFB204264720FFF77BF8009061
:102910000469002C14D02079B8420BD16079B04200
:102920000CD0009821461030F6F756FE204604F4ED
:10293000F3D705E02468002CEDD101E0002C0AD18A
:1029400030460121083005F471D004460146009854
:102950001030F6F747FE277166713246A01D0299C6
:10296000F5F782FC04986D1C8542B9DB05B0F0BD1B
:1029700002290000004870479045010170B50646E5
:1029800010480D46007800281AD04720FFF782F83B
:10299000A91D8BB2014603220B4805F4CDD0044695
:1029A0000A482A46807820700120607005206080E7
:1029B000A5803146A01DF5F757FC204605F4F8D058
:1029C00070BD00003747002006470000C04D0020C2
:1029D00070B584B00E461446054601AA69463046D5
:1029E000FFF728FE6846028802A80199F5F73CFC2B
:1029F00002A844550246684601883046FFF758FE53
:102A000004B070BD10B504464720FEF7FBFF044933
:102A1000216009216181183060600120208110BD92
:102A2000A0450101FFB583B00C464720FEF7EAFF41
:102A30000546808861882678401887B2059805F495
:102A400039D1012807D03846FCF7C2FD6946FFF7A7
:102A5000DEFE002802D0022007B0F0BD012105985B
:102A600005F43AD10C3C0020AC602873684600782D
:102A7000687301AA02A9FFF7DDFDA8680199044661
:102A8000895D0C34890720D5A188C28808318BB2B2
:102A90003102C1200001891D05F44ED006461320E5
:102AA0003070A88861884018B080A088F0803046D7
:102AB000A288A11D0830F5F7D7FB304605F478D081
:102AC0000121059805F408D101E004F425D701207F
:102AD00007B0F0BD10B5FAF7DFFC002010BDFFB560
:102AE00083B00C464720FEF78DFF0546808861883D
:102AF0002678401887B2059805F4DCD0012807D065
:102B00003846FCF765FD6946FFF781FE002802D0D4
:102B1000022007B0F0BD0C3CAC602E736846007814
:102B2000687301AA02A9FFF785FDA8680199044608
:102B3000895D0C34890720D0A188C28808318BB206
:102B40003102C1200001891D04F4F6D70646122087
:102B50003070A88861884018B080A088F080304626
:102B6000A288A11D0830F5F77FFB304605F420D080
:102B70000121059805F4B0D001E004F4CDD6012080
:102B800007B0F0BD10B50C464720FEF73BFF80882C
:102B90006188A31D401880B2A1880022FAF712FCB8
:102BA000002010BDF8B5488800900C468E88F9F7D3
:102BB0008BFD00281DD0182E01D9182700E03746BC
:102BC000324626A00099F8F747FE0025002F08D9C5
:102BD000601981792AA0F8F73FFE6D1CADB2BD42A5
:102BE000F6D3BE4202D928A0F8F736FE28A0F8F79F
:102BF00033FE0098022821D0062804D0082822D0CD
:102C00000C2829D124E0022E26D1E0882149012870
:102C100002D0002808D01FE001200870F9F754FD09
:102C2000002819D01CA006E000200870F9F74CFD20
:102C3000002811D01EA0F8F70FFE0DE0A188A01DFE
:102C4000F9F75EFD08E0A188A01DF9F79DFC03E0FF
:102C5000A188A01DFAF772F90020F8BD5B424C452F
:102C60005D20777269746520696E643A20617474BE
:102C70005F6964783D2575206C656E3D25750000A3
:102C80002025303258000000202E2E2E000000009B
:102C90000D0A0000374700205B424C455D206E6FF7
:102CA0007469667920656E61626C65640D0A000066
:102CB0005B424C455D206E6F746966792064697370
:102CC00061626C65640D0A00FFB581B0002768463B
:102CD000078048881C460D46082825D00C2828D097
:102CE0000A282AD005206946088016A6684600886A
:102CF0002146083083B21548039A04F41DD7877122
:102D000029780446017068460288A280698861803B
:102D1000002A03D03146E01DF5F7A6FA204604F458
:102D200047D7002005B0F0BD6846F9F7A3FC06467A
:102D3000DCE76846FAF762F802E06846F9F7C2FF96
:102D40000646D3E74E53494E4700000005470000B2
:102D500070B516460C46104604F4ACD7012818D1BD
:102D6000A1791A48002916D0217806230902324693
:102D7000891D04F4E1D60546A078FFF73AFD2880C6
:102D800080202871284604F413D70021304604F42B
:102D9000A3D7002070BDA1883246891D8BB221784F
:102DA0000902891D04F4C8D60546A078FFF721FD65
:102DB000288000202871A0886880A288E11D681DF5
:102DC000F5F752FA284604F4F3D6DEE7140C0000B7
:102DD000F3B583B005001AD02868019028468038E2
:102DE0000290C76F04983E1F864200D906462846C7
:102DF000F8F788FD04460091324629460498FCF70E
:102E0000CDFD0199002806D0016005B0F0BD049801
:102E1000F8F7AAFDF9E729600299002CCF670AD0DC
:102E200021686218291F8A4202D9291B091F2160C3
:102E300000996160E9E7024A00991160E5E7000046
:102E40001048002010B5012400206407206004F41D
:102E5000C9D52E4802882E480168002004F44ED6B9
:102E60002C4802882C480168012004F447D62B48DE
:102E7000008882B22A480168022004F43FD629481B
:102E8000008882B228480168032004F437D6274816
:102E9000416AF02211434162254817F421D62648A1
:102EA0002449016025494161254981602549C16066
:102EB000254981612549C161264925488863FCF778
:102EC000C7FD2068C0B2F6F7B7FB2348007800289A
:102ED00006D0002018F44AD101460020F6F7B2FBD4
:102EE0002068C0B2F6F7B4FBF6F7B8FB2068C0B2B2
:102EF00017F4C8D62068C0B217F4D2D62068C0B282
:102F000018F490D00120206010BD00001C010020AA
:102F1000180100202401002020010020340100209D
:102F2000300100202C010020280100204025024013
:102F300074020020500250008080024000080F0000
:102F400058086A00420500000F0505060F000F0330
:102F50004000D0004080024062000020F0B5314CBB
:102F600083B0E06980075AD502202062A56B082053
:102F700018F4A0D1012018F4ABD12B49002708691F
:102F800040194608B219801A086128480068F5F708
:102F900041FE0022264BF5F793FD019100903E2162
:102FA0002846F6F761FB80197941F5F741FE019B50
:102FB000009AF5F71DFDF5F787FE05461D4A00232B
:102FC000F5F70AF906461B49F6F74EFB1A49281A87
:102FD000081A81B222041948324342600160206B12
:102FE0000821884308432063A06907210907884313
:102FF000A061A169012081430143A1612062FCF726
:1030000027FD0F48104A0078410041180D48081864
:103010004178D1610D498078C8600D48077003B0D0
:10302000F0BD000000800240A802002090000020B7
:1030300000408F407102000070020000408002409A
:1030400010400020B044010140250240802502408C
:103050008000002000B50A4683B000210091019154
:1030600001466846F5F7CFFF0199009803B000BD0F
:10307000704770474368826801699A608368426854
:103080005A604A68824201D182684A600022026125
:103090000868401E08600868704700000148006921
:1030A00070470000B4470020F8B51746204A06468E
:1030B0000024906B0725401C90631069814232D335
:1030C00014206D1E1B496843411824206043801959
:1030D0000122FFF76DF90419002DF1D12420144DC0
:1030E0006043801902226968FFF762F904192420FD
:1030F000604380190222A968FFF75AF904192420B5
:103100006043801904220C49FFF752F90419242066
:103110006043801903220949FFF74AF90419002F77
:1031200001D00020386000F0DBFE2046F8BD000032
:10313000B4470020E85E0020B05F0020C45F00209C
:103140000146083100224160D243C16082600161C2
:1031500000210160704700210161704730B40C68A4
:10316000621C02D00246083202E0026904E01A46FC
:1031700053681D68A542FAD953684B6099608A600C
:10318000516008610168491C016030BC70474268A9
:103190004A6093688B609368596091600861016828
:1031A000491C01607047000072B604480168491C60
:1031B0000160BFF34F8FBFF36F8F70470848002047
:1031C00005490868002804D0401E086000D162B696
:1031D000704772B6FEE700000848002000281CD0A7
:1031E00070B504460D4D083C6068E968084201D19D
:1031F00072B6FEE72268002A01D072B6FEE7884365
:10320000606000F01BF960686968401868602046DB
:10321000FFF7A4F800F064FE70BD7047F04700208F
:103220000120044900074860BFF34F8FBFF36F8F41
:103230007047000000ED00E010B500280FD00949EC
:103240008A6B002A01D072B6FEE78A6B521C8A6331
:103250000021FEF7F5FF00F043FE002801D1FFF743
:10326000DFFF10BDB447002002498A6A0260496945
:1032700041607047B4470020F0B585B0002705468F
:1032800007702C4801690291006924214843FFF727
:1032900039F906004CD000220299FFF705FF039789
:1032A0000290002841D90398242148438019017BCA
:1032B000052911D20A007A4412799218974402041F
:1032C00006080A00582408E0522406E0422404E0DC
:1032D000532402E0442400E0002441682846F5F726
:1032E00013F82846F4F7E4FF0F2804D220212954CC
:1032F000401C0F28FBD32F542D180398242148433A
:103300008019018C826801920091036922460AA10A
:103310002846F8F7B1FA2846F4F7CAFF451903988A
:103320000299401C03908842BDD33046FFF756FFF8
:1033300005B0F0BDB44700200925630925750925AE
:10334000750925750D0A0000014901204862704782
:10335000B447002010B50C46002809D0054909687B
:103360001831FFF7FBFE01212046FEF769FF10BD73
:1033700072B6FEE7B447002070B50B4604002FD0AC
:10338000226D002A0ED0E16C994200D21946E06A03
:10339000884225D0012A23D1124D2A68944203D1B4
:1033A00072B6FEE772B6FEE7E162A269002A02DBAE
:1033B0000722511AA16114220B4E504361698019F2
:1033C00081420DD1201DFFF755FEE06AA9698842B0
:1033D00000D9A861142148438019211DFFF7D7FEA9
:1033E00070BD0000B4470020E85E002010B582B038
:1033F0000D4800240190234680220CA100940D4822
:1034000000F090FB012803D0401C0BD172B6FEE700
:1034100072B600210848C94301630121C1614461BA
:1034200000F052F802B010BDE847002049444C4576
:103430000000000009230101B44700200248816B0D
:10344000491C816370470000B4470020164B986BFD
:10345000002802D001205862704700205862986905
:10346000142102464A4311498A58002A0AD10028E9
:1034700006D01422401E42438A58002AF7D001E0A9
:1034800072B6FEE7142210B4424351184A680C4643
:10349000526808344A60A24201D152684A60D16839
:1034A0001960986110BC7047B4470020E85E0020A6
:1034B0000148406870470000F047002001488068DC
:1034C00070470000F047002070B50F48016AFF22E6
:1034D000120411430162016A1202114301620B4C92
:1034E00000252561A5610A487D21C9000068F4F71F
:1034F00049FE401E60610720206106480560F4F720
:10350000F7FD002070BD000000ED00E000E000E0ED
:10351000004000200848002010B50246002101208C
:1035200000F00CF8041E07D00021416001600B463A
:103530000A46C16000F05BF8204610BDF8B517469A
:103540000E46050016D0002E16D070435030FEF700
:10355000D9FF04000CD020465030002E0ED0206041
:10356000266420460121E56300F00AF84C20075547
:103570002046F8BD72B6FEE70020E7E72460EFE7DB
:1035800070B50D46040026D0FFF70EFE216CE06BEF
:1035900048432168411861600021A1632168A1604E
:1035A000E06B216C401E48432168224641180020F0
:1035B000C0434032E1601071507120461030002D40
:1035C0000BD0FFF7BDFD20462430FFF7B9FDFFF714
:1035D000F7FD012070BD72B6FEE721690029F6D023
:1035E00000F04CFC0028F2D0FFF71AFEEFE7FFB521
:1035F000002783B00446002803D00498002802D096
:1036000006E072B6FEE7206C002801D072B6FEE735
:103610000698022804D1E06B012801D072B6FEE7BB
:1036200000F03CFB002804D10598002801D072B6B8
:10363000FEE720462546103040350290FFF7B4FDE6
:10364000A06BE16B884208D30698022805D0059844
:1036500000284AD0002F4BD04EE0069E0499A56B5F
:103660000027226C002A11D0002E19D0E068F4F750
:10367000FBFDE168206C091AE1602268914202D2E8
:103680006168081AE060022E17D019E0206800284F
:1036900016D1606800F082FB0746002060600FE0F2
:1036A000A068F4F7E1FD216CA0684018A060616893
:1036B000884205D32068A06002E0002D00D06D1E76
:1036C0006D1CA563606A002806D02046243000F0F7
:1036D000D5FB002802D103E0002F01D0FFF7A0FDA9
:1036E000FFF76EFD012007B0F0BDFFF769FD20E098
:1036F0006846FFF7B9FD0127FFF762FDFFF79EFE61
:10370000FFF752FD04202856401C00D128710520E7
:103710002856401C00D16871FFF752FD05A9684684
:1037200000F0CEF9002807D02046FEF7B1FE00F0E9
:10373000D7FB002007B0F0BDFFF736FDA06BE16BB3
:10374000884201D1012600E00026FFF739FD002E56
:103750000ED005990298FFF7FDFD2046FEF798FE72
:1037600000F0BEFB002800D068E7FFF759FD65E7D1
:103770002046FEF78DFE00F0B3FB5FE7FFB583B098
:103780001E461746040003D00498002802D006E025
:1037900072B6FEE7206C002801D072B6FEE7022E5A
:1037A00004D1E06B012801D072B6FEE7F4F7B4FC57
:1037B0000190A06BE16B884208D3022E06D0002452
:1037C0000198F4F7ADFC204607B0F0BD204640302C
:1037D000052500904557324620460499FEF75CFDCA
:1037E000681C04D000986D1C45710124E8E7606AEC
:1037F0000028FAD02046243000F040FB0028F4D006
:10380000002FF2D001203860EFE7F7B5002784B031
:103810000446002803D00598002802D006E072B6BE
:10382000FEE7206C002801D072B6FEE700F036FA01
:10383000002804D10698002801D072B6FEE7204681
:103840002546243040350290FFF7AEFCA66B002ED3
:1038500021D0226C059B002A0BD0E0688018E06024
:103860006168884201D32068E06001461846F4F799
:10387000FBFC761EA6632069002807D02046103086
:1038800000F0FCFA002801D0FFF7CAFCFFF798FC13
:10389000012007B0F0BD0698002802D0002F05D007
:1038A00008E0FFF78DFC002007B0F0BD6846FFF789
:1038B000DBFC0127FFF784FCFFF7C0FDFFF774FC7A
:1038C00004202856401C00D1287105202856401C91
:1038D00000D16871FFF774FC06A9684600F0F0F8A3
:1038E000002811D02046FEF7D3FD00F0F9FAFFF7CB
:1038F0005BFCA06B002827D00026FFF761FC002EA0
:10390000A2D0002007B0F0BDFFF74EFCA06B00284E
:1039100012D00026FFF754FC002E0FD00699029813
:10392000FFF718FD2046FEF7B3FD00F0D9FA002896
:103930008AD1FFF775FC87E70126EBE72046FEF703
:10394000A7FD00F0CDFA7FE70126D6E7F3B5002703
:1039500085B004460097002804D0206C002803D0CE
:1039600072B6FEE772B6FEE700F098F9002804D1BF
:103970000698002801D072B6FEE72046254624307E
:1039800040350190FFF710FCA06B002817D0401EB7
:10399000A0632068002802D1FEF72EFE6060206937
:1039A000002807D02046103000F068FA002801D027
:1039B000FFF736FCFFF704FC012007B0F0BD0698C6
:1039C000002802D0002F0AD00DE00098002801D076
:1039D00072B6FEE7FFF7F4FB002007B0F0BD02A8C7
:1039E000FFF742FC0127FFF7EBFBFFF727FDFFF78F
:1039F000DBFB04202856401C00D1287105202856E6
:103A0000401C00D16871FFF7DBFB06A902A800F09B
:103A100057F800281BD02046FEF73AFD00F060FA68
:103A2000FFF7C2FBA06B00283ED00026FFF7C8FBC3
:103A3000002EA7D0009800283ED0FFF7B5FB606AA3
:103A4000002833D0206B07210068091A2FE0FFF708
:103A5000ABFBA06B002808D00026FFF7B1FB002EBF
:103A60001CD02068002802D009E00126F5E7FFF706
:103A70009BFB606800F0C6F90090FFF7A1FB069978
:103A80000198FFF767FC2046FEF702FD00F028FAD8
:103A9000002800D076E7FFF7C3FB73E72046FEF768
:103AA000F7FC00F01DFA6DE70126BFE70021606812
:103AB000FFF762FCFFF784FB002007B0F0BD0000B9
:103AC000F8B50D46040012D0002D12D0FFF76CFBA4
:103AD000134E726963682868D11A471C0BD0276897
:103AE000B66AB74209D0934207D8012413E072B6F0
:103AF000FEE772B6FEE700240DE0884208D9401ABE
:103B000028600748816A216040696060002402E003
:103B1000002001242860FFF753FB2046F8BD000079
:103B2000B4470020FFB585B090000F9F0E9D029016
:103B3000FEF7E8FC06001ED05C20FEF7E3FC040064
:103B400016D0266305990191089900913046029993
:103B5000069EA5220391F4F799FB0399206B091F98
:103B60004018C008C0000290400708D072B6FEE7B7
:103B70003046FFF733FB0020C04309B0F0BD2118E9
:103B8000325C20310A75315C002902D0401C1028BB
:103B9000F5D3264600204036F070072D00D30625C9
:103BA000E5620020E5642065201DFFF7D4FA204679
:103BB0001830FFF7D0FA24610720411B6462A1612D
:103BC000002161653176009A01990298FEF720FD87
:103BD0002060002F00D03C602546FFF7E5FA284E14
:103BE0003069401C30613068264F002803D0F069EE
:103BF000002821D026E035603069012822D1002438
:103C000014206043C019FFF79BFA641C072CF7D3FC
:103C10001D48FFF795FA1D48FFF792FA1C48FFF779
:103C20008FFA1C48FFF78CFA1B48FFF789FA1648F1
:103C300070601430B06005E03068E96AC06A88429C
:103C400000D83560F06A401CF0626864E86AB169C7
:103C5000884200D9B06114214843C019291DFFF7DB
:103C600096FAFFF7ADFAF069002806D03068E96AE5
:103C7000C06A884201D2FFF7D3FA012009B0F0BD33
:103C8000B4470020E85E0020745F0020885F0020B9
:103C90009C5F0020B05F0020C45F00200648C1691F
:103CA000002904D0806B002803D000207047012039
:103CB0007047022070470000B44700200148406967
:103CC00070470000B4470020F8B5324F0026B86BAB
:103CD000002808D0386A401C3862786A002800D072
:103CE00001263046F8BD7D696D1C7D6115D178686F
:103CF0000068002801D072B6FEE77868B96879607C
:103D0000B860B86A401CB86278680068002813D0B0
:103D10007868C068C06840683863386B854211D3E2
:103D20007868006800280AD07868C068C46860684D
:103D3000854211D2386305E00020C043ECE7002043
:103D4000C043386338681421C06A48431249085890
:103D50000128C2D90126C0E7201DFFF78BF9A06A10
:103D6000002803D020461830FFF784F9E06AB969CB
:103D7000884200D9B8611421484307494018211DE1
:103D8000FFF705FAE06A3968C96A8842C8D3012694
:103D9000C6E70000B4470020E85E002070B50021AF
:103DA0000446002828D0154D2868844201D072B6F8
:103DB000FEE7206D002808D0401E2065E36CE26A13
:103DC0009A4219D0002802D016E072B6FEE7201DF4
:103DD000FFF750F9E06C0721E062081AA061E06A81
:103DE000A969884200D9A8611421484304494018B0
:103DF000211DFFF7CCF90121084670BDB447002012
:103E0000E85E002070B504460020002C2AD0194D31
:103E1000E16A2A68D26A914225D2A069002804DBAF
:103E200028680721C06A081AA061E06A1422124EAD
:103E3000504361698019814210D1201DFFF71AF9A2
:103E40002868C06AE062A969884200D9A861142183
:103E500048438019211DFFF79AF902E02868C06ADB
:103E6000E062012070BDE16C2A68D26A9142F8D309
:103E700070BD0000B4470020E85E002070B5C06847
:103E8000C468002C0BD0204618300646FFF7F2F825
:103E9000104DA86B002804D031460F480EE072B6D2
:103EA000FEE7201DFFF7E6F8E06AA969884200D91D
:103EB000A8611421484309494018211DFFF767F9FB
:103EC000E06A2968C96A884202D90120686270BD27
:103ED000002070BDB44700209C5F0020E85E0020F9
:103EE000F8B52E4D0027A86B002808D0FFF75CF925
:103EF000A86B401EA863A86B002802D046E072B6EB
:103F0000FEE72869002841D0254E306800282AD0D5
:103F1000F068C46820461830FFF7ACF8201DFFF7A2
:103F2000A9F8E06AA969884200D9A8611421484328
:103F30001C494018211DFFF72AF9E06A2968C96A5F
:103F4000884201D30120686230680028E0D1002C4B
:103F500009D068682946006800281BD04868C068F6
:103F6000C068406808632C6A002C09D00126FFF75E
:103F7000ABFE002800D06E62641EF8D100202862DB
:103F8000686A002802D00127FFF74AF9FFF718F9FD
:103F90003846F8BD0020C043E4E70000B4470020E5
:103FA0009C5F0020E85E002040BA7047C0BA7047AE
:103FB0000138FDD170470000F7B50325AD06286A2A
:103FC00082B016460C46400840002862286A02214A
:103FD00008432862286A8007FCD4662068600127AD
:103FE0002F61A86AC005FCD5992068602F61A86A76
:103FF000C005FCD5FF209130FFF7DAFFFF23013326
:10400000AB626846EF60352169602F61A96AC90516
:10401000FCD5AB62A969EF60C9B205226A602F6165
:10402000AA6AD205FCD5AB62AA690902D2B21143D1
:104030000180C80702D0032005B0F0BDAB626869FB
:10404000FF210831884368616869C91E08436861B7
:1040500002980002483068600820A860EE602F6176
:10406000A86AC005FCD5FF200130A8620023F61C19
:10407000B0080ED0B2081148006899006054060AD2
:1040800009194E70060C000E8E705B1CC8709A42A7
:10409000F1D8FF200130A8626869FF210831884308
:1040A0006861686938436861286A8008800028620E
:1040B000286A38432862002005B0F0BD8000000C5B
:1040C000032080064169FF22083291434161426921
:1040D00001210A434261026A920892000262026A66
:1040E0000A43026270470000002003218906096A22
:1040F000490849000322920611621146096A022208
:10410000114303229206116200BF03218906096A46
:10411000022211400229F8D0D101032292069162B5
:104120000321D1609F2151600121116100BF032152
:104130008906896AFF22013211409142F7D1032298
:1041400092069162114688694969FF2208329143BB
:10415000032292065161114649690122114303224B
:10416000920651611146096A890889001162114657
:10417000096A01221143032292061162704700006E
:104180000000010200000000010203040138FDD11B
:1041900070470000F0B40324A406236A5B085B00A8
:1041A0002362236A02252B432362236A9B07FCD4E4
:1041B000FF230133A3626569DE1DB543656165694F
:1041C0001E1D3543656100026B3060600820A060F1
:1041D000E26001262661A06AC005FCD5A362002327
:1041E000D21C90080ED095080F4800689A00885499
:1041F000070A52185770070C000E97705B1CD0709E
:104200009D42F1D86069FF2108318843606160698F
:1042100030436061206A800880002062206A304359
:104220002062F0BC002070478000000CF8B5064604
:1042300001200025C004864201D90520F8BD0324D1
:10424000A406206A400840002062206A0221084338
:104250002062206A8007FCD4FF270137A76200F0A4
:10426000BBF8002801D0032515E00620606001217D
:104270002161A06AC005FCD5A762300220306060D1
:104280002161A06AC005FCD5A7620C4800F0C8F8FF
:10429000002800D102256069FF2108318843606150
:1042A0006069012108436061206A80088000206203
:1042B000206A084320622846F8BD0000E696010007
:1042C000F7B506460120C00482B01546864202D9E1
:1042D000052005B0F0BD03208006016A49084900A9
:1042E0000162016A022211430162016A8907FCD45A
:1042F000FF2101318162F2B28C1AA54200D8ACB222
:104300000398009000F068F8002840D10621480684
:10431000416001210161816AC905FCD5FF2101319C
:104320000320800681624169FF2208329143416186
:104330004169042211434161310232314160C4605C
:104340000022002C16D9009887183B78F878194677
:104350007B7800061B021943BB781B0419430143F9
:104360000802F978000A0906084319490860121D75
:10437000A242E8D30121032080060161816AC905B8
:10438000FCD5FF2101318162124800F049F8A542B5
:1043900009D00398361900192D1BFF24013403900E
:1043A000A542ADD8ABE7032080064169FF22083261
:1043B000914341614169012211434161016A8908C8
:1043C00089000162016A11430162002005B0F0BD5D
:1043D0008000000C1A06000038B401250320800676
:1043E0006A46C560352141600561816AC905FCD511
:1043F000FF24013484628169C560CBB2052141602C
:104400000561816AC905FCD5846280691902C0B260
:10441000014388B21180C00700D0012038BC70472A
:10442000F8B400210125032292066B46D56035249D
:1044300054601561946AE405FCD5FF270137976243
:104440009469D560E4B2052656601561966AF60552
:10445000FCD5976296692402F6B234431C80E307C8
:1044600022D0814202D9F8BC002070470322920674
:104470006B46D560352454601561491C946AE40587
:10448000FCD597629469D560E4B205265660156143
:10449000966AF605FCD5976292692402D2B214435B
:1044A000A2B21C80D207DCD1F8BC0120704700000A
:1044B00000171300171000170E001709001704004B
:1044C000170000171801171401171501171900001C
:1044D0000028000200000000032800020000000085
:1044E000292A00020080800003280002000000004A
:1044F000242A00020080800003280002000000003F
:10450000252A00020080800003280002000000002D
:10451000272A00020080800003280002000000001B
:10452000262A00020080800003280002000000000C
:10453000282A0002008080000328000200000000FA
:10454000232A000200800800032800020000000067
:104550002A2A000200800800032800020000000050
:10456000502A00020080070039E00001C7DF000187
:10457000C5DF0001C3DF000100140000E1E000011D
:10458000130C00001DF30001031400009DE1000165
:1045900037280101B1270101652701011927010110
:1045A000130C0000E1F30001150C0000C1F4000140
:1045B000170C0000F9F10001000C000039F20001B5
:1045C00006470000DF2A010103470000852B010197
:1045D00008470000252A01010E470000712601014D
:1045E00005470000512D0101FFFF000011D200011D
:1045F000130E000039E50001150E000049E400012A
:10460000170E0000B9E90001190E000091E9000140
:10461000E845010105000000F7B586B000200290D2
:104620005C48154604695C480E46824201D905463D
:1046300002E0002D00D10125002C08D0A1880698A9
:10464000814204D1E088B04201D101200290534858
:10465000039084460698010431430020002C1CD0AE
:104660000A0CA7888BB2974207D1E7889F4204D1F2
:10467000002807D02168016007E020462468002C4C
:10468000EFD10AE0614622680A602168002902D061
:104690000020206001E061464860002C07D1022123
:1046A000102000F095F8069981800446C680280104
:1046B000052100F077F807467D200E464643EFF3CC
:1046C0001085012080F31088684600F087F885F394
:1046D000108800980490C0190501019927202D0920
:1046E0008E1900010591864203D96D1C2D012D09FB
:1046F000361AE660A5600398294F86460020844656
:1047000070460068002813D0A268E1680091C36871
:1047100081680193531A1B011B09BB420AD29142C3
:1047200003D1019A0099914204D984460068E9E7CF
:104730007246546020606046002801D0046001E0A9
:1047400071460C60134802990069002901D1A0420A
:1047500003D1C168806800F047F8EFF310840120AE
:1047600080F3108802A800F039F884F310880399C8
:1047700002980191291A090109090090B94204D24D
:10478000A84205D10198864202D8032000F032F8F1
:1047900009B0F0BDC8010020FFFF7F02D801002052
:1047A000FFFFFF0730B50B46014600202022012401
:1047B00009E00D46D5409D4205D31D469540491B55
:1047C0002546954040191546521E002DF1DC30BD9E
:1047D00003B40148019001BD2D7A010003B40148E2
:1047E000019001BD5DB6020003B40148019001BD16
:1047F0009DB6020003B40148019001BDAD780100EF
:1048000030B4C36882688868084D141A2401C968E6
:104810002409AC4203D2904204D18B4202D830BC6E
:104820000120704730BC002070470000FFFFFF07E9
:104830000A0C838889B2934204D1C088884201D18E
:10484000012070470020704770B4054600680022C0
:10485000002810D00B0C86888CB29E4207D1C688E7
:10486000A64204D10168002A07D0116006E0024682
:1048700000680028EFD170BC7047296001680029EA
:1048800003D00021016070BC70476A6070BC704743
:10489000F0B5104F026886460025002A10D0C8687F
:1048A0008C6893688446E01A00010009D668B84213
:1048B00008D2A34201D1B44504D915461268ECE7E9
:1048C000704641600A60002D01D02960F0BD70463D
:1048D0000160F0BDFFFFFF0770B584B004460E46CF
:1048E000EFF31085012080F3108802A8FFF776FF10
:1048F00085F3108802980399024600900191A01A4E
:10490000000107490009884204D2A24205D101985A
:10491000864202D8012004B070BD002004B070BDF2
:10492000FFFFFF0730B583B00446EFF31085012089
:1049300080F310886846FFF751FF85F310880199CE
:1049400000986160206003B030BD000000280002C4
:10495000000000000328000200000000002A000AF6
:10496000008020000328000200000000012A00024D
:10497000008002000328000200000000042A000258
:10498000008008000328000200000000A62A0002A0
:10499000008001000328000200000000C92A000274
:1049A000008001000028000200000000032800022F
:1049B00000000000052A0020008004000229000AEF
:1049C000000002000328000200000000292B000A5A
:1049D0000080100003280002000000002A2B0002C3
:1049E00000801000FFFF0000EDCA0001A40D0000D0
:1049F0005DEC0001A50D000091EC00011A0D000016
:104A0000A9F10001150D0000F1EC0001000D0000FE
:104A10001DED00011C0D0000DFF10001A70D0000DD
:104A2000FDF00001A80D0000EBF10001020C0000F8
:104A3000D1F20001000C0000A9F20001010E0000FB
:104A4000D5E700010F0E000091EB0001110E0000F0
:104A5000F5EB00012C0E000075EB0001030E0000C9
:104A60002DE900010A0E0000E9EA0001300E000005
:104A700069EB00010C0E00001DEC0001000E0000AF
:104A800041E70001090E000069E70001010F000085
:104A90002DCD0001020F0000B5C90001030F000079
:104AA00011CD0001040F0000F90A0101E4490101E0
:104AB00036470020010019000214000019E200012D
:104AC000B84A010101000000004C01010300000090
:104AD00001102EC78A0E7390E111C20860270000F2
:104AE000002800000000000000000000000000009E
:104AF0000002000000000328000000000000000089
:104B0000000000000000000A0000000001002EC7A5
:104B10008A0E7390E111C20860270000000400C0F3
:104B20000002012900000000000000000000000059
:104B30000000000A008014000328000000000000AC
:104B40000000000000000000000A00000000020059
:104B50002EC78A0E7390E111C20860270000001072
:104B600000C0000202290000000000000000000058
:104B700000000000000A008014000328000000006C
:104B800000000000000000000000000A000000001B
:104B900003002EC78A0E7390E111C208602700003F
:104BA000000A00C00002032800000000000000000E
:104BB000000000000000000A0000000004002EC7F2
:104BC0008A0E7390E111C20860270000000200C045
:104BD00000020328000000000000000000000000A8
:104BE0000000000A0000000005002EC78A0E739026
:104BF000E111C20860270000000A00C000020000A6
:104C000004470000C92C01010A470000A52B01013F
:104C100007470000D52A0101585001012450010125
:104C20005DAA000100500101E84F010121AE000121
:104C300008500101084F010149AC00011C5001015D
:104C4000444E010135A80001B44F0101AC4E0101F1
:104C5000BDA70001784F0101444F010131AB0001B4
:104C600090500101804E0101A19E0001A050010160
:104C700030510101699F000160500101BC4F0101E9
:104C8000499B0001A8500101D44D01017D9B000109
:104C900020510101B05001015D980001744F0101E4
:104CA0000C4E010101AC000198500101E84E0101D8
:104CB00015AC000128510101E8500101CDA9000106
:104CC000185101017C4F0101DDAD000110500101BF
:104CD0006850010131AD000101020304050607001F
:104CE00040404040404040404041414141414040BF
:104CF00040404040404040404040404040404040B4
:104D00000502020202020202020202020202020280
:104D10002020202020202020202002020202020247
:104D20000290909090909010101010101010101091
:104D300010101010101010101010100202020202B9
:104D400002888888888888080808080808080808E9
:104D500008080808080808080808080202020240B3
:104D6000E04C01015B6F74615D2062696E61727974
:104D7000206D6F6465204F4E202D2073656E64207A
:104D800030784341204F5441206672616D65732035
:104D90006E6F770D0A28626C655F70726F746F6357
:104DA0006F6C2E6D642073656374696F6E20362E90
:104DB000363B204F54415F41424F5254206F722086
:104DC00033732069646C65206578697473290D0AF2
:104DD000000000006273736574203C6669656C6452
:104DE0003E203C76616C3E3A2077726974652062A1
:104DF0006F6F7473657474696E67206669656C643F
:104E000020286361726566756C2129006F74613AB0
:104E1000205541525420656E74657273204F544181
:104E20002062696E617279206672616D65206D6FB6
:104E3000646520287365652068656C70206F7461F7
:104E40002900000073686F772064657669636520C8
:104E5000696E666F202874656D702F7664642F66A6
:104E6000616E2C2073616D6520617320424C45207A
:104E7000494E464F5F515545525920616C6C29008F
:104E8000617070676574205B6A736F6E5D3A207342
:104E9000686F772061707020706172616D73202877
:104EA0006C65642F70776D2900000000626C656C82
:104EB0006F67205B6F6E7C6F66665D3A20424C4583
:104EC0002074726166666963206C6F67202865765E
:104ED000656E7473202B206672616D65206865783D
:104EE0002064756D7029000072657365743A2073D3
:104EF000797374656D2072657365742028726562BC
:104F00006F6F74290000000073686F772046726528
:104F10006552544F532072756E74696D6520696EC9
:104F2000666F2028757074696D652F7461736B737B
:104F30002F686561702F7461736B206C69737429BD
:104F4000000000006C6564203C317C323E203C6FE8
:104F50006E7C6F66667C746F67676C653E3A206333
:104F60006F6E74726F6C20626F617264204C454486
:104F7000000000006F7461006C65640075617274FC
:104F80007273743A2072652D696E697420555341AD
:104F9000525431202831313532303020384E3129C9
:104FA0002C20666C75736820727820717565756544
:104FB00000000000626C656C6F67000062736475CE
:104FC0006D703A2073686F7720626F6F74736574C9
:104FD00074696E67207265636F7264202B20637240
:104FE0006320636865636B0073686F77206669721E
:104FF0006D776172652076657273696F6E0000006F
:1050000076657273696F6E00737973696E666F008F
:1050100075617274696E666F000000006465766980
:105020006E666F0068656C70205B636D645D3A202E
:105030006C69737420636F6D6D616E6473202F20D3
:1050400073686F77206F6E6520636F6D6D616E643E
:1050500027732068656C700068656C700000000044
:10506000627364756D70000075617274696E666F4D
:105070003A2073686F77205553415254312070693C
:105080006E732F626175642F666F726D61740000BC
:10509000617070676574000072657365740000006C
:1050A0006170707365740000627373657400000052
:1050B0006170707377205B317C325D3A2073776961
:1050C00074636820626F6F742062616E6B20286366
:1050D000726320766572696669656429202B207287
:1050E00065626F6F74000000666163746F72793A75
:1050F00020726573746F726520706172616D7320C8
:10510000746F2064656661756C747320616E6420D1
:105110007265626F6F7400007561727472737400EF
:105120006170707377000000666163746F7279005C
:10513000617070736574203C6C65647C70776D3E43
:10514000203C76616C3E207C206170707365742019
:105150006A736F6E207B226C6564223A3530307D35
:105160000000000075736167653A206170707365B7
:1051700074203C6C65647C70776D3E203C76616C7D
:105180003E207C20617070736574206A736F6E209E
:105190007B226C6564223A3530302C2270776D2288
:1051A0003A35307D0D0A000061707073773A2062E5
:1051B000616E6B256C7520696D6167652063726334
:1051C000206D69736D6174636820287265636F7206
:1051D000642030782530386C582C206163747561F8
:1051E0006C2030782530386C58290D0A00000000FA
:1051F0002020202020202020206231616464727CE5
:105200006232616464727C623173697A657C623295
:1052100073697A657C62316372637C623263726344
:105220007C62317665727C6232766572203C68659C
:10523000787C6465633E0D0A000000005C52010149
:10524000004000201C08000030950001705801014A
:105250001C480020BC710000F02A0000A00600904D
:10526000D00300011005A00000FF01D200010006DC
:1052700051C20200200001302B11D80D49086849A5
:105280006813F008FB0498EFF78EFF0446C188808E
:1052900088FF22FFF79DFD2046FFF73AFCB3E705A4
:1052A000B0F0BD98100707D8010020C804202930AD
:1052B000D70200004B1847FBFD06460520307075ED
:1052C000800099B181301D3946E5F773FD3046F90C
:1052D000F70EFF0E22294642200445FD07403011FB
:1052E0002E0CD0534B052203212846FDF733FE1226
:1052F0001E40274B75002D05D0398F002902D000A4
:1053000099897900E000211176FAF74BF8044D28CD
:1053100059F9F7FBFE0020285180100600040020F8
:105320000777107838B5049C0094014CA04738BD2D
:105330005143F84A26468F1839462036FD6D707D58
:1053400080311191C97FA0370E91224639781532EC
:105350000F92F14A109203292BD0002873D0F17DCF
:105360000F980CF00DF800286FD068886946088304
:10537000F0B597B008780C460F90002014900F9865
:1053800048214843FE492246401806468036109080
:10539000F17F0091C56DA0301690014E100A27468E
:1053A00012922037F74A1552146C2AD061783C29A2
:1053B00049D0432947D0787D00287DD0F97D1298C7
:1053C00000F0FCF9002878D0698868468184687A02
:1053D000297A000409020843E97908430690A97A6A
:1053E00008A84172E97A8172297BC17229460D3180
:1053F0000E380E9100F02FFAA878400733D500211F
:1054000032E0907E012806D0507E401E0006000E3D
:10541000507603D006143004DB480106141200F065
:10542000D2F9169A01211170A978D448C9075C36BF
:1054300090264823594308180022A0300270FF200C
:10544000F07752E001220270A878CC49C0074CD016
:105450000098482358434020101442E0E97C08A8F3
:105460000173297D4173697D8173A97DC108100D88
:105470000174297E4174697E8174B189BC102281D6
:10548000F189C181318A0182109940318A8F8283EA
:10549000C98F0184B188C183F18841840021C1840E
:1054A00042241472B848817808A8C17401E04DE123
:1054B0001BE002260675C821CC140C02D4E87A80C1
:1054C0000705D5297B0E14300A7EF908A908750353
:1054D000A90F0C1412002801D11698067060783CB0
:1054E0002870D030E1628A143D0A82A2884A82A2E2
:1054F000790A75E2794A75207A8875E07EC875A0C8
:105500008B0883E08B4883208C8883608CC8832140
:1055100046243108A800F0A4F9787A08A94871B89F
:105520007A8871A08DC8140585206B0BC210050CFC
:1055300090012018103F75387D0875B87D8875A8D2
:1055400078C006C017401CC8758E486946028A0A92
:1055500087428A4A87827D08A90A77C27D4A7702F4
:105560007E8A77428B10A90A80828B4A80807F08CE
:105570007104A900A4380432F9000A14487C494097
:105580001803907C30129900F05DF90398F97D8042
:1055900030817003990922A0310A700121C1700382
:1055A0009800218166E18B490041660521C16601B1
:1055B0006715996030C97E002904D0724981610164
:1055C0002102E02ABA48098161817500998182240B
:1055D000400DF6F8022802D2012100F003F9122052
:1055E0001B05F906280CD20A215F4A41438918FF9E
:1055F000318131497F890703D5FA7D7C23FCF896F8
:105600001005FFF81699E035C41A01AE18180920E4
:1056100000F0FBF821460F31059100284ED02023E1
:105620003E22002156241C06F6F806460A96031769
:1056300014986C1ED03A04200EE03C2070700120BB
:105640003071009870801620052CD0B01D5A2407A8
:10565000F2F8F87D7071AC201306D521463046096A
:10566000310C3000F0E7F803E030460A12DD202567
:10567000C8100630461230053032DA1A12121A14E7
:1056800006D0F8E08B309A16709A2813B083B87A57
:10569000B077304600F0BFF83AE0287B7071DC202C
:1056A00007B01D00F0C2F8163006B4F83DE0149EB5
:1056B0001A2EC23008A7F801210646019E120D9E3F
:1056C000300470703198200BF87D820709D5717114
:1056D000B01D6A3004A5F80AB6400B30461DE0C084
:1056E00007C00F7071B2129978100BB081208CF046
:1056F00081608C308278227462300483F8066012F4
:105700001660302477F81421017000994180B97D2A
:10571000017100F075F81598807E022826D1607816
:105720001499084322D0082C120B2C100461F81293
:105730002C1C0C61784170297881700FE040640462
:105740001C06C00600200A6E0512390412400C1D0A
:1057500088031C0820B1A201000411A005100799BC
:105760008180397E81563C064AF8002017180510C2
:105770000640BA7047C004600D03B40148019001AF
:10578000BD919B02000C83E1980C837D9F0C7004FB
:1057900049FA010C8309D30C836D5B24933D99482E
:1057A0008290488355073083D59C3083397B18100D
:1057B00027796D0100002101804180818070470AB6
:1057C0007802704B7843708A788270CA78C2700B06
:1057D0007903714A7942711A20046802600E0F340D
:1057E000704740063414497B41700570F1F7F3FCB3
:1057F0002068F1F7A4FB256003141B2400761C0924
:1058000080024080C10240062B066419F8B54E782C
:105810004821F0B248432349214D41180C46AA7E45
:10582000A0340027282C22EDC3020010B5074CE05D
:1058300069000408D5FFF7F3FF0548007800280247
:10584000D10120C0032062100006115012C658007A
:10585000045DF4010001CD8007100669B90001055F
:1058600004000457D12D017A12AA01E1D6000000EC
:020000040102F7
:10400000D8B90020694102017141020165720201C3
:1040100000000000000000000000000000000000A0
:1040200000000000000000000000000029760201EE
:104030000000000000000000274102012D7602016F
:104040007B4102017B4102017B4102017B41020174
:104050007B4102017B4102017B4102017B41020164
:104060007B4102017B4102017B4102017B41020154
:104070007B4102017B4102017B4102017B41020144
:104080007B4102017B4102017B4102017B41020134
:104090007B4102017B4102017B4102017B41020124
:1040A0007B4102017B4102017B4102017B41020114
:1040B000357802017B4102017B4102017B41020113
:1040C0000348854601F076F8004800473DBD0201EF
:1040D000D8B9002040BA7047C0BA70470138FDD146
:1040E0007047000040BA7047C0BA704770467047CA
:1040F000084B19680868203080F30988022080F393
:104100001488BFF36F8F3FBCAE4608BC04BC62B6D8
:1041100018470000B4470020EFF3108072B67047D4
:1041200080F310887047EFF309800E4B1A6820382F
:104130001060F0C044464D4656465F46F0C008B594
:1041400072B60BF019FA62B60CBC11680868103030
:10415000F0C8A046A946B246BB4680F3098820387D
:10416000F0C81847B4470020044880470448004777
:10417000FEE7FEE7FEE7FEE7FEE7FEE785760201E3
:10418000C140020130B50B46014600202022012427
:1041900009E00D46D5409D4205D31D469540491B7B
:1041A0002546954040191546521E002DF1DC30BDC4
:1041B00070B500242546002801DA01244042002978
:1041C00001DA01254942FFF7DDFFAC4200D0404251
:1041D000002C00D0494270BDF0B51FB40646002047
:1041E00082B005464024019100901BE001992246CF
:1041F0000F46304600F02DFE049A059B801A994127
:1042000010D310461946224600F013FE361A8F418D
:104210000197224601200021009F00F00AFE381875
:104220004D4100902046641E0028DFDC019B009871
:104230002946324607B0F0BD01464139192900D858
:10424000203070470549064A08685043054A8018DF
:104250000860400870470149086070470C4800201A
:104260006D4EC6413930000003460B439B0703D017
:1042700009E008C9121F08C0042AFAD203E00B782B
:104280000370401C491C521EF9D27047D2B201E0A3
:104290000270401C491EFBD270470022F6E710B5A1
:1042A00013460A4604461946FFF7F0FF204610BDA4
:1042B000421C0178401C0029FBD1801A704710B5C0
:1042C000002200E0521C835C8C5CA34201D1002BD5
:1042D000F8D1D8B2E1B2401A10BDC9B203E00378F8
:1042E0008B4203D0401C521EF9D20020704730B5DB
:1042F00004460020034600E05B1C934203D2E05CCE
:10430000CD5C401BF8D030BD03460A780270401CDB
:10431000491C002AF9D11846704730B505460020DF
:10432000034600E05B1C934205D2EC5CC85C201A9B
:1043300001D1002CF6D130BD0FB400B58DB009907D
:104340000B9010A900200091C0430A9000200C900F
:1043500006480690064807906A4609A80F9900F09B
:10436000B1FD0DB008BC04B018470000E54E0201D5
:10437000054F0201FFB5087889B01546FF2805D022
:10438000491C2D2804D00022002407E000240BE063
:104390000122F9E70A235C430419491C0878FF2825
:1043A000F8D1002A00D06442002004902A78014607
:1043B0002D2A01D02B2A0FD16D1C2D2A02D00022CC
:1043C000049209E00122FBE700260A2233466D1C15
:1043D00000F0F2FC381871412F78FF2FF4D10C9ABD
:1043E000A218069202460A4304D0FF23069A91338C
:1043F000DA4205DA002109980A4606C00DB0F0BD80
:104400000024B74AB54D2646079200F011FC0290F1
:1044100006980391002801DA474200E00746390573
:104420000020AF4A001C51410191009012E0F807B2
:1044300007D022462B463046079900F0D9FA0646A7
:10444000079122462B461046194600F0D1FA044641
:104450000D467F10002FEAD10698019B0028009A94
:104460000399029806DA00F02BFB3246079B00F016
:1044700027FB05E000F0BCFA3246079B00F0B8FAD3
:10448000049A002A02D00122D2075140099A03C29D
:10449000B4E7FFB591B0002009900025ED432E2030
:1044A0009E685C681F460190B9696D1C1298884728
:1044B0000090396A88470028F6D10098401C0AD03D
:1044C0000D20C0018443002E12DD00982B2809D056
:1044D0002D280DD103E00020C04315B0F0BD012010
:1044E00080020443B9696D1C12988847761E0090BB
:1044F00003A9600501D52D2000E02B206A4610732A
:10450000491C0CA80F9102900AE0B9696D1C129821
:10451000884700900120400204431398761E0560EE
:10452000002E02DD00983028EFD0019900988842D3
:1045300046D18020044308E00998401E09900120DC
:10454000400204431399681C0860B9696D1C761E0B
:104550001298884700903028EED031E001998842C7
:1045600005D1200603D480200443761E1EE0009867
:1045700003F06EFB002826D001204002044307A967
:104580000F980331761E88420BD200980F9930386D
:1045900008700F98401C0F90200607D50998401E00
:1045A00003E0200602D40998401C0990A00502D51A
:1045B0001399681C0860B9696D1C129888470090AF
:1045C000002ECBDC59E0002E57DD0098652801D085
:1045D000452852D1A00550D5032000028443B96973
:1045E0006D1C761E129888470090002E0CDD2B283B
:1045F00004D02D2808D1FF2001300443B9696D1C77
:1046000012988847761E0090E00501D52D2100E024
:104610002B21029801700298401C0290019025E025
:104620000120400204430EA902980131761E8842FF
:104630000ED20098029930380006000E087003D19F
:104640000299019881420AD90298401C029006E022
:10465000E00501D5234801E0224840420990B969AC
:104660006D1C12988847009013980560002E04DD99
:10467000009803F0EDFA0028D2D1F9691298884722
:104680000F99FF200870029903AA087000200A9071
:104690000B900CA90AA8099BFFF76CFEA00502D499
:1046A0000120C04319E72420044209D0E00713D1B8
:1046B00038680B9A0A99031D3B60006806C00BE03E
:1046C0000B990A9800F05CFB0146E00704D13868BA
:1046D000021D3A60006801602846FEE600001440B2
:1046E0000000F03FF1D8FFFFF7B582B00F4600267B
:1046F000029C03F099F90090006801902578641CF1
:10470000002D05D000F0CAFB0068405DC007F5D160
:104710002B2D02D02D2D1CD0641E0098002101608D
:1047200039462046049A00F0FFFB0146002F04D0D2
:104730003868A04201D102983860009800680228C9
:104740000BD00098019A0260700506D5484205B06A
:10475000F0BD012080020643DFE70846F7E7F8B521
:1047600002464A40D40F42004B0052085B089A426E
:1047700002D20246084611464A0023D0C30D4A0021
:10478000DDB2120EAD1A202D35DA49020126490A92
:10479000F6058A19002C00D0524220214F1B1146E9
:1047A000B9402A411018C20D9A4221D0002C17D0CE
:1047B000012D08DCDA05801AD20F8019D207DBB28E
:1047C00000F060FCF8BDDA05801A012340001B06EA
:1047D000C01880185A428018CA0F1043490007E0D9
:1047E0004908C2071143DA05801A80194008801869
:1047F00000F040FCF8BD61000122511A001BF7E7F0
:104800000122D2075140AAE70122D2075040A6E771
:10481000024670B54A40D30FDB0740002DD04A0056
:104820002AD0010E140E000212020919400A520A7F
:104830008418E50104465443000A120A2E0450432A
:10484000A4194219200CC543AA18120C0125AD0366
:10485000521C521912047F39240400D0521C1043F8
:1048600001D44000491EC2B20C06C0092018401CE9
:104870004008802A02D003E0002070BD40084000BC
:10488000002900DA0020184370BD0000F0B507468B
:104890000846584087B0C00F049048000E465900A3
:1048A00040084908BC1A884105D2384631461E46A0
:1048B00017460B4602465800400810434CD0300DB6
:1048C000039040055900400D490D0590401A029093
:1048D000402872DA18030121000B090508430190F2
:1048E00004980092002805D0019952420020884186
:1048F00000920190029840210A1A0199009800F054
:1049000098FA05460C466B4607CB00F0B3FAC0197F
:104910007141039A0E0D0023D71756401A467A406C
:10492000164344D0049A002A2DD0029A012A039AF1
:1049300015DC1205C01A914101263605001C714193
:10494000D20F059ED2070093019202962A46234673
:1049500000F0DEFB07B0F0BD38463146FAE7160539
:10496000224A0F46B218C01AB74101210905001C9E
:104970004F4100187F41114618187941E20F10434A
:104980006D19644113E0E2076D0815436408C2071E
:104990001443039A01261205C01A91413605001CE2
:1049A0007141CE07400830434908C01851412A469A
:1049B000234600F0A0FBCDE7FFE70498012240006A
:1049C000C117121A00238B4104983146C417381AB4
:1049D000A141EEE730B40124E407634030BC55E761
:1049E00030B40124E407614030BC4FE70000E0FF31
:1049F000F0B51FB488B00B99099800244840099974
:104A0000C00F490049080991C0070B99009049005F
:104A100049080B9109990898A64608431CD00B99A0
:104A20000A98084318D0099801244000420D480014
:104A3000410D099824050003000B204309900B98B1
:104A40000003000B20430B9050181C494018002213
:104A500001901446104605E0002001460DB0F0BD5F
:104A6000032801DA034600E003239C46C11A0AAE7C
:104A70000AE05F0008ADED5B4F00F75B7D43002768
:104A8000AA187C41491C5B1E6145F2DD410004AB64
:104A90005A522104120C0A43240C401C0828DFDB64
:104AA000019802900099704601910090059B049A2C
:104AB0000799069800F02CFBD0E700000DFCFFFFE3
:104AC000F0B50C465C4085B0E40FE40703944C005D
:104AD000002664085900944649080246029622437B
:104AE00021D062460A431ED06200570D4A000E03D1
:104AF0002303550D012402462C492405781B1B0B6A
:104B0000360B401823432643614600901C46501A3A
:104B1000B44103D30098401C009002E09218009822
:104B20005B41002803DA0020014605B0F0BD0020FB
:104B3000012109050746864611E064461D46141BFF
:104B4000B54106D36546521BB341744607430C4337
:104B5000A646CD0740084908284392185B41054600
:104B60000D43EAD11046184313D060461946504011
:104B70007140084306D06046101AB34106D20122A4
:104B8000002306E000220123DB0702E00122D243DA
:104B90005310009874460105381C6141029C039D26
:104BA0000019694100F0A7FABFE70000FD0300000B
:104BB00070B54B005B0803430BD04B005C0D002627
:104BC00033466542B341D417AD1AA34102DB00203E
:104BD000014670BD12053018514170BD10B500225C
:104BE0009623114600F04EFA10BD00000EB5C21714
:104BF000C10F5040CA0740180021054B0293019293
:104C000000910A460B4600F083FA03B000BD000095
:104C1000330400000EB505490291002100910A46B7
:104C20000B46019100F074FA03B000BD330400009C
:104C30000EB5054A0292002200921346019200F03E
:104C400067FA03B000BD000033040000C20F41004A
:104C500040020123400ADB05D207090EC0187F2954
:104C600001DA00207047962903DC9623591AC840C0
:104C700001E096398840002AF4D040427047000095
:104C800070B5CD0F4A0009030123090B1B05194319
:104C90000B4BED070024520D9A4201DA002070BD43
:104CA000074B34339A4203DC9A1A00F0D2F802E040
:104CB0000449511888402C43F1D0404270BD000097
:104CC000FF030000CDFBFFFF4A0009030123090B8E
:104CD0001B0519430A4B10B5520D9A4202DA002007
:104CE000014610BD064B34339A4203DC9A1A00F099
:104CF000B0F810BD034BD21800F09BF810BD0000B7
:104D0000FF030000CDFBFFFFC20FD20740004008A9
:104D10000BD0C10D0723DB01C91840020905400A69
:104D20001143C208400711437047002001467047F5
:104D300010B5002904DB0124E40740428C412146E0
:104D4000002B04DB1C460123DB075242A3418B42AC
:104D500000D1824210BD000010B5002904DB0124FF
:104D6000E40740428C412146002B04DB1C46012312
:104D7000DB075242A341994200D1904210BD00008E
:104D8000CB0FDB07490010B5490802460A4307D09C
:104D90000A0D07240903E401090B121B002A01DC98
:104DA000002010BDC900440F0C43C100E018D2051B
:104DB000801800F05FF910BDF0B51FB486B0002078
:104DC0000090019002900698069980B2049007988E
:104DD000090C02040014114307900027089D09984C
:104DE00006913E463C4603900398A9B20204000C8B
:104DF000039004982D0C154348430021224600F0EF
:104E000018F8C719714110340E46402CECDB3846B7
:104E1000029A00F00EF8009A019B80180090594108
:104E200002980191103002904028CCDB00980BB022
:104E3000F0BD10B5202A04DB0146203A9140002045
:104E400010BD914020239C1A0346E3401943904033
:104E500010BD10B5202A04DB0846203AD0400021BE
:104E600010BD0B46D340D0402024A21A91400843E5
:104E7000194610BD10B5202A06DBCB170846203A8C
:104E80001041C1170B4306E00B461341D0402024CC
:104E9000A21A91400843194610BD0000004870470F
:104EA0008C0E030110B50446FFF7F8FF0068005DA3
:104EB000C007C00F10BD00000268137851180160D0
:104EC0001846704710B5D160044951610449116218
:104ED00000211161114600F08FF910BDB94E020199
:104EE000A54E02014268002A08D001680B78491CCF
:104EF000002B03D0521E06C0184670470121C16026
:104F0000881E70474268002A0BD0C3680168002BD6
:104F100007D183688B4204D0491E521C06C0002072
:104F200070470020C0437047F7B582B0029C00274D
:104F30002078641C15460197302802D0002D15D02A
:104F400015E020780127641C782804D0582802D066
:104F5000002D09D00BE0002D01D0102D07D1002726
:104F600010252078641C02E0082500E00A250026B0
:104F7000009610E00099012769430818020C2946A1
:104F800080B2714300908E183804864201D301200C
:104F900001902078641C294600F01EF90028E9DA07
:104FA0000398002805D0002F01D0641E00E0029C69
:104FB00004600198002806D002F036FD022101604D
:104FC000C81E05B0F0BD009930040843F9E70000A1
:104FD0000FB400B589B00CA900910B990023CB60E8
:104FE000204B214A06930792042201921F4A029203
:104FF0001F4A089202466B460020FFF74AFA09B0A2
:1050000008BC04B0184770B586B006460020C043FF
:105010000190002015460C46009102910490324602
:10502000694604A8FFF7D4FF024604982118002D12
:1050300005D0002801D0084600E0204628600498EA
:1050400000280DD0002A02DD0098884208D0081BF5
:105050000190009432466946029404A8FFF7B8FF15
:1050600006B070BDE54E0201054F0201FFFFFF7F54
:10507000A54E0201002904DA401C490001D1400874
:105080004000704770B40024050C05D110240004C2
:1050900002D1002921D01124050E01D100020834CB
:1050A000050F01D10001241D850F01D18000A41C32
:1050B000002801DB4000641C002908D020252E1B9D
:1050C0000D46F540A14000D00121294308430106C7
:1050D0001B1B000ADB1D02D5002070BC7047DB05DE
:1050E000181880180029F8DA401C4900F5D170BC66
:1050F00040084000704710B5002B08DA0024401C1F
:10510000614192185B411A4301D14008400010BD33
:10511000F0B51FB482B005460C0003D0084602F07B
:105120006BFC02E002F068FC203002460090214651
:105130002846FFF77EFE049B059A04460F46184357
:105140001143084314D0184610431BD00098402147
:105150000A1A18460599FFF77CFE05460E46009A86
:1051600005990498FFF765FE084305D0012004E087
:105170002046394607B0F0BD0020C11705430E4355
:105180002C43374300990E986305401A7905E40AC9
:1051900000220C43FD0A0A3002D500200146E9E74F
:1051A0000105101969410C9C0D9D00196941FFF71B
:1051B000A2FFDFE7064C0125064E05E0E36807CCB9
:1051C0002B430C3C98471034B442F7D3FEF77CFFD6
:1051D00068130301881303013A2800D230382023D2
:1051E00002469A43412A01D310463738884201D3F8
:1051F0000020C04370470000F3B58DB000200A9036
:1052000001200B90002608460C300C46099062697C
:10521000012109989047051E2ED0252D2DD0216AF9
:105220008847002818D06269012109989047216AAF
:1052300088470028F7D1411E62690998904700E02D
:10524000761CA1690D988847216A88470028F7D104
:10525000E1690D988847DAE7A1690D988847074604
:10526000A84201D1761CD2E7E1690D9888477F1CDE
:1052700002D10A98002877D049E1002762693D46AB
:105280003946099890472A280CD16269012109986A
:105290009047012506E00A214F433F18303FEBD4E9
:1052A0001020054362690121099890470146303971
:1052B0000A2903D29B498F42DEDCECE7E90600D4E1
:1052C000994F6C280AD04C2810D0682824D06A281E
:1052D0002ED074280CD07A280AD00DE06269012102
:1052E000099890476C2823D004211CE02020054316
:1052F0006269012109989047A760656065284FD0D1
:1053000026DC582839D01ADC452849D012DC25285B
:1053100034D04128B0D143E0626901210998904717
:10532000682802D008210D43E6E70120C002DEE72D
:105330000220DCE7462833D047282CD130E05B2818
:1053400070D061282CD063286CD0642823D161E010
:105350006F284FD009DC662822D0672820D0692822
:1053600026D06E2817D12EE0CDE070284DD07328BE
:105370006FD075284ED078280DD154E0A1690D98D2
:1053800088470546252800D16CE7E1690D988847D4
:105390006D1C00D16DE7BAE00A224CE00A2252E00F
:1053A000012023466A46C0430D99FFF772F8A3E037
:1053B0002846402108436060A807234601D5002203
:1053C00039E000223FE0E80700D020E72068011D17
:1053D00021600068290501D5067018E7290701D565
:1053E000068014E7A90703D5F117066041600EE7B0
:1053F00006600CE72846402108436060A807234662
:1054000001D5082217E008221DE048492846084037
:10541000606016E02846402108436060A8072346E4
:10542000BCD5B9E715E02846402108436060A807CD
:1054300007D5234610220120C0430D99C046C0461F
:105440005AE0234610220120C0430D99C046C046B1
:1054500052E000210C910B460091632802D05B289A
:1054600007D043E0E80601D40120A06001200090AD
:105470003CE062690121099890475E2805D101202E
:105480000C9001466269099890472169002906D16C
:105490000B4601AA8F00491CD3510829FADB0028CA
:1054A00035D0216900290ED1C117C90E09184A113A
:1054B000930001AA9A1849094901411A0120136869
:1054C00088400343136062690121099890475D2871
:1054D000E5D10C98002808D0002001AB81005A5873
:1054E000401CD2435A500828F8DB01AB0120224669
:1054F000C0430D99C046C04600280ADA401C06D1B8
:105500000B98002803D00020C0430FB0F0BD0A98CC
:10551000FBE7E90702D10A99491C0A9136180020D5
:105520000B9074E6CCCCCC0CFFFFFF7FF1F7FFFFB4
:1055300070B58D180478401CA207920F01D1027833
:10554000401C231106D10378401C03E006780E703E
:10555000401C491C521EF9D1002B15D002780C2694
:105560008A1A3440401C0C2C03D0A401121B9B1C33
:1055700008E004782402121B401CF8E714780C7031
:10558000491C521C5B1EF9D5A942D3D3002070BD23
:1055900003B40148019001BD232A000003B401486F
:1055A000019001BD397B010003B40148019001BDA8
:1055B000B17B010003B40148019001BDBD80010031
:1055C00003B40148019001BD6D56000003B40148C9
:1055D000019001BD6560000003B40148019001BD68
:1055E000A1B3020003B40148019001BDAF7F0000E8
:1055F00003B40148019001BD1979010003B40148C9
:10560000019001BDB551000003B40148019001BDF6
:105610002D7A010003B40148019001BDD37E000042
:1056200003B40148019001BDD97C010003B40148D5
:10563000019001BD697E000003B40148019001BDE5
:10564000C37F000003B40148019001BDB57C010097
:1056500003B40148019001BD5DB6020003B40148E6
:10566000019001BD9D7B010003B40148019001BD83
:10567000D97B010003B40148019001BD7D7F010089
:1056800003B40148019001BDAD78010003B40148A5
:10569000019001BDE954000003B40148019001BD2F
:1056A0009957000003B40148019001BDED57000077
:1056B00003B40148019001BD1D7C000003B4014802
:1056C000019001BD617D010003B40148019001BD5D
:1056D000957D010003B40148019001BDDD7D01000D
:1056E00003B40148019001BD0D2A000003B4014834
:1056F000019001BDAB52000003B40148019001BD0F
:10570000E579010003B40148019001BDFD7A010073
:1057100003B40148019001BDE1AA020003B40148AD
:10572000019001BDF58F000003B40148019001BD57
:105730006DB1020003B40148019001BDE1FE00001B
:1057400003B40148019001BD250E010003B40148D6
:10575000019001BDB143000003B40148019001BDB7
:1057600085AC020003B40148019001BDA1AC020068
:1057700003B40148019001BD25B0020003B4014803
:10578000019001BDB5B2020003B40148019001BD12
:10579000D1B2020003B40148019001BD8529000087
:1057A000C943416070470268702392B29A430A432A
:1057B0000260704770B5044602F024F8002818D043
:1057C0008069002815D0FFF709FA05462046FFF743
:1057D00005FA2946FFF718F8FFF796FA064A074B2D
:1057E000FFF76EF90022064BFFF750F8FFF7C8FAF3
:1057F00070BD044DEAE700001F85EB51B81E014063
:105800000000394000803B4470B50D460646002438
:1058100001F0F8FF002816D0C169002913D0026AF0
:10582000002A10D08BB290B289B292B2102D0CD057
:10583000202D0AD0302D17D0402D15D0502D13D04B
:10584000602D11D022E0002070BD891AB01AAF225D
:1058500092005043FEF7ACFC044696340FD47D20F2
:10586000C000844211DC11E0191AAF22301A120173
:105870005043FEF79DFC4B21C900441801D500247C
:1058800004E0E1200001844200DD0446204670BDB2
:1058900070B5104CA0421BD185140121284601F09F
:1058A00063FE0021284601F05FFE0121284601F039
:1058B0004FFE094860610020206060601F21A160E8
:1058C00006492161A06160622062A0620448E06133
:1058D00070BD000000080240080A02000000FC0F32
:1058E0002E6D00000029016802D00122114301E061
:1058F000490849000160704704220029816902D0EB
:105900001143816170479143816108480649C16232
:105910000749016307494163074981630749C16337
:1059200008490748086070472200780000080240D4
:10593000E700E1009F00BF04190C051670206E28D7
:105940006E2B00004008024002220029016801D0AD
:10595000114300E0914301607047C06880B2704716
:105960000246526800200A4200D001207047000021
:10597000044A9068C90640094001C90E014391607C
:10598000704700000008024070B5054649480C46C3
:105990004EC88CB003960293019200914EC80796B0
:1059A0000693059204914268016880680992089103
:1059B0000A90414A00996846914217D1282104F083
:1059C00043FA0A99884211D1022D1ADB002064683B
:1059D00002460B900BA92046FEF786FE05460B9863
:1059E000A04209D00078002806D101E033A004E0ED
:1059F000012D0AD0022D08D03EA004F023FB0CB0EC
:105A000070BD0198012809D001250198A84207D14D
:105A1000294647A004F0B0FA0CB070BD0225F4E7A7
:105A2000012D6C4614D01834012D13D0474822683C
:105A3000824206D16068002803D00721890388428A
:105A40000AD9294642A0636804F096FA0CB070BDEA
:105A50000834E9E74C48EAE74CA004F0F3FA61683F
:105A6000206804F0F1F9A268824206D00346294674
:105A7000544804F081FA54A0BFE729465FA0636848
:105A8000E26804F079FA6846019503F0FDFD00280C
:105A900001D06AA0B1E76EA004F0D4FAC82009F0E2
:105AA00061FCBFF34F8F72497048C860BFF34F8FDE
:105AB000FEE700000040000111C011CA6170707360
:105AC000773A20626F6F7473657474696E672072C1
:105AD00065636F726420696E76616C69642C2072F4
:105AE000656675736520746F207377697463680DDC
:105AF0000A00000075736167653A20617070737702
:105B0000205B317C325D20286E6F20617267203D02
:105B10002073776974636820746F20746865206FE0
:105B2000746865722062616E6B290D0A00000000C6
:105B300061707073773A20616C7265616479206F6F
:105B40006E20415050256C750D0A00000040020186
:105B500061707073773A2062616E6B256C7520728C
:105B600065636F726420696E76616C696420286178
:105B70006464723D30782530386C582073697A65DA
:105B80003D256C75290D0A0000800001617070735D
:105B9000773A20766572696679696E6720746172FA
:105BA00067657420696D616765206372632028668C
:105BB0006577207365636F6E6473292E2E2E0D0A30
:105BC00000000000D4120301202020202020207299
:105BD000756E20424C45204F544120746F207772DF
:105BE00069746520612076616C696420696D616704
:105BF000652066697273740D0A000000617070732D
:105C0000773A2062616E6B256C7520696D616765FE
:105C1000206F6B20287665722030782530386C58DC
:105C20002C20256C752042292C20737769746368B9
:105C3000696E672E2E2E0D0A0000000061707073D1
:105C4000773A20666C617368206661696C0D0A00A2
:105C500061707073773A20646F6E652C2072657383
:105C6000657474696E672E2E2E0D0A000400FA0505
:105C700000ED00E010B50B488CB01EC803940293F1
:105C8000019200911EC80794069305920491426800
:105C9000016880680A9009920891684603F022FD25
:105CA0000CB010BD00400001F0B58DB00E460328C9
:105CB00007DA54A004F0C6F95AA004F0C3F95F480B
:105CC0000FE00024B76822460BA938460B94FEF774
:105CD0000BFD05460B98B84202D00078002804D08E
:105CE00057A004F0AFF90DB0F0BD5A4B87CB039726
:105CF00002920191009087CB07970692059104903C
:105D00009A68596818680A920991534A009908904C
:105D10006846914205D1282104F096F80A998842F4
:105D20000DD0009401940294039404940594069475
:105D300007940894099449A00A9404F083F955A1A2
:105D40007068FEF7BCFA002804D0706801786229F8
:105D500008D02BE0012D03D0022D01D04FA0C0E7C9
:105D600001953AE04178312902D0322902D01DE074
:105D700002AC00E006AC51A1801CFEF7A0FA00289E
:105D800016D070684FA1801CFEF799FA002819D030
:105D900070684EA1801CFEF792FA00281AD0706835
:105DA0004BA1801CFEF78BFA002815D049A098E77C
:105DB0004E48854204D04E48854201D04DA090E720
:105DC00025600AE007208003854201D958A088E7B2
:105DD000656002E0A56000E0E5602A465DA07168AC
:105DE00004F0CAF8684603F04FFC002801D062A016
:105DF00077E766A004F026F9684603F073FC0DB05F
:105E0000F0BD000075736167653A20627373657455
:105E1000203C6669656C643E203C76616C3E0D0AF0
:105E20000000000020206669656C643A206163749C
:105E3000697665203C317C323E0D0A001C1303015B
:105E400062737365743A206261642076616C756573
:105E50000D0A00000040000111C011CA6273736591
:105E6000743A206578697374696E67207265636F30
:105E7000726420696E76616C69642C20726562754B
:105E8000696C642066726F6D2073637261746368FD
:105E90000D0A0000616374697665000062737365C2
:105EA000743A20616374697665206D75737420623D
:105EB000652031206F7220320D0A00006164647227
:105EC0000000000073697A650000000063726300DF
:105ED0007665720062737365743A20756E6B6E6FCF
:105EE000776E206669656C640D0A00000080000111
:105EF0000040020162737365743A20616464722029
:105F00006D7573742062652043414949435F415078
:105F100050315F42415345206F722043414949430C
:105F20005F415050325F424153450D0A000000006E
:105F300062737365743A2073697A65206578636566
:105F4000656473207468652062616E6B2073697A82
:105F5000650D0A0062737365743A202573203D2035
:105F600030782530386C582C2077726974696E67E8
:105F70002E2E2E0D0A00000062737365743A20669F
:105F80006C617368206661696C0D0A0062737365E9
:105F9000743A206F6B20287665726966696564299A
:105FA0000D0A000000B583B0002103200B4601223A
:105FB00001910090920203A1034809F049FE03B049
:105FC00000BD0000434C4900D163020110B5022816
:105FD00005DB48680DA1FEF772F9002805D00D48D1
:105FE0000078002804D00CA103E007F09FF910BD51
:105FF0000BA110A003F0C0FF124C13A0218903F0E5
:10600000BBFF1CA0E16803F0B7FF10BD6A736F6EA1
:10601000000000009847002076616C696400000071
:1060200064656661756C7420286E6F742073617688
:1060300065642900706172616D733A2025730D0AE1
:1060400000000000B45E002020206C6564203D202C
:1060500025752020286C65643120626C696E6B2088
:1060600068616C6620706572696F642C206D73299D
:106070000D0A0000202070776D203D20256C7520D2
:10608000202870776D20647574792C202525290DC2
:106090000A000000F3B595B015980D46032807DAFD
:1060A0006F4803F0CFFF6FA003F0CCFF79A023E08F
:1060B0007FA16868FEF703F9002810D00020AE68C1
:1060C0000246009069463046FEF70EFB04460098F3
:1060D000B04202D0007800287BD077A00CE00024EA
:1060E0000226B00014902858FEF7E2F80746E0199F
:1060F000801C502804D975A003F0A4FF17B0F0BD90
:10610000002C03D0202069460855641C14983A4698
:10611000295868460019FEF7A7F81598E419761C67
:106120008642DEDB002069460855451E6E462C4639
:1061300005F0B2FC304603F0DDFD060023D003F08D
:10614000BEFD00281FD069A1304603F081FD07463F
:1061500003F0ACFD002800D07D6965A1304603F056
:1061600077FD074603F0A2FD002800D07C69002DD2
:1061700013DA002C22DA5FA003F064FF304603F04C
:106180003DFD17B0F0BD65A003F05CFF002EF8D018
:10619000304603F033FD17B0F0BD2946664832396A
:1061A000814209D3654A322165A003F0E5FE3046FD
:1061B00003F024FD17B0F0BD002C0BDB642C09DDCF
:1061C000642164A003F0D8FE304603F017FD17B039
:1061D000F0BD14E0304603F011FD002D01DB6248F4
:1061E0000581002C01DB6048C46007F0F3F800284B
:1061F00001D05EA080E707F099F817B0F0BD3BA191
:106200006868FEF75CF8002807D039A16868FEF7D7
:1062100056F800280DD05CA06EE72046464932387B
:10622000884203D3454A322145A015E04E480481F7
:1062300009E0642C05D9642146A003F09DFE17B047
:10624000F0BD4948C46007F0C5F8002801D055A04A
:1062500052E7224659A0696803F08EFE17B0F0BDE0
:106260009012030120206C6564203D206C65643130
:1062700020626C696E6B2068616C66207065726963
:106280006F642035302E2E3130303030206D730D5C
:106290000A000000202070776D203D2070776D206F
:1062A0006475747920302E2E31303020250D0A008F
:1062B0006A736F6E000000006170707365743A203D
:1062C0006261642076616C75650D0A00617070739F
:1062D0006574206A736F6E3A206C696E6520746F06
:1062E0006F206C6F6E670D0A000000006C65640023
:1062F00070776D00617070736574206A736F6E3AA9
:10630000206E6F206B6E6F776E206B657920286C26
:1063100065642C2070776D290D0A00006170707320
:106320006574206A736F6E3A2070617273652066BF
:1063300061696C0D0A000000DF26000010270000D4
:106340006C65642072616E67652025752E2E25753B
:106350000D0A000070776D2072616E676520302E27
:106360002E25750D0A000000B45E00206170707368
:106370006574206A736F6E3A20666C61736820667C
:1063800061696C0D0A000000756E6B6E6F776E2090
:10639000706172616D20286C65642C2070776D29A6
:1063A0000D0A00006170707365743A20666C617349
:1063B00068206661696C0D0A000000002573203DAD
:1063C00020256C752C2073617665640D0A00000031
:1063D000002498B0F8A527461594661E2846129406
:1063E000FDF766FF81B2284603F046FBFE48002514
:1063F0008078002839D06421684603F09DFA00288F
:1064000016D06846007802F037FE00280ED0F64914
:106410000020887003F00EFBF4A52846FDF748FF26
:1064200081B2284603F028FB03F014FB002518E096
:10643000643502F071FDF748854212D3EA49002025
:10644000887002F069FD02F05DFD03F0F3FAF2A03E
:106450000190FDF72DFF81B2019803F00DFB03F0D1
:10646000F9FAE14880780028C5D10021C94368467F
:1064700003F062FA0028B9D01598002805D0002151
:106480001591694609788142B0D0129801281FD031
:10649000022826D0684600781B287DD009287CD0A9
:1064A0000D287BD00A287AD0082879D07F2877D089
:1064B000014620395F2999D23F2C72D2E149085513
:1064C000641CA4B20121684603F0D6FA27468DE782
:1064D000684600785B2802D00020129086E70220F0
:1064E000FBE70020129068460078412816D0422829
:1064F000EDD1002EEBDB761E57D4BB484078801BD5
:10650000C01DC117490F0918C908C900401A8101E7
:10651000CD4809184038FDF7F7FE49E0B248711C34
:1065200002789142D3DA4078761C801BC01DC117D7
:10653000490F0918C908C900401A8101C248091841
:106540004038FDF7E1FEBF480290FDF7B1FE85B28D
:10655000BEA42046FDF7ACFE81B2204603F08CFAC3
:106560000024002F0BD9BCA00190FDF7A1FE81B241
:10657000019803F081FA641CA4B2BC42F3D3B3A423
:106580002046FDF795FE81B2204603F075FA002DF6
:1065900034D02946029805E036E038E0E2E0E3E056
:1065A00081E18EE103F068FA28E0A6490020087036
:1065B000A4480290FDF77CFE85B2A4A42046FDF716
:1065C00077FE81B2204603F057FA0024002F0BD942
:1065D000A1A00190FDF76CFE81B2019803F04CFA86
:1065E000641CA4B2BC42F3D398A42046FDF760FE1D
:1065F00081B2204603F040FA002DCAD12F469148BF
:10660000FDF756FE84B2F1E601201290EEE603F0AB
:1066100011FA8C4800252F46019003F044FC13909A
:10662000224620210198FDF758FE002860D10199EB
:1066300008551399149000295AD9149803F036FC80
:10664000224616900199FDF768FE002819D1002F07
:106650000AD102A81699FDF757FE02A8FDF728FEF9
:1066600085B20DE06D1EADB2A54206D92A4602A83C
:106670001699FDF752FE0028F4D1002102A84155D9
:106680007F1C14981399401C14908842D5D3002F76
:1066900064D0012F1AD0A5422BD902AF3F2C5DD276
:1066A000AC425BD23819012103F0E6F90198395D5B
:1066B0000155641CA4B2F1E73819012103F0DCF99B
:1066C0000198395D0155641CA4B200E002AF3F2C73
:1066D00044D2AC42F0D3019920200855641C5EA539
:1066E000A4B22846FDF7E4FD81B2284603F0C4F9C0
:1066F00034E05AA52846FDF7DBFD81B2284603F0B9
:10670000BBF91398002500281CD9284603F0CEFBBE
:10671000074622460199FDF700FE00280ED13846B3
:10672000FDF7C6FD81B2384603F0A6F94CA73846FE
:10673000FDF7BEFD81B2384603F09EF913986D1C3B
:106740008542E2D345A52846FDF7B2FD81B2284631
:1067500003F092F92146019803F024FC274603F048
:1067600079F943E60A2000E00D20159003F062F964
:106770003AA52846FDF79CFD81B2284603F07CF936
:106780003049002008550D462878002877D0164C4F
:10679000207800280AD06078C01D4007C10D2A4823
:1067A00008182946FDF78BFD002868D06078810124
:1067B00025480818294656E00D0A434C49207265C1
:1067C0006164792E2054797065202768656C702784
:1067D00020666F7220636F6D6D616E64732E0D0A9B
:1067E00063616969632D3E00444700200D0A5B6FB9
:1067F00074615D2061626F727465642C20626163F4
:106800006B20746F20434C490D0A63616969632DE5
:106810003E000000102700000D0A5B6F74615D20D0
:1068200069646C652074696D656F75742C20626194
:10683000636B20746F20434C490D0A63616969637F
:106840002D3E0000D0500020105100200D636169E2
:1068500069632D3E00000000200000000D0A0000CA
:10686000202000000BE0FDF74FFD6078401C400742
:10687000400F60702078082801D2401C2070002052
:1068800003F0DAFB134803F01DFB13A42046FDF7C9
:106890000FFD81B2204603F0EFF803F0DBF800248F
:1068A0002746661EA2E5002CFCD0641E0CA5A4B2EF
:1068B0002846FDF7FDFC81B2284603F0DDF82746A7
:1068C00094E508A52846FDF7F3FC81B2284603F0BD
:1068D000D3F88BE5D050002063616969632D3E00D9
:1068E000082008000700000010B50C46022812DB43
:1068F0000EA16068FDF7E3FC002809D00CA16068D8
:10690000FDF7DDFC002804D00AA003F09BFB10BDBE
:10691000012001F075FF01F06DFF002801D003A1F7
:1069200000E003A10AA003F027FB10BD6F6E00007A
:106930006F66660075736167653A20626C656C6F9F
:1069400067205B6F6E7C6F66665D0D0A000000005D
:10695000626C65206C6F673A2025730D0A00000099
:10696000F8B502F0DFF9074602F0D8F90546254AE6
:1069700025A128A003F000FB02F002FA01462CA09A
:1069800003F0FAFA2F48874203D12FA003F05AFBF5
:1069900015E000F037FF044602F024FA06460A210B
:1069A0003846FDF705FC0A460146002C01D0A069D7
:1069B00000E00020009033462BA003F0DDFA02F047
:1069C0002DFA014632A003F0D7FA3548854203D1AB
:1069D00034A003F037FB03E029463AA003F0CCFAD9
:1069E00009F002FA7D21C900FDF7CCFB014639A070
:1069F00003F0C2FA08F0F2FD01463AA003F0BCFA37
:106A0000F8BD00001500010056312E30302E323115
:106A1000000000006669726D776172653A20257327
:106A2000202830782530386C58290D0A00000000E5
:106A30006375722062616E6B3A2041505025750D6E
:106A40000A000000FF7F0000636869702074656DB4
:106A5000703A2041444320726561642074696D6519
:106A60006F75740D0A000000636869702074656DAD
:106A7000703A2025642E2564204320286164633DFC
:106A80002575207472696D3D256C75290D0A00000D
:106A90007664643A202575206D560D0A00000000CA
:106AA000FFFF000066616E2072706D3A206E2F61EC
:106AB00020286E6F20746163686F6D65746572293C
:106AC0000D0A000066616E2072706D3A2025750D0A
:106AD0000A000000757074696D653A20256C752098
:106AE000730D0A006672656520686561703A20253D
:106AF0007520420D0A00000002F0D6FB00280DD0E0
:106B000007A003F09FFAC82008F02CFCBFF34F8FBA
:106B100011491048C860BFF34F8FFEE70FA0F0E7A0
:106B2000666163746F72793A20666C61736820776E
:106B300072697465206661696C65642C2072657386
:106B4000657474696E6720616E797761792E2E2E77
:106B50000D0A00000400FA0500ED00E066616374B0
:106B60006F72792064656661756C747320726573E9
:106B7000746F7265642C20726573657474696E67D6
:106B80002E2E2E0D0A00000070B5194D0E4602285B
:106B900019DB00240C20604329587068FDF78FFB37
:106BA000002807D0641C102CF4D312A0716803F0E5
:106BB000E3F970BD0C20444360194268295916A0BE
:106BC00003F0DAF970BD17A003F03CFA0024204668
:106BD0000C21484341194A6829580FA003F0CCF909
:106BE000641C102CF3D312A003F02CFA70BD00002B
:106BF000440D0301756E6B6E6F776E20636F6D6D64
:106C0000616E643A202573202874727920276865A4
:106C10006C7027290D0A00002020252D38732025AF
:106C2000730D0A00636F6D6D616E64733A0D0A0037
:106C30006B6579733A20544142203D20636F6D703B
:106C40006C6574652C2055502F444F574E203D20C5
:106C5000686973746F72790D0A00000070B50C4694
:106C6000032823DB60680178312902D0322906D05D
:106C70001CE04078002819D1184E012504E0407826
:106C8000002813D1164E402516A1A068FDF717FB6A
:106C900000280FD014A1A068FDF711FB00280ED02A
:106CA00012A1A068FDF70BFB00280DD011A003F086
:106CB000C9F970BD2946304600F05AFB08E0294664
:106CC000304600F051FB03E02946304600F022FB3D
:106CD00011A0A268616803F04FF970BD000C01407B
:106CE000000801406F6E00006F666600746F676792
:106CF0006C65000075736167653A206C6564203CC3
:106D0000317C323E203C6F6E7C6F66667C746F67B0
:106D1000676C653E0D0A00006C65642025732025B4
:106D20007320646F6E650D0A0000000010B5034803
:106D300003F088F901F0CEFE10BD0000900E0301B3
:106D400006A003F07FF9C82008F00CFBBFF34F8FBB
:106D500007490648C860BFF34F8FFEE77265736549
:106D60007474696E672E2E2E0D0A00000400FA0559
:106D700000ED00E010B509F037F87D210446C900A8
:106D8000FDF700FA0246214610A003F0F5F808F0DE
:106D90001BFA014614A003F0EFF808F025FC0446A6
:106DA00008F01CFC024605212346090311A003F04C
:106DB000E3F81DA003F046F92749002008700846B3
:106DC00008F0F0FA244803F03DF910BD75707469BD
:106DD0006D653A20256C75207469636B73202825D6
:106DE0006C752073290D0A007461736B733A20254A
:106DF000750D0A00686561703A20746F74616C20CB
:106E0000257520422C206672656520257520422C50
:106E1000206D696E20657665722066726565202535
:106E20007520420D0A0000006E616D652020202053
:106E300020202020202020202073746174652020D1
:106E40007072696F2020737461636B28772920202A
:106E50006E756D0D0A000000F04E002010B506A002
:106E600003F0F0F8E12149020BA003F085F816A029
:106E700003F0E8F810BD00007573617274313A20B8
:106E800054583D5042362052583D504237202841F8
:106E90004634290D0A000000626175643A20256CB1
:106EA000752C2038206461746120626974732C2011
:106EB0006E6F207061726974792C20312073746F49
:106EC00070206269740D0A00666C6F7720636F6EC4
:106ED00074726F6C3A206E6F6E653B2074783A2046
:106EE000444D41204348312028706F6C6C65642903
:106EF0003B2072783A205258444E452069727120E6
:106F000071756575650D0A0010B5E12464022046AF
:106F100002F058FD214602A003F02EF810BD00003B
:106F200075736172742072657365743A20256C758F
:106F300020384E312C207278207175657565206679
:106F40006C75736865640D0A0000000010B506A139
:106F500008A003F011F80DA003F074F819480168B7
:106F600019A003F009F810BD56312E30302E323101
:106F7000000000006669726D776172652076657247
:106F800073696F6E3A2025730D0A00006D636D2DD5
:106F90006464632D626C653A20424C4528726474C7
:106FA000737329202B204672656552544F53202B52
:106FB000205541525428444D4129202B20434C490F
:106FC0000D0A00000040002053797374656D436F13
:106FD0007265436C6F636B203D20256C7520487A89
:106FE0000D0A00004860704701681A4A11400160AC
:106FF0000021016041608160C160174A17499042D9
:1070000004D148680F22104348607047144A9042E8
:1070100004D14868F022104348607047114A9042FA
:1070200005D148680F2212021043486070470E4A8B
:10703000904205D148680F22120310434860704700
:107040000A4A9042FBD148680F221204104348605C
:1070500070470000FEFF00000800024000000240F0
:107060001C00024030000240440002405800024030
:107070000029016802D00122114301E0014A1140B8
:1070800001607047FEFF00000246096800201142BF
:1070900000D001207047000030B403680D4A0C6A2C
:1070A00013408A684D6922430C692C4322438C6942
:1070B0002243CC6922434C6A22438C6A22431A43FE
:1070C0000260CA6842600A6882604968C16030BC78
:1070D000704700000F80FFFF002B01D01061704748
:1070E00000201061704700000149486170470000AE
:1070F00000040140054B002219685B69014003420E
:1071000002D0002900D0012210467047000401403F
:1071100010B4837919490268002B28D00B68934377
:107120000B604A6803689A434A60027952181368F0
:107130000468234313608A6803689A438A60CA68B4
:1071400003689A43CA604279102A06D051180A6827
:10715000006802430A6010BC70478A6803681A43DB
:107160008A60CA6800680243CA6010BC7047007930
:10717000401801689143016010BC70470004014051
:107180000B680022002B56D0F0B401240B68944009
:1071900023424AD04B68022B01D0122B16D1130781
:1071A0000AD5456A5307DB0E0F269E40B5434E694C
:1071B0009E402E43466209E0056A5307DB0E0F2608
:1071C0009E40B5434E699E402E4306624B68012B9C
:1071D00005D0112B03D0022B01D0122B06D145680C
:1071E000DB06DB0FA54393402B4343600568530048
:1071F00003279F400E79BD43B607B60F9E402E432E
:107200000660C5688E68BD439E402E43C660856893
:107210000126A543CC6894402C438460C46A9E40F8
:107220000D69B4439D402543C5620B68521CD34091
:10723000ABD1F0BC70477047054901600022426045
:107240000F218260416101210261C160704700002D
:10725000FF3F0000816270478161704742694A4088
:107260004261704782B0EFF30884FCF73FFF4007AC
:1072700001D5EFF309840AA000F084FBE0680090D8
:107280000CA0A3686268216800F07CFBE0690090B4
:1072900014A0A3696269216900F074FBFEE7000095
:1072A0000A2A2A2A20486172644661756C74202A71
:1072B0002A2A0A00523020203D2530386C582052AE
:1072C0003120203D2530386C5820523220203D2579
:1072D00030386C5820523320203D2530386C580A05
:1072E00000000000523132203D2530386C58204CCF
:1072F0005220203D2530386C5820504320203D2519
:1073000030386C5820785053523D2530386C580A2C
:107310000000000010B5FFF7A1FF10BD30B5054615
:107320000E4887B00C46854202D10121042004E0BA
:107330000B48854210D10121082000F021F90948AD
:10734000844209D86846FFF777FF0120019069461B
:1073500000942846FFF714FF07B030BD0008014035
:10736000000C0140FF3F000010B5FFF773FF10BD98
:1073700010B5FFF771FF10BD10B400214156FF2377
:10738000CAB29207D40E4278A3409207120EA240CE
:1073900000290BDA0907090F08398C081049A400E5
:1073A0006118CC699C431443CC6107E08C080D49FB
:1073B000A40061180C689C4314430C60827801217E
:1073C0000078002A04D0C006C00E8140064803E0C1
:1073D000C006C00E81400548016010BC7047000027
:1073E00000ED00E000E400E000E100E080E100E00A
:1073F000F7B5FFB004460025A5B00520EFF31087D0
:10740000FF210090453102A8FCF747FFEFF31086FB
:10741000FF21453153A8FCF740FF53A801300190EC
:107420009822224953A8FCF71FFF012080F31088FF
:107430000198804786F3108801221D491203032614
:107440005300360388420AD194421AD09C4201D19B
:10745000151116E0B44210D101256D0211E0154955
:1074600088420AD1944201D115460AE09C4201D1DA
:107470001D4606E03546AC4203D000987FB028B0E8
:10748000F0BD06ACFF22013441320B4902A8FCF7E3
:10749000EBFE012080F310882846A69AA599A04704
:1074A00087F310887FB028B0F0BD000014020301FC
:1074B000C440130085601300D400030110B5EFF33E
:1074C0001084012181F31088FF2109064018034927
:1074D0000968884784F3108810BD0000044000202C
:1074E00010B50848064901600749416007498160B5
:1074F000C922920006490748FCF7B6FE10BD0000FD
:10750000F14800200440002085490020594800200F
:10751000B80203015048002010B5EFF31084012396
:1075200083F31088FF231B06C018034B5B68984742
:1075300084F3108810BD000004400020034AD16A83
:10754000102399430143D1627047000000100240AC
:10755000044A0029516901D0014300E0814351618F
:107560007047000000100240044A0029916A01D0CF
:10757000014300E081439162704700000010024027
:10758000044A0029916901D0014300E081439161DF
:107590007047000000100240012205491206012830
:1075A000086802D09043086070471043FBE7000072
:1075B0000010024030B4164A516804231940154B9C
:1075C00001D0042901D0036001E013490160516832
:1075D000124B8906890F5B5C0168D9404160536892
:1075E0000F4C5B055B0FE35C0D46DD408560536827
:1075F0009B045B0FE35CD940C160D16AC90601D529
:10760000084901E07D21C903016130BC70470000D9
:10761000001002400090D0030048E801AC020301D2
:10762000B002030100093D007047000010B5FCF7EF
:1076300073FD044608F0DEFB002803D00120034957
:10764000000748602046FCF76BFD10BD00ED00E030
:1076500010B50A4C2069411C01D000280AD1012034
:10766000064934220003FFF7C3FE2069411C03D002
:10767000002801D0024810BD002010BD1C48002089
:1076800045480020F0B5564C85B0E0692104084318
:10769000E0618120534D00062863534868615348D8
:1076A00028625348032201689203914301605149C3
:1076B00034228014FFF79CFE4E4B4F4E18694F4FFB
:1076C000411C29D0002827D0A9691A784909490105
:1076D000D206D20E0A43AA612168EA1391432160BF
:1076E00021687F22120291430002084320606068F3
:1076F000304360606068B84360606068211508438B
:107700006060206A3E4908402062206AD968090208
:107710000843206205B0F0BD6168204631436160D6
:107720006168B943616061680127BF0239436160E4
:10773000002104917D21C9000391002100917F2146
:107740004024002502950191026861028A4302608B
:107750000E11234908687F2212029043220202433D
:107760000A600520FCF7BAFC0120FCF7B7FC1C48B6
:10777000406B800704D4284603996D1C8842F3D9D6
:107780001748C06B80B2B04201D9811B00E0311AAA
:10779000B94202D2E2B28FB20292B04201D3019456
:1077A00000E00094019A00988018C005000EA042E5
:1077B00003D0044604988142CBD8094801687F224F
:1077C00012029143029A12020A4302604168490878
:1077D0004900416041684907FCD405B0F0BD000094
:1077E00000100240007000400F0800001800020066
:1077F000001001401C4800200000010000070000AC
:10780000FF00F8FF10B50A4C2069411C01D0002888
:107810000AD10120064934220003FFF7E9FD20695F
:10782000411C03D0002801D0014810BD002010BD2C
:107830001C48002010B502F09BF810BD10B40B06D8
:10784000CC065B0FE40E0121A140012B07D0022BD7
:1078500007D01430002A026805D00A4304E00C3037
:10786000F8E71030F6E78A43026010BC704700006A
:107870000029818903D001225203114301E0024A09
:107880001140818170470000FFDF0000002A828ADA
:1078900001D00A4300E08A43828270470246128880
:1078A00000200A4200D00120704770B40A06530F2E
:1078B000CE060125F60E2A460024B240012B0FD039
:1078C000022B10D0838A1340090A00888D4028407B
:1078D000002B02D0002800D00124204670BC704745
:1078E00083891340F0E7038AEDE7000070B5044692
:1078F000008A86B00D461B490840E9880143218271
:10790000A08919492A890840A98811436A89024334
:107910001143A181A08A15490840A9890143A18288
:107920006846FFF747FE1248844201D1039800E001
:1079300002982968192289005043FCF723FC064667
:107940006421FCF71FFC0501280964214843301A13
:1079500000013230FCF716FC0007000F284320819D
:1079600006B070BDFFCF0000F3E90000FFFC00008F
:10797000003801408088C005C00D7047C905C90D99
:10798000818070470FB410B503A9044B044A0298D4
:1079900000F066F910BC08BC04B0184739A5020114
:1079A000C40100200FB410B504A9074B02AA039824
:1079B00000F056F9044602A9002000F0F8FC204629
:1079C00010BC08BC04B01847AF8302017CB5154653
:1079D000024600201C4600290BD0491E009201914E
:1079E000044B6A462146284600F03AF9009A0021E5
:1079F00011707CBD998302012021020C01D010215D
:107A00001046020A01D010460839020901D010467A
:107A1000091F820801D01046891E420801D0881E25
:107A20007047081A70470000004870471848002047
:107A300030B5002805D0164C021F206800230146EF
:107A400005E0084630BD904203D803464068002850
:107A5000F9D1002B00D05968002B0AD01C68D51A28
:107A6000A54204D11268A4181A461C6002E05A60AC
:107A700000E02260002807D01468851AA54203D1CF
:107A800005686419146040685060184630BD0000F5
:107A900010480020F1B50E4C0F480C4E001B0D4F46
:107AA000C508ED0000221146009804F00DF80028EA
:107AB00003D13068002801D00020F8BD3C600020D0
:107AC0002560606001203060ECE700001448002071
:107AD000DCAF002010480020D8B10020F0B51FB462
:107AE00086B00998089A030D0021024314D051482A
:107AF000514A1818504305141198012810981AD0AB
:107B0000281A401C00264D4F4D49009601910490C3
:107B1000002812DA444211E01198012449A30128F7
:107B200001D11098C1430698119A84600360C26025
:107B300041600BB0F0BD4042E4E70446210500205F
:107B40003F4A001C51410391029012E0E00707D028
:107B500032463B4601990098FCF74AFF019100909C
